:1000000000000220BD8C0000E58C0000E78C0000A1
:10001000E98C0000EB8C0000ED8C0000000000007B
:10002000000000000000000000000000EF8C000055
:10003000F18C000000000000F38C0000F58C000043
:10004000F78C0000DD60000081900000F58B00005F
:10005000E98B0000F78C0000F78C0000F78C0000A3
:1000600049400000F78C0000F78C0000F78C00007E
:10007000F78C0000F78C0000F78C0000F78C000074
:10008000F78C000005910000F78C0000F78C000051
:10009000F78C0000F78C0000F78C0000F78C000054
:1000A000F78C0000F78C0000F78C0000F78C000044
:1000B000F78C0000F78C000000000000000000003A
:1000C000F78C0000F78C0000F78C0000F78C000024
:1000D000F78C0000F78C0000F78C0000F78C000014
:1000E000F78C00000000000000000000000000008D
:1000F00000000000F78C000000000000F78C0000FA
:1001000000000000000000000000000000000000EF
:1001100000000000000000000000000000000000DF
:1001200000000000000000000000000000000000CF
:1001300000000000000000000000000000000000BF
:1001400000000000000000000000000000000000AF
:10015000000000000000000000000000000000009F
:10016000000000000000000000000000000000008F
:10017000000000000000000000000000000000007F
:10018000000000000000000000000000000000006F
:10019000000000000000000000000000000000005F
:1001A000000000000000000000000000000000004F
:1001B000000000000000000000000000000000003F
:1001C000000000000000000000000000000000002F
:1001D000000000000000000000000000000000001F
:1001E000000000000000000000000000000000000F
:1001F00000000000000000000000000000000000FF
:1002000010B5054C237833B9044B13B10448AFF350
:1002100000800123237010BD440200200000000074
:1002200064E8000008B5034B1BB103490348AFF372
:10023000008008BD000000004802002064E80000C3
:10024000154B002B08BF134B9D46A3F5803A0021A8
:100250008B460F461348144A121A0BF0E9F90F4B5C
:10026000002B00D098470E4B002B00D09847002061
:10027000002104000D000D48002802D00C48AFF307
:1002800000800BF08DF92000290008F051FF0BF0E1
:1002900061F900BF0000080000000220000000001B
:1002A0000000000044020020BC900120000000007B
:1002B0000000000010F0010310D104280CD90368DD
:1002C000C3F30F1343B1013B9B001A1DC1180979F9
:1002D00011B101339342F9D1184670470023FBE76F
:1002E000037883B11A0601D40130704703F0C003CC
:1002F000C02B08BF0130024610460132037803F0DC
:10030000C003802BF8D0704708B5002103780BB9E3
:10031000084608BDFFF7E4FF0131F7E738B50022D2
:1003200004460D46411C092004F0C2F940B16300A7
:10033000024643F0010342F8043F0023A34200DBDE
:1003400038BD55F8231042F8041F0133F6E70128A1
:1003500038B504DC1C20BDE8384001F075BA0D68E2
:10036000EA0701D41120F6E74868C30706D4042839
:1003700004D9036803F00F03042B01D00E20EAE731
:1003800003F0FAFF6D10002D044603DDFFF7BCFFFC
:10039000A84206DA1220DEE72046FFF7A1FF013D62
:1003A0000446012DF8D120787F2808DDDF280ADCFB
:1003B0006378800100F4F86003F03F0318434000C5
:1003C00040F0010038BDEF280ADC637800039B0190
:1003D00080B203F47C630343A07800F03F00EDE7B4
:1003E000F72810DC637880041B0303F47C3300F4EB
:1003F000E0101843E37803F03F030343A078800143
:1004000000F47C60DAE74FF0FF30D8E7486838B591
:10041000C3070D4606D4042804D9036803F00F026D
:10042000092A04D00B20BDE8384001F00DBA446819
:10043000C3F30F1364105A1EA2420BD8032194FB7E
:10044000F1F16429A8BF64210329ACBF5918D91C54
:1004500004F06AF90368C3F30F13013B9C4208D20E
:10046000A31C013464002A6840F8232044F00104EE
:100470004460002038BD01282DE9F84304DC1C202D
:10048000BDE8F84301F0E0B902284E680CD08C6852
:10049000E70709D56410012CB8BF0124F50705D57D
:1004A0004FF0FF30BDE8F8830124F7E7042EF7D9B9
:1004B00033680D6803F00F02042A30D1E80706D430
:1004C000042D04D92B6803F00F03042B01D00E2058
:1004D000D6E73046FFF7EEFEA042E1DB304603F000
:1004E0004BFF0646284603F047FF03780146002BE2
:1004F000D6D0601E30440BF06AFC01460028CFD0F5
:10050000012433780BB18E4203D3640044F0010020
:10051000C8E73046FFF7E4FE01340646F1E7092A52
:1005200038D177687F10BC42BADCE90729D4042DA2
:1005300027D92B6803F00F03042B22D1284603F0A0
:100540001BFF804604F1010956F82900854203D1BA
:10055000600040F00100A5E7C2070ED404280CD9C2
:10056000036803F00F03042B07D103F005FF0146D6
:1005700040460BF0F3FB0028C7D0B9454C46E1DDFF
:100580008EE7631C56F82320AA42BED0BB421C460D
:10059000F7DD85E7032A83D1C3F30F17C3F3417354
:1005A000C3EB8707BC423FF77BAFEB0728D4042D92
:1005B00026D9286800F00F03032B17D1C0F30F13BF
:1005C000C0F3417005F10408C0EB83003F1A013C01
:1005D00040440336BC423FF763AF3219434683427F
:1005E00019460FD315D1601C4000B2E7042B07D188
:1005F000284603F0C1FE80462846FFF75BFEE5E78C
:100600000F203DE712F8015F09788D4203F10103E5
:10061000E5D00134DEE7000001282DE9F0470E4661
:1006200004DC1C20BDE8F04701F00EB90868C207E1
:1006300006D4042804D9036803F00F03042B01D067
:100640000E20EFE74B6813F00109F9D1042BF7D91D
:100650001B6803F00F03042BF2D103F08DFE044658
:10066000706803F089FE82460BF082FB804670B909
:100670002046FFF749FE05460122A918092004F08B
:1006800017F8354F386098B90020BDE8F08751461B
:1006900020460BF09CFB231A5D425D4120466F1CF7
:1006A0000028E9D0514640440BF091FB3D46F6E767
:1006B0006B0043F001034360B8F1000F19D12046ED
:1006C000FFF70EFE4D45064601DC3868DDE7311BBD
:1006D000204604F06EF80028D6D009F102023B68EB
:1006E00043F822003046FFF7FBFD09F101093446CB
:1006F000E8E7012D02D133688360C6E75146204602
:100700000BF065FB01268146B9F1000F14D0B5420C
:10071000DBDBA9EB0401204604F04BF80028B3D042
:100720003B68013609EB080443F826005146204691
:100730000BF04DFB8146E7E7B542C6DB20460BF0E8
:1007400017FB0146204604F034F800289CD00136FF
:100750003B6843F82600B8E7746D012008B503F044
:10076000EFFD400040F0010008BDC30711D404288C
:100770000FD9026802F00F03032B0AD101F0030323
:10078000C3F104035B0703F0C04322F0C0421343EC
:1007900003607047002838B504DC1C20BDE83840F1
:1007A00001F052B80C68E50701D40D20F6E70128E6
:1007B0001CD04B68DA07F8D55B10FF2B01D913204A
:1007C000ECE71A0442EA03621A4342EA0322641085
:1007D00024EAE474E11C8910032003F069FF054654
:1007E00010B12146FFF7C1FF284638BD0022EEE7D1
:1007F00001282DE9F0470546884604DC1C20BDE8A9
:10080000F04701F021B84C6814F0010701D10D2028
:10081000F5E7022802D08B68DA07F8D5D8F800602F
:10082000F30700F1A980042E40F2A680326864101C
:10083000012C02F00F03B8BF0124092B28D17668E0
:10084000022D4FEA660605D0D8F808305B109E42AC
:10085000A8BF1E46351B0135012225EAE575A918FA
:10086000092003F025FF074648B16D00034645F017
:100870000105D8F8002043F8045FA64202DA3846A2
:10088000BDE8F087013452F8241043F8041FF4E760
:10089000042B43D1304603F06FFDFFF735FD022DE9
:1008A000824605D0D8F808305B109842A8BF9A4617
:1008B000A24504DA0020BDE8F04703F073BF3046DC
:1008C00003F05AFD0546A74222DB304603F054FDF3
:1008D000A94606462846FFF703FD0134A245054612
:1008E000F8DAA0EB0905284603F05CFF074600286C
:1008F000C5D003F041FD0446D8F8000003F03CFDEC
:10090000A9EB060101442A4620460AF06DFEB6E72F
:100910002846FFF7E5FC01370546D4E7032B2BD12A
:10092000C2F30F13022DC2F34172C2EB830205D052
:10093000D8F808305B109A42A8BF1A46A24206DADD
:10094000002211460320BDE8F04703F0B1BE151B9D
:100950000423291D002291FBF3F1032003F0A8FEDC
:10096000074600288BD001352946FFF7FEFEE11C23
:100970002A4631440430C8E7212040E70028F8B572
:1009800004DC1C20BDE8F84000F05EBF0C6814F0E9
:10099000010711D06410FF2C01D91320F2E70022C7
:1009A0000121032003F084FE054618B10121FFF761
:1009B000DCFE04712846F8BD042CEED9256805F04C
:1009C0000F05042D19D12046FFF774FC3A46C11CCF
:1009D000064691FBF5F1032003F06AFE0546002868
:1009E000E8D03146FFF7C1FE204603F0C5FC324691
:1009F0000146281D0AF0F8FDDCE7092D1DD16668C7
:100A000076100423F11C3A4691FBF3F1032003F026
:100A10004FFE05460028CDD03146FFF7A6FE043430
:100A2000B742C7DA54F8043FDA0704D55B10FF2B4E
:100A3000B3D8EA1913710137F2E7032DADD125467A
:100A4000B8E77F2902DC017001307047B1F5006F13
:100A50000CDA03468A1162F03F0203F8022B01F020
:100A60003F0161F07F01417018467047B1F5803F4A
:100A70000FDA0B1363F01F030370C1F3851301F04A
:100A80003F0163F07F0361F07F01437081700330A9
:100A90007047B1F5883F0DDAF0230370902343705F
:100AA0008B1101F03F0163F07F0361F07F018370E0
:100AB000C1700430704710B510F0010402D044102A
:100AC000204610BD042812D9026802F00F02042A41
:100AD00007D103F051FC0A222146BDE810400BF07B
:100AE0000BBA032A03D10A2221460430F5E70D2070
:100AF00000F0AAFEE4E7000000282DE9F7430F46C6
:100B000003DC1C2000F0A0FE16E00C6814F00105C8
:100B100006D1042C1FD9236803F00F03042B0DD139
:100B20002046FFF7C8FF6C4601462046FFF789FFC5
:100B3000011B204603F03DFE044635E0092B0AD197
:100B40006668DFF8849076104FF00108B04504DD48
:100B500000F080FED8B12A20D4E708F1010854F84B
:100B60002800FFF7A8FF7F280BDDB0F5006F0ADB38
:100B7000B0F5803F09DB4845D4BF04200020054480
:100B8000E4E70120FBE70220F9E70320F7E7284626
:100B900003F008FE044638B1D7F8008003F0ECFB00
:100BA00001250746B54203DD204603B0BDE8F083CA
:100BB000013558F82500FFF77EFF01463846FFF75C
:100BC00040FF0746EEE700BFFF0F01000128F8B520
:100BD00007460D4604DC1C20BDE8F84000F034BE9A
:100BE0000868FFF768FF06466868FFF764FF022F92
:100BF000044606D0A868FFF75EFF051E02DC292028
:100C0000EAE70125A642D5BFA41B341B94FBF5F4EB
:100C100094FBF5F4D4BF013401344FF0000204F129
:100C200001014FF00900C8BF6D4203F041FD50B112
:100C30006200034642F0010243F8042F6D00760083
:100C40000022944200DCF8BD46F0010143F8041F85
:100C500001322E44F5E710B5044611F0010011D120
:100C600004290ED90B6803F00F03042B09D10846A1
:100C700003F082FB014620460BF070F8B0FA80F0DA
:100C8000400910BD0020FCE70128F8B50D4604DC42
:100C90001C20BDE8F84000F0D7BD4E68F20706D42E
:100CA000042E04D9336803F00F02092A01D00B2067
:100CB000EFE7746809686410C3F30F13A34298BF89
:100CC00003F1FF3411F001070DD0481000283ADD80
:100CD000844238DB06EB8003844218DD9A6843F8CF
:100CE000042F0130F8E71A48FFF7B5FF40B10123A0
:100CF000BC4201DA0020F8BD013746F82730F7E79B
:100D000029681448FFF7A7FF50B1002CF2D0012248
:100D1000631C013C9440144346F823207460E9E7C7
:100D20002868C30711D404280FD9036803F00F0300
:100D3000042B0AD1FFF7BFFE0028C8D12968064856
:100D4000FFF789FF08B11220A3E71120A1E700BF38
:100D5000EFCC0000F3CC0000F8CC0000002310B56D
:100D60000B70C3070C4606D50E4942102046BDE85D
:100D700010400AF0B7BF28B90B492046BDE8104023
:100D80000AF0D0BF042801D10849F6E709D9036861
:100D900003F00F03042B04D103F0EEFA04490246DA
:100DA000E4E710BDB8D90000FACC000000CD000087
:100DB00005CD00002DE9F04301288FB081460E4695
:100DC00007DC1C2000F040FD054628460FB0BDE8BA
:100DD000F0830B6813F0010440F0A180042B40F273
:100DE000D5801B6803F00F03092B40D1274656F826
:100DF000273013F0010806D1042B04D9186800F03D
:100E00000F00092801D02220DCE75B680137B945D3
:100E100004EB6304EBD10122A11803F049FC054661
:100E200008B90025D1E7640044F00104446042465B
:100E300000F1080456F822104B6808685B10C0F3F4
:100E40000F10984298BF00F1FF3304310020834215
:100E500007DC013223EAE373BA4204EB8304E9DBE3
:100E6000B3E751F804CF44F820C00130EFE7032B7B
:100E700040F08C80274656F8270010F00108C2D1B8
:100E80000428C0D9036803F00F02032A38D1C3F342
:100E90000F12C3F34173C3EB82031C440137B945FE
:100EA000E9D10423E11C002291FBF3F1032003F0BC
:100EB000FFFB05460028B4D02146FFF756FC00F1A1
:100EC000040956F82840E10720D4042C1ED92068D4
:100ED00000F00F03032B19D1C0F30F13C0F34170BF
:100EE000C0EB830003344B46A3EB0902824211DBC3
:100EF00008F101080028A8BF8144B845E1DB64E798
:100F0000042A80D1FFF7D6F90444C7E72046FFF74B
:100F1000D1F9E7E714F8012F03F8012BE4E70025E6
:100F20002C4656F82500C20732D4042830D903686D
:100F300003F00F02042A32D1FFF7BCF90444013553
:100F4000A945EED1204603F02DFC054600283FF4CC
:100F500068AF041DB04606EB890958F8046BF30727
:100F600028D4042E26D9336803F00F02042A34D182
:100F70003046FFF79FF90746304603F0FDF93A4641
:100F8000014620460AF030FB3C4421E02546C8E7F4
:100F900001A9FFF7E3FE01A80AF0EAFECEE7032A63
:100FA0007FF431AFC3F30F12C3F34173C3EB82037A
:100FB0001C44C4E701A93046FFF7D0FE01A80AF09F
:100FC000D7FE01A90646024620460AF00DFB34442E
:100FD000C145C2D100232370F7E6032AF8D1C3F339
:100FE0000F17C3F34173C3EB87073A46311DC8E7B8
:100FF0002DE9F04F002893B00F4607DC1C2000F0CD
:1010000023FC0546284613B0BDE8F08F0D6815F0A7
:10101000010806D1042D04D92B6803F00F03092B16
:1010200001D00B20EBE76E687610002E03DC404603
:1010300003F0B8FBE5E7012826D04868C20723D4AF
:10104000042821D9036803F00F03042B1CD103F0FB
:1010500093F9044620460AF08BFE0435731E814640
:10106000009303FB00FB05EB860A55F8040FC3074A
:1010700071D404286FD9036803F00F02042A05D144
:10108000FFF718F983440AE0384CE3E7032A69D1F3
:10109000C3F30F12C3F34173C3EB82039B44AA450E
:1010A000E3D1584603F07EFB05460028AAD0D7F8C6
:1010B00000A0B9F1000F03D0786803F05DF9044691
:1010C000284603F059F90AF1040307460193019BEE
:1010D00053F804AF0193504603F04EF91AF00103A0
:1010E0000146029302D1BAF1040F04D805A9504673
:1010F000FFF734FE05A9084603910AF039FEDDE941
:10110000023183468BB9BAF1040F0ED9DAF8000028
:1011100000F00F0CBCF1030F01BFC0F30F13C0F3BD
:1011200041700AF10401C0EB830B38465A460AF0BD
:101130005BFA5F44B9F1000F08D0009B434505DD21
:1011400038464A4621460AF04FFA4F4408F1010852
:101150004645BCD156E705A9FFF700FE05A80AF0F1
:1011600007FE8FE703F008F9F9E700BF4BD2000054
:10117000021E10B513DD0B6813F001041CBF5C10D8
:1011800024EAE474012A00D04A68611C092003F0B3
:101190008FFA18B1640044F00104446010BD0024CB
:1011A0000122F2E70A6838B512F0010436D1042AA8
:1011B00034D91368496803F00F00092818D1506822
:1011C000C3F30F134010834298BF03F1FF30151D86
:1011D000A04205DC01330220984205DB002038BD27
:1011E00045F8041F0134F3E742F820100130F3E71B
:1011F000032813D1C80704D41320BDE8384000F0F9
:1012000023BB4910FF29F7D80432C3F30F1302EBB5
:1012100083039A42E2D202F8011BFAE70B2000F0A6
:1012200013FBDBE72DE9F0414E6816F00107884615
:1012300029D1042E27D9326802F00F03092B12D1CD
:101240007068C2F30F124510AA4200D8551ED8F894
:10125000008018F0010F1AD04FEA6804002C49DD15
:10126000A54220DA46E0042B04D13046FFF722F8ED
:101270000546ECE7032B08D1C2F30F10C2F341720D
:10128000C2EB8005E3E70025E1E73D46DFE74146A5
:101290003248FFF7E0FCA8B10AF0BCFC90FBF5F384
:1012A00003FB1500441C002F55D1042E53D933687D
:1012B00003F00F03092B26D1013456F824402046B1
:1012C000BDE8F08141462648FFF7C5FCC8B9B8F132
:1012D000040F11D9D8F8003003F00F03042B0BD101
:1012E0004046FFF7E8FB041EB9D141461D48FFF711
:1012F000B2FC08B1122000E01120BDE8F04100F07E
:10130000A3BA2C46CFE7042B1DD1304603F034F8A6
:10131000012C05460FDCFEF7E3FF461B304603F0C9
:1013200041FA04460028CAD003F026F8324629467E
:101330000AF05AF9C3E72B78013C002BDAD0284693
:10134000FEF7CEFFE4E7032B05D13444E4786400D4
:1013500044F00104B3E70B20CFE700BFE8CC000066
:10136000F3CC0000F8CC00002DE9F0414C6814F0FB
:10137000010788462ED1042C2CD923688E6803F0EF
:101380000F02092A13D16568C3F30F136D10AB4226
:1013900000D85D1ED8F800103448FFF75CFC68B335
:1013A000236803F00F03092B1ED1012317E0032A42
:1013B00010D1F20704D41320BDE8F04100F044BA84
:1013C0007710FF2FF7D8C3F30F15C3F34173C3EBA7
:1013D0008505DFE70B20EFE7013344F823609D42EA
:1013E000FADA0020BDE8F081032BFAD1033401239F
:1013F0009D42F6DB04F8017F0133F9E7D8F800805D
:1014000018F0010F0ED04FEA6800002822DD854257
:1014100020DB236803F00F03092B21D1013044F8AE
:101420002060DEE741461248FFF715FCB0B9B8F17D
:10143000040F11D9D8F8003003F00F03042B0BD19F
:101440004046FFF738FB0028E0D141460948FFF746
:1014500002FC08B11220AFE71120ADE72846D8E71B
:10146000032B04BF2418E770BBE700BFEFCC0000DC
:10147000F3CC0000F8CC0000086808B5C3071BD403
:10148000042819D9036803F00F02092A01D1406822
:1014900008BD032A09D1C3F30F12C3F34170C0EB97
:1014A0008200400040F00100F2E7042A04D102F07B
:1014B00063FFFEF729FFF4E70120E9E7024A03484A
:1014C0000E2104F0F9BE00BF78CC000070CC000003
:1014D000002070470420704701207047002003F06F
:1014E00061B900207047002070470020704700203D
:1014F0007047002070470020704700207047002090
:101500007047002070470000024A03480D2104F094
:10151000D3BE00BF90CD0000F8CD00007047037827
:1015200083B11A0601D40130704703F0C003C02B09
:1015300008BF0130024610460132037803F0C003B1
:10154000802BF8D070470000F8B511F00105064671
:101550001446084626D104293FD90B6803F00F032F
:10156000042B3AD1D30714D4042A36D9136803F0D4
:101570000F03042B31D102F0FFFE0546204602F096
:10158000FBFE014628460AF0E9FB00282DDB1ED1B0
:1015900026E002F0F1FE29460A220AF0ADFC0546DB
:1015A000601011E012F0010715D1042A15D9136853
:1015B00003F00F03042B10D110464D1002F0DCFE97
:1015C0000A2239460AF098FC85420EDB08DD002E1F
:1015D00009DC00200CE04D10E2E7064B0F221A70E8
:1015E0000136022EF5D8042002E0701700F0040046
:1015F000F8BD00BF840200202DE9F0412E4F0646C1
:101600000024E500EB191B79032B0AD00134FF2CD1
:10161000F7D1304604F064FE002808BF4FF0FF30D9
:1016200048E030460AF0A4FB31460246E0B204F03E
:10163000DFFE00283CD1E9594A680B1D9042E5D0F5
:1016400053F8045FF02D00F10100F7D1800000F1A4
:101650000803CA18D007D9D4042AD7D9CB5803F025
:101660000F010429D2D1C3F30F13013302EB83001E
:10167000C507CBD40428C9D952F8233003F00F038F
:10168000042BC3D102F078FE4FF003080546092170
:1016900028460AF056FB0028B8D0B8F1010800F13E
:1016A0000105F4D1314628460AF091FB8542ADD1BF
:1016B00064F0FF00BDE8F0819086012010B510F0C5
:1016C000010402D04410204610BD042812D902683B
:1016D00002F00F02042A07D102F04EFE0A22214630
:1016E000BDE810400AF008BC032A03D10A222146B3
:1016F0000430F5E7014B0D221A70E4E78402002064
:1017000010F0010210B516D1042802D90268C2F304
:101710000F1211F0010310D1042902D90B68C3F391
:101720000F13934216D1043000EB83020331904231
:1017300005D301200BE00022EBE70023F1E710F8CE
:10174000014B11F8013F1CB9B3FA83F0400910BDF9
:101750009C42ECD00020FAE72DE9F74F80468946FD
:101760009A46304F304E6AB102233B7001233360FA
:101770003368DFF8D0B00024FC54444504DB03B0E8
:10178000BDE8F08F3260F3E759F824003168C307F1
:1017900007EB0105C1F5487105D5244A43102846D9
:1017A0000AF06CFA04E0C8B9214A28460AF066FA41
:1017B0001C480AF0DDFA3060BAF1000F0CD008F1D5
:1017C000FF33A34208DDB0F5487F05D2431C202239
:1017D0003A540022FA5433600134CEE7042801D190
:1017E000144AE2E71BD9026802F00F03042B06D16A
:1017F000019102F0C1FD104A01990346CFE7092B80
:1018000003D143685A465B10C9E7032B08D1C2F3E2
:101810000F13C2F34172C2EB8303084ABFE70123EF
:10182000074ABCE785020020A8050020B8D90000BF
:10183000FACC000000CD0000E7DF00007FD0000000
:101840008AD0000070D00000014B18700020704753
:1018500084020020024B1878003018BF0120704726
:101860008402002008B500231A46FFF775FF034BDA
:101870000348196805F036FA002008BDA8050020C5
:101880008502002010B502F0A1FA084C231D014684
:101890001F2218460AF086FA0AF06AFA0430800815
:1018A000000140F004002060204610BD60020020CE
:1018B0002DE9F04F85B000F1180104690291D0E9DB
:1018C0000232824601EB8404BC4F4169029800EB6E
:1018D0008109397803EB820529BB53F82230B84AD5
:1018E0001E1203F07F03043552F82330904643F074
:1018F000010318479AF8010005F0D2F900238AF88D
:10190000003021E03B7873B92B681E1203F07F038F
:10191000043558F82330EAE7029A231D9A1AD82A88
:1019200026DD1A233B70DAF808209AF8023039785D
:101930009AF80100AA1A921043EA022205F0B6F9B9
:1019400000238AF800303B70DAF80830ED1A029B69
:10195000E41AA9EB0309AD10A4104FEAA903CAF8D1
:101960000C50CAF81040CAF8143005B0BDE8F08F2A
:1019700022461C463B781660002BD4D12B681E12E1
:1019800003F07F03043558F82330B0E7029A231D93
:101990009A1AD82A02DD1A233B70C4E721461C4656
:1019A0002B680B603B782A1D0BB11546BBE76B68B3
:1019B0001E1203F07F03083558F8233097E7029A88
:1019C000231D9A1AD82A02DD1A233B70ABE7224660
:1019D0001C463B7805EB86061660002BA3D12B68CE
:1019E0001E1203F07F03043558F823307FE7029A74
:1019F000231D9A1AD82A02DD1A233B7093E7224648
:101A00001C46704B53F8263013603B78002B8AD16C
:101A10002B681E1203F07F03043558F8233066E765
:101A2000684B54F8042D43F826203B78002B7FF4B4
:101A30007AAF2B681E1203F07F03043558F8233069
:101A400055E7DFF880B15BF82600FFF737FE3A78FC
:101A50005AB9009054F8040DFFF730FE009B18446B
:101A6000400040F001004BF826003B78002B7FF44B
:101A70005AAF2B681E1203F07F03043558F8233049
:101A800035E7029B221DD31AD82B02DD1A233B70A7
:101A900049E7029B21464B4534BF59F80C3C0123D2
:101AA0000B603B781446002B7FF43DAF2B681E1271
:101AB00003F07F03043558F8233018E7029B221DFA
:101AC000D31AD82B02DD1A233B702CE7029B4B451F
:101AD00018D259F80C3C06F180465B10C3EB8373B7
:101AE000033E334459F8233023603B781446002BDF
:101AF0007FF419AF2B681E1203F07F03043558F8EA
:101B00002330F4E618233B700023EDE7029B4B459E
:101B100018D259F80C3C54F8042D5B1006F180469D
:101B2000C3EB8373033E334449F823203B78002BF7
:101B30007FF4F9AE2B681E1203F07F03043558F8CA
:101B40002330D4E618233B70F0E7029B4B4529D2A3
:101B500059F80C3C06F180465B10033EC3EB8373DF
:101B6000334459F82300FFF7A9FD834654F8040DC8
:101B7000FFF7A4FD59F80C3C5B10C3EB837358448A
:101B80001E44400040F0010049F826003B78002B3D
:101B90007FF4C9AE2B681E1203F07F03043558F89A
:101BA0002330A4E618233B70F0E7029A231D9A1A0B
:101BB000D82A09DD1A233B70B5E600BF8402002055
:101BC00070CE0000888E012022461C4659F826302F
:101BD00013603B78002B7FF4A6AE2B681E1203F037
:101BE0007F03043558F8233081E654F8043D49F862
:101BF00026303B78002B7FF496AE2B681E1203F044
:101C00007F03043558F8233071E659F826004FEA6F
:101C1000600B54F8040DFFF751FD584440003B7829
:101C200040F0010049F82600002B7FF47CAE2B68C1
:101C30001E1203F07F03043558F8233057E6029B49
:101C4000A4EB8604A3420BD83B78002B7FF46BAE49
:101C50002B681E1203F07F03043558F8233046E644
:101C6000C84802F079FB3B78002B7FF45CAE2B6810
:101C70001E1203F07F03043558F8233037E6002E98
:101C800005EB8605FFF660AE3B78002B7FF44BAE8C
:101C90002B681E1203F07F03043558F8233026E624
:101CA00054F8043D042B04D1002E05EB8605FFF605
:101CB0004BAE3B78002B7FF436AE2B681E1203F040
:101CC0007F03043558F8233011E654F8043D042B03
:101CD00004D0002E05EB8605FFF636AE3B78002BD0
:101CE0007FF421AE2B681E1203F07F03043558F8F1
:101CF0002330FCE554F8040CC307A4F1040B0BD506
:101D00004010013800280ADB400040F0010005EBDC
:101D10008605CBF8000017E6FFF7D0FCF1E73B782B
:101D20000BB15C46FFE52B681E1203F07F035C4697
:101D300058F823300435DAE5029A029B04F10C0BC3
:101D4000ABEB0202A9EB0303D82A4FEAA30302DD9F
:101D50001A233B70E7E5A146740004F4FF7646F0D1
:101D60000106C9F80060DAF808209AF80200AD1AF6
:101D7000AD1040EA052040005B0043F0010340F055
:101D80000100C9F80400C9F808303A788AF802E07E
:101D900051F83C30CAF808305C461AB103F1080526
:101DA000D946C0E503F10C059B681E1203F07F03C2
:101DB000D94658F823309AE5029B54F8046C4B45F9
:101DC0002FD1F70720D4042E17D9336803F00F035F
:101DD000042B13D1304602F0CFFA09F0C9FFB0F559
:101DE000487F28BF4FF448700630643004F046FB4B
:101DF00070B9043DDDF80890A6E507D0002E14BFA9
:101E00004FF400700720F0E70A20EEE70720ECE728
:101E100031469AF8010004F060FF00238AF8003090
:101E2000E8E759F80C3C58495A106FF00303534344
:101E30000C3B09EB030449F8036059F8083C5A10BD
:101E40008AF80220D2B2C3F3552351F83220CAF8DF
:101E5000082059F8041C4FEA6109029901EB89092D
:101E60003978043402EB830500297FF45CAD52F825
:101E700023301E1203F07F03043558F8233036E573
:101E800054F8040CFFF71AFC1E288346A4EB8604C2
:101E900025DC00280BDC3B78002B7FF444AD2B685D
:101EA0001E1203F07F03043558F823301FE501F0BC
:101EB00079FFABF1030B834401F074FF334BA0EBCC
:101EC0000B009842F8D83B78002B7FF42CAD2B68A0
:101ED0001E1203F07F03043558F8233007E5012371
:101EE0008AF8003001F05EFF0A385844CAF804004E
:101EF0002AE554F8040CFFF7E1FBA4EB8604061E68
:101F00000BDC3B78002B7FF40EAD2B681E1203F028
:101F10007F03043558F82330E9E41D4B9E4202DD6F
:101F20001D233B70FFE401238AF8003001F03AFFE3
:101F30004FF47A7303FB06000A38D7E700233046D4
:101F4000A4EB8604134E1A462146FFF705FC3168C0
:101F5000114802F02EFC114B316818600E4804F055
:101F60006DFD31680C4804F0BDFE3B78002B7FF41A
:101F7000DAAC2B681E1203F07F03043558F82330C7
:101F8000B5E400BF9CD00000908601207F969800A9
:101F900080EE3600A8050020850200200800002001
:101FA0003B78A4EB8604002B7FF4BDAC2B681E129B
:101FB00003F07F03043558F8233098E4504604F0CA
:101FC000C1FA3B78002B7FF4AEAC2B681E1203F0F5
:101FD0007F03043558F8233089E454F8043C002B7F
:101FE00044D154F80C0C10F0010B1ED04FEA600BDA
:101FF0004FEA4B0343F0010344F8083CBBF1000FE8
:1020000040F388804FEA4B0343F0010354F80C0C73
:1020100044F8043C54F8083CC107CBEB63032AD5D1
:1020200001335B0043F0010330E004281BD903684F
:1020300003F00F02092A01D14068D7E7042A09D129
:1020400002F09AF90378002BD2D0FFF768FA0BF16F
:10205000010BF7E7032A06D1C3F30F1BC3F3417348
:10206000C3EB8B0BC4E719233B705CE44FEA630BB3
:102070000BF1FF3BC2E7042849D9026802F00F02C6
:10208000092A11D103F1020B50F82B3049F8263000
:102090003B78002B7FF447AC2B681E1203F07F03C4
:1020A000043558F8233022E4042A2BD1039309EB9A
:1020B0008603009302F060F9039B83465E1C012EA9
:1020C00012DC5846FFF72BFAA0EB0B06304602F065
:1020D00069FB034670B1039002F04EF9324659464F
:1020E00009F082FA039B05E09BF80030013E23B91A
:1020F00012223A70009A1360CAE75846FFF70FFAA7
:102100008346DCE7032A02D11844037989E71923BF
:102110003B7008E40435BBE7029A04EB86039B1A84
:10212000D82B11DC0122002E06F1FF3310DC3B78A6
:10213000002B7FF4F8AB2B681E1203F07F030435ED
:1021400058F82330FFF7D3BB1A233B70FFF7EBBBE4
:1021500022601E460434E6E7029A231D9B1AD82B00
:1021600003DD1A233B70FFF7DEBB029B4B452AD2EF
:1021700054F8040CFFF7A2FA002821DD59F80C3CB2
:102180005B1083421CDBC3EB8373184400F1804077
:102190000438A4EB860359F820201A606FF003007E
:1021A0003B7800FB06440434002B7FF4BCAB2B6867
:1021B0001E1203F07F03043558F82330FFF797BB56
:1021C00020233B70EAE71823FBE7C04B1A68A4EB17
:1021D00086036FF003001A603B7800FB064404346A
:1021E000002B7FF4A0AB2B681E1203F07F03043595
:1021F00058F82330FFF77BBB54F8043C042B3B78A2
:10220000A4F1040204BF05EB8605224613B114466F
:10221000FFF789BB2B681E1203F07F03144658F8A2
:1022200023300435FFF763BB54F8043D042B1CBF77
:10223000002323603B781CBF05EB86050434002B8C
:102240007FF471AB2B681E1203F07F03043558F83E
:102250002330FFF74CBB002EA4EB860115DC1C23BA
:102260003B7000226FF003003B780A6000FB0644DD
:102270000434002B7FF457AB2B681E1203F07F034E
:10228000043558F82330FFF732BB0B684FF0000CD1
:102290005B1051F82C0010F0010202D10D233B70AD
:1022A000E0E7401083420CF1010CA8BF03466645ED
:1022B000EFDC5B0043F00102D4E7002EA4EB8601C3
:1022C00015DC1C233B7000226FF003003B780A6092
:1022D00000FB06440434002B7FF425AB2B681E1250
:1022E00003F07F03043558F82330FFF700BB0B6879
:1022F0004FF0000C5B1051F82C0010F0010202D1DD
:102300000D233B70E0E7401083420CF1010CB8BF95
:1023100003466645EFDC5B0043F00102D4E754F866
:10232000081C11F0010F4FEA86031ED054F8042C4C
:10233000D0071AD55210B2EB610FA4EB0303D4BF40
:10234000002204221A606FF003003B7800FB064471
:102350000434002B7FF4E7AA2B681E1203F07F03DE
:10236000043558F82330FFF7C2BA54F8042C6FF044
:102370000100A4EB030BFFF7E7F8CBF80000E2E75E
:1023800054F8081C11F0010F4FEA86031ED054F8D0
:10239000042CD0071AD55210B2EB610FA4EB030343
:1023A000B4BF002204221A606FF003003B7800FBE8
:1023B00006440434002B7FF4B6AA2B681E1203F0E7
:1023C0007F03043558F82330FFF791BA54F8042CF2
:1023D0004FF0FF30A4EB030BFFF7B6F8CBF800008B
:1023E000E2E754E9020181424FEA860314D1E31A7D
:1023F00004221A606FF003003B7800FB06440434AB
:10240000002B7FF490AA2B681E1203F07F03043583
:1024100058F82330FFF76BBA0428A4EB030B01D85C
:10242000002315E0C307FBD4036803F00F03042B5C
:10243000F6D1CB07F4D40429F2D90B6803F00F03CB
:10244000042BEDD1FFF75CF900280CBF0023042317
:10245000CBF80030CEE754E9020181424FEA86030F
:1024600014D1E31A00221A606FF003003B7800FBDE
:1024700006440434002B7FF456AA2B681E1203F086
:102480007F03043558F82330FFF731BA0428A4EB52
:10249000030B01D8042315E0C307FBD4036803F042
:1024A0000F03042BF6D1CB07F4D40429F2D90B681F
:1024B00003F00F03042BEDD1FFF722F900280CBF26
:1024C00004230023CBF80030CEE700BF0800002033
:1024D00054F8081C11F0010F4FEA86031ED054F87F
:1024E000042CD0071AD55210B2EB610FA4EB0303F2
:1024F000CCBF002204221A606FF003003B7800FB7F
:1025000006440434002B7FF40EAA2B681E1203F03D
:102510007F03043558F82330FFF7E9B954F8042C49
:102520000120A4EB030BFFF70FF8CBF80000E3E763
:1025300054F8081C11F0010F4FEA86031ED054F81E
:10254000042CD0071AD55210B2EB610FA4EB030391
:10255000ACBF002204221A606FF003003B7800FB3E
:1025600006440434002B7FF4DEA92B681E1203F00E
:102570007F03043558F82330FFF7B9B954F8042C19
:102580000220A4EB030BFEF7DFFFCBF80000E3E72C
:1025900054F8043C042BA4EB860314BF042200224D
:1025A0001A606FF003003B7800FB06440434002BF4
:1025B0007FF4B9A92B681E1203F07F03043558F885
:1025C0002330FFF794B954F8080CFFF777F88346E7
:1025D00054F8040CFFF772F85844A4EB860340004B
:1025E00040F0010018606FF003003B7800FB0644E8
:1025F0000434002B7FF497A92B681E1203F07F038D
:10260000043558F82330FFF772B954F8080CFFF777
:1026100055F8834654F8040CFFF750F8ABEB000074
:10262000A4EB8603400040F0010018606FF0030047
:102630003B7800FB06440434002B7FF474A92B681C
:102640001E1203F07F03043558F82330FFF74FB90B
:1026500054F8080CFFF732F8834654F8040CFFF7DF
:102660002DF800FB0BF0A4EB8603400040F00100C6
:1026700018606FF003003B7800FB06440434002B25
:102680007FF451A92B681E1203F07F03043558F81C
:102690002330FFF72CB954F8040CFFF70FF88346EA
:1026A000B8B91F233B70A4EB86036FF00300C3F897
:1026B00000B03B7800FB06440434002B7FF433A9C0
:1026C0002B681E1203F07F03043558F82330FFF700
:1026D0000EB954F8080CFEF7F1FF90FBFBFB4FEA34
:1026E0004B0B4BF0010BDEE754F8040CFEF7E6FF52
:1026F0008346B8B91F233B70A4EB86036FF0030039
:10270000C3F800B03B7800FB06440434002B7FF490
:102710000AA92B681E1203F07F03043558F82330F2
:10272000FFF7E5B854F8080CFEF7C8FF90FBFBF381
:1027300003FB1B0B4FEA4B0B4BF0010BDCE754F890
:10274000040CFEF7BBFF0028B8BF4042A4EB860391
:10275000400040F0010018606FF003003B7800FB80
:1027600006440434002B7FF4DEA82B681E1203F00D
:102770007F03043558F82330FFF7B9B8012EA4EBD6
:10278000860B32D1DBF80000FEF798FF02460028E6
:10279000B4BF4FF0FF330123934202DC11461A46C7
:1027A0000B4601339B1A0392009309F033FA009B06
:1027B000039A90FBF3F101FB130313445B0043F016
:1027C0000103CBF800306FF003003B7800FB0644B8
:1027D0000434002B7FF4A7A82B681E1203F07F039C
:1027E000043558F82330FFF782B8022E0BD1DBF8FE
:1027F0000000FEF763FF0090DBF80400FEF75EFFC9
:10280000009B0246C8E764230122CAE7A4EB860BBB
:102810005946304602F023F93B78CBF800006FF0C0
:10282000030000FB06440434002B7FF47CA82B68D3
:102830001E1203F07F03043558F82330FFF757B812
:1028400054F8080CFEF73AFF834654F8040CFEF7E0
:1028500035FF0BEA0000A4EB8603400040F00100C6
:1028600018606FF003003B7800FB06440434002B33
:102870007FF459A82B681E1203F07F03043558F823
:102880002330FFF734B854F8080CFEF717FF8346DF
:1028900054F8040CFEF712FF4BEA0000A4EB860389
:1028A000400040F0010018606FF003003B7800FB2F
:1028B00006440434002B7FF436A82B681E1203F064
:1028C0007F03043558F82330FFF711B854F8080C8B
:1028D000FEF7F4FE834654F8040CFEF7EFFE8BEA95
:1028E0000000A4EB8603400040F0010018606FF088
:1028F00003003B7800FB06440434002B7FF413A84C
:102900002B681E1203F07F03043558F82330FEF7BE
:10291000EEBF54F8040CFEF7D1FEC043A4EB8603CF
:10292000400040F0010018606FF003003B7800FBAE
:1029300006440434002B7EF4F6AF2B681E1203F01D
:102940007F03043558F82330FEF7D1BF54F8080C44
:10295000FEF7B4FE834654F8040CFEF7AFFE0BFA04
:1029600000F0A4EB8603400040F0010018606FF017
:1029700003003B7800FB06440434002B7EF4D3AF05
:102980002B681E1203F07F03043558F82330FEF73E
:10299000AEBF54F8080CFEF791FE834654F8040CC1
:1029A000FEF78CFE4BFA00F0A4EB8603400040F0EB
:1029B000010018606FF003003B7800FB064404340C
:1029C000002B7EF4B0AF2B681E1203F07F0304359A
:1029D00058F82330FEF78BBF54F80C0CFEF76EFE50
:1029E000834654F8080CFEF769FE8BFB002354F86D
:1029F000040CCDE90023FEF761FEDDE90023C0F100
:102A0000200CB0F1200103FA0CFC22FA00F040EA9D
:102A10000C005CBF43FA01F10843A4EB860E4000B2
:102A200040F00100CEF800003B786FF0030000FB9F
:102A300006440434002B7EF476AF2B681E1203F09C
:102A40007F03043558F82330FEF751BFA4EB860B03
:102A500059463046FEF78CFB3B78CBF800006FF010
:102A6000030000FB06440434002B7EF45CAF2B68AB
:102A70001E1203F07F03043558F82330FEF737BFEA
:102A8000A4EB860421463046FEF78CFB3B78002BF6
:102A90007EF449AF2B681E1203F07F03043558F80B
:102AA0002330FEF724BFA4EB860B59463046FEF7D1
:102AB000B9FB3B78CBF800006FF0030000FB064445
:102AC0000434002B7EF42FAF2B681E1203F07F031B
:102AD000043558F82330FEF70ABFA4EB86042146DC
:102AE0003046FEF741FC3B78002B7EF41CAF2B6890
:102AF0001E1203F07F03043558F82330FEF7F7BEAB
:102B0000A4EB860B59463046FEF7B6FC3B78CBF873
:102B100000006FF0030000FB06440434002B7EF439
:102B200002AF2B681E1203F07F03043558F82330E0
:102B3000FEF7DDBE54F8040C01F01EFC54F8083C0E
:102B4000DA072AD4042B0CD91B6803F00F03013BCE
:102B5000082B10D8DFE803F0052127230F0F0F0FF4
:102B60002500CC4909F0FAF8A4EB8603002814BF2D
:102B7000002204221A606FF003003B7800FB064439
:102B80000434002B7EF4CFAE2B681E1203F07F03BB
:102B9000043558F82330FEF7AABEBF49E2E7BF4923
:102BA000E0E7BF49DEE7BF49DCE7029B261DF31AD9
:102BB000D82B03DD1A233B70FEF7B5BE01F0FAF8FF
:102BC0002346400040F0010018603B783446002B5B
:102BD0007EF4A9AE2B681E1203F07F03043558F86B
:102BE0002330FEF784BE029B261DF31AD82B03DD8B
:102BF0001A233B70FEF797BE01F0D4F8AA4B224689
:102C000003EA40003B7840F0010034461060002B9E
:102C10007EF489AE2B681E1203F07F03043558F84A
:102C20002330FEF764BE029B261DF31AD82B03DD6A
:102C30001A233B70FEF777BE01F0BCF89B4B1B6874
:102C400098423DBFC3F5830303F63713C018C01A7B
:102C50004000234640F0010018603B783446002BCA
:102C60007EF461AE2B681E1203F07F03043558F822
:102C70002330FEF73CBE01F09DF88C4B18603B788A
:102C8000A4EB8604002B7EF44EAE2B681E1203F0DC
:102C90007F03043558F82330FEF729BE03F0DAFB32
:102CA000B30068B9E41A3B78002B7EF43CAE2B6885
:102CB0001E1203F07F03043558F82330FEF717BEC9
:102CC000304627467A4EE41A01231A462146FEF77B
:102CD00043FD3068643003F0D1FB18B9043D3C4635
:102CE000FEF732BE9AF801203168724804F00DF800
:102CF00001238AF8003001F055F86F4A33681268F2
:102D0000063302FB0300FFF7F1B803F0A3FBB300A7
:102D100068B9E41A3B78002B7EF405AE2B681E12CE
:102D200003F07F03043558F82330FEF7E0BD30464A
:102D300027465F4EE41A002201232146FEF70CFDD0
:102D40003068643003F09AFB0028C7D0594803F07C
:102D50005DFDCDE7FEF796FDA4EB860B3B78CBF847
:102D600000006FF0030000FB06440434002B7EF4E7
:102D7000DAAD2B681E1203F07F03043558F82330B8
:102D8000FEF7B5BD3B78A4EB8604002B7EF4CBADFB
:102D90002B681E1203F07F03043558F82330FEF72A
:102DA000A6BDA4EB860B584601F03BF83B78CBF868
:102DB00000006FF0030000FB06440434002B7EF497
:102DC000B2AD2B681E1203F07F03043558F8233090
:102DD000FEF78DBDA4EB860B584601F024F83B7836
:102DE000CBF800006FF0030000FB06440434002B16
:102DF0007EF499AD2B681E1203F07F03043558F85A
:102E00002330FEF774BDA4EB860B5946304600F024
:102E100093FC3B78CBF800006FF0030000FB064406
:102E20000434002B7EF47FAD2B681E1203F07F0369
:102E3000043558F82330FEF75ABDA4EB860420462B
:102E400000F0F4FF3B78002B7EF46DAD2B681E1272
:102E500003F07F03043558F82330FEF748BDA4EB98
:102E6000860B5946304600F0DBFB3B78CBF8000080
:102E70006FF0030000FB06440434002B7EF453ADD6
:102E80002B681E1203F07F03043558F82330FEF739
:102E90002EBD00BFACD00000B4D00000BBD00000FD
:102EA000C2D00000C7D00000FEFFFF7FB0050020A9
:102EB000A80500208502002004000020A4EB860461
:102EC000204601F0ADF83B78002B7EF42CAD2B684A
:102ED0001E1203F07F03043558F82330FEF707BDB8
:102EE0000121304601F05AF83B78002B7EF41BADEF
:102EF0002B681E1203F07F03043558F82330FEF7C9
:102F0000F6BC0021304601F049F83B78002B7EF4F6
:102F10000AAD2B681E1203F07F03043558F82330E6
:102F2000FEF7E5BCA4EB860B584600F0EFFF3B78BC
:102F3000CBF800006FF0030000FB06440434002BC4
:102F40007EF4F1AC2B681E1203F07F03043558F8B1
:102F50002330FEF7CCBCA4EB860B584600F0EAFF0A
:102F60003B78CBF800006FF0030000FB064404340C
:102F7000002B7EF4D8AC2B681E1203F07F030435BF
:102F800058F82330FEF7B3BCA4EB8604204600F0CB
:102F90009FFF3B78002B7EF4C6AC2B681E1203F01B
:102FA0007F03043558F82330FEF7A1BCA4EB860458
:102FB000204604F0BDFB3B78002B7EF4B4AC2B68BC
:102FC0001E1203F07F03043558F82330FEF78FBC40
:102FD000A4EB860B584604F095FC3B78CBF8000038
:102FE0006FF0030000FB06440434002B7EF49BAC1E
:102FF0002B681E1203F07F03043558F82330FEF7C8
:1030000076BCA4EB8604204604F0E2FA3B78002B61
:103010007EF489AC2B681E1203F07F03043558F848
:103020002330FEF764BCA4EB860B584604F0ECFAA0
:103030003B78CBF800006FF0030000FB064404343B
:10304000002B7EF470AC2B681E1203F07F03043556
:1030500058F82330FEF74BBCA4EB860421463046DB
:1030600002F046F93B78002B7EF45DAC2B681E1213
:1030700003F07F03043558F82330FEF738BCA4EB87
:1030800086042146304601F019FF3B78002B7EF480
:103090004AAC2B681E1203F07F03043558F8233026
:1030A000FEF725BCA4EB86042146304601F0DAFF8A
:1030B0003B78002B7EF437AC2B681E1203F07F03A5
:1030C000043558F82330FEF712BCA4EB86042146E1
:1030D000304601F0EDFF3B78002B7EF424AC2B68EA
:1030E0001E1203F07F03043558F82330FEF7FFBBB0
:1030F000A4EB860B5946304604F018FD3B78CBF81C
:1031000000006FF0030000FB06440434002B7EF443
:103110000AAC2B681E1203F07F03043558F82330E5
:10312000FEF7E5BBA4EB860B5946304604F006FDDE
:103130003B78CBF800006FF0030000FB064404343A
:10314000002B7EF4F0AB2B681E1203F07F030435D6
:1031500058F82330FEF7CBBBA4EB860B594630461C
:1031600004F0F4FC3B78CBF800006FF0030000FBA8
:1031700006440434002B7EF4D6AB2B681E1203F0F9
:103180007F03043558F82330FEF7B1BBA4EB860B60
:103190005946304604F0B8F83B78CBF800006FF0A1
:1031A000030000FB06440434002B7EF4BCAB2B6808
:1031B0001E1203F07F03043558F82330FEF797BB47
:1031C000A4EB86042146304602F016F83B78002B2B
:1031D0007EF4A9AB2B681E1203F07F03043558F868
:1031E0002330FEF784BBA4EB86042146304601F071
:1031F00087FF3B78002B7EF496AB2B681E1203F002
:103200007F03043558F82330FEF771BBA4EB860B1F
:103210005946304601F0EEFE3B78CBF800006FF0E7
:10322000030000FB06440434002B7EF47CAB2B68C7
:103230001E1203F07F03043558F82330FEF757BB06
:10324000A4EB86042146304601F07EFE3B78002B3D
:103250007EF469AB2B681E1203F07F03043558F827
:103260002330FEF744BB002E40F38580012E54F836
:1032700004BC44D11BF0010F4ED1BBF1040F4BD95C
:10328000DBF8003003F00F03042B45D1584601F062
:1032900073F8FEF7B1F903465A1CA4EB86046AD012
:1032A000022E49D11BF0010F3FD1BBF1040F3CD9D5
:1032B000DBF8002002F00F02092A36D1DBF8040007
:1032C000261FC0F347000122824228DD04EB800460
:1032D00023F0FF0212F5807F30D11E02B6B2064302
:1032E0004FEA262E48495FFA8EFC01EBCC031B798E
:1032F000032B3EF421AD02233B70FEF714BB022EDC
:103300000AD154F8080CC10706D4042804D903686C
:1033100003F00F03042BBAD04FF0FF33BCE70132A8
:103320005BF8221046F8041FCEE70B233B70002306
:1033300023600434FEF7F7BA0020C9E7029AA21A04
:10334000A4EB800B9210CAF81020594698472F4AD8
:10335000002313603B78CBF800000BF10404002B32
:103360007EF4E1AA2B681E1203F07F03043558F89F
:103370002330FEF7BCBA002323603B78221D13B133
:103380001446FEF7D0BA2B681E1203F07F031446D2
:1033900058F823300435FEF7AABA029BE31A9B10B3
:1033A000A4EB8604CAF810302146304603F072FAC6
:1033B0003B78002B7EF4B7AA2B681E1203F07F0324
:1033C000043558F82330FEF792BA029BE31A9B109B
:1033D000A4EB860BCAF810305946304603F05AFA6F
:1033E0003B78CBF800006FF0030000FB0644043488
:1033F000002B7EF498AA2B681E1203F07F0304357D
:1034000058F82330FEF773BA90860120746D0120BE
:103410002DE9F84F224D0023002B03F1FF3706DA88
:1034200001F07CFF03F046FB03F01EFD1927002688
:10343000DFF8788030461B4B1A68B24215DD2B68E6
:10344000194C01339342A8BF00232B60D5F800909C
:10345000F02303FB09F304EB030AE35CA346EBB19F
:10346000022B04D15046FEF723FA3B46D4E7012B4A
:103470000DD108B900F096FCF02303FB09F39B443F
:10348000DBF80420821A42459CBF0222E254F0235A
:1034900003FB09F914F80930022BE3D00136CAE71F
:1034A00000000020AC050020307D01207F969800B0
:1034B0000A4B4FF480721A60094B01211964D3F84A
:1034C00040250532C3F84825C3F84C254FF4402267
:1034D000C3F80423034B1970704700BF00E100E0FC
:1034E00000800040F705002004207047F8B5D1E9BE
:1034F000004514F001002DD015F001002AD0641011
:103500001C2C3CD81F4F6D1041F288363B5DAE42FB
:10351000A8BF2E46012B05D00121204605F09EFFB5
:1035200001233B55184B1B780BB9FFF7C1FF002D4A
:103530004FF00003154A0EDC154940F2DC50FF2520
:10354000D65CB44204BF21F81300D5540133042BD8
:10355000F6D10420F8BDD15C8C4203D10C4A22F88C
:103560001360F6E70133042BF5D10023D15CFF296A
:1035700001D1D454F2E70133042BF7D1E9E700205D
:10358000E8E700BFD8050020F70500201C00002058
:103590000E00002070B5D1E9004514F001001BD0E9
:1035A00015F0010018D064101D2C28BF1B24154EE7
:1035B000335D012B05D00121204605F04FFF01238B
:1035C0003355114B6D10A5F110029A420F4B04D9DF
:1035D0004FF0FF321A60042070BD1C600C4B0D4888
:1035E00090FBF5F018800C4B1B780BB9FFF760FFD0
:1035F0000A4B01229A64D3F848251044C3F84805C1
:10360000E9E700BFD80500209086010018000020DF
:103610000C00002020A10700F705002000800040DA
:1036200070B50C68E30704D40D20FEF70DF90120F6
:1036300070BD64101C2C14D8012814DD4B68042BB9
:1036400014BF002502250A4E335DAB4204D0294643
:10365000204605F003FF3555204605F045FF0128BB
:1036600003D00020E4E70025EDE70420E0E700BFF9
:10367000D805002070B50D680128CCBF4C68012426
:1036800015F0010042D014F001003FD06D10002D64
:1036900005DC1F4B0122C3F80825002036E064102A
:1036A0001C2CFAD81B4E335D012B05D0012120467E
:1036B00005F0D4FE012333550A22174B93FBF5F393
:1036C000053393FBF2F3154A154952F824201548A7
:1036D000120242F00312C1F810250D4AC2F810057B
:1036E000C2F814150121C2F80415A2F5A832106918
:1036F0000020C2F810054FF6FF708342A8BF0346B2
:10370000C2F840350420C2F80012116070BD00BF3D
:1037100000F00140D805002000B4C404CCE3000050
:103720000060004040A10040002802DC1C20FEF7A1
:103730008BB8012070470000F8B50B68DA07074620
:103740000D4604D40D20FEF77FF8012009E05B1040
:103750000A2B07D0062B1FD103F068FF400040F072
:103760000100F8BD05230D4A0D4E52F82340335D8C
:103770002BB10021204605F071FE00233355012FA7
:1037800006DD6B68042B03D10221204605F066FE9E
:10379000204605F06DFDE1E7E5D9D6E744D100000C
:1037A000D805002010B510F0010402D044102046C6
:1037B00010BD042812D9026802F00F02042A07D1B2
:1037C00000F0DAFD0A222146BDE8104008F094BB63
:1037D000032A03D10A2221460430F5E70D20FEF723
:1037E00033F8E4E70228F8B50C4604DC1C20BDE8F9
:1037F000F840FEF729B80868FFF7D4FF064660686E
:10380000FFF7D0FF0546A0686E4CFFF7CBFF1C2DDD
:1038100094FBF0F400F2B5826B4F7B5D012B05D079
:103820000121284605F01AFE01237B550021284678
:1038300005F03EFE002C3CD02046013800BF00BF02
:1038400000BF00BF00BF00BF00BF00BF00BF00BF80
:1038500000BF00BF00BF00BF00BF00BF00BF00BF70
:1038600000BF00BF00BF00BF00BF00BF00BF00BF60
:1038700000BF00BF00BF00BF00BF00BF00BF00BF50
:1038800000BF00BF00BF00BF00BF00BF00BF00BF40
:1038900000BF00BF00BF00BF00BF00BF00BF00BF30
:1038A00000BF00BF00BF00BF00BF00BF00BF00BF20
:1038B000C3D106F00101284605F0FAFD002C3CD0EA
:1038C0002046013800BF00BF00BF00BF00BF00BFDF
:1038D00000BF00BF00BF00BF00BF00BF00BF00BFF0
:1038E00000BF00BF00BF00BF00BF00BF00BF00BFE0
:1038F00000BF00BF00BF00BF00BF00BF00BF00BFD0
:1039000000BF00BF00BF00BF00BF00BF00BF00BFBF
:1039100000BF00BF00BF00BF00BF00BF00BF00BFAF
:1039200000BF00BF00BF00BF00BF00BF00BF00BF9F
:1039300000BF00BF00BF00BFC3D1C6F3400128468F
:1039400005F0B6FD002C41D02046013800BF00BF75
:1039500000BF00BF00BF00BF00BF00BF00BF00BF6F
:1039600000BF00BF00BF00BF00BF00BF00BF00BF5F
:1039700000BF00BF00BF00BF00BF00BF00BF00BF4F
:1039800000BF00BF00BF00BF00BF00BF00BF00BF3F
:1039900000BF00BF00BF00BF00BF00BF00BF00BF2F
:1039A00000BF00BF00BF00BF00BF00BF00BF00BF1F
:1039B00000BF00BF00BF00BF00BF00BF00BF00BF0F
:1039C000C3D103E040420F00D8050020C6F38001B8
:1039D000284605F06DFD002C3CD02046013800BF84
:1039E00000BF00BF00BF00BF00BF00BF00BF00BFDF
:1039F00000BF00BF00BF00BF00BF00BF00BF00BFCF
:103A000000BF00BF00BF00BF00BF00BF00BF00BFBE
:103A100000BF00BF00BF00BF00BF00BF00BF00BFAE
:103A200000BF00BF00BF00BF00BF00BF00BF00BF9E
:103A300000BF00BF00BF00BF00BF00BF00BF00BF8E
:103A400000BF00BF00BF00BF00BF00BF00BF00BF7E
:103A500000BFC3D1C6F3C001284605F029FD002CE4
:103A60003CD02046013800BF00BF00BF00BF00BFF0
:103A700000BF00BF00BF00BF00BF00BF00BF00BF4E
:103A800000BF00BF00BF00BF00BF00BF00BF00BF3E
:103A900000BF00BF00BF00BF00BF00BF00BF00BF2E
:103AA00000BF00BF00BF00BF00BF00BF00BF00BF1E
:103AB00000BF00BF00BF00BF00BF00BF00BF00BF0E
:103AC00000BF00BF00BF00BF00BF00BF00BF00BFFE
:103AD00000BF00BF00BF00BF00BFC3D1C6F30011CD
:103AE000284605F0E5FC002C3CD02046013800BFFC
:103AF00000BF00BF00BF00BF00BF00BF00BF00BFCE
:103B000000BF00BF00BF00BF00BF00BF00BF00BFBD
:103B100000BF00BF00BF00BF00BF00BF00BF00BFAD
:103B200000BF00BF00BF00BF00BF00BF00BF00BF9D
:103B300000BF00BF00BF00BF00BF00BF00BF00BF8D
:103B400000BF00BF00BF00BF00BF00BF00BF00BF7D
:103B500000BF00BF00BF00BF00BF00BF00BF00BF6D
:103B600000BFC3D1C6F34011284605F0A1FC002CCC
:103B70003CD02046013800BF00BF00BF00BF00BFDF
:103B800000BF00BF00BF00BF00BF00BF00BF00BF3D
:103B900000BF00BF00BF00BF00BF00BF00BF00BF2D
:103BA00000BF00BF00BF00BF00BF00BF00BF00BF1D
:103BB00000BF00BF00BF00BF00BF00BF00BF00BF0D
:103BC00000BF00BF00BF00BF00BF00BF00BF00BFFD
:103BD00000BF00BF00BF00BF00BF00BF00BF00BFED
:103BE00000BF00BF00BF00BF00BFC3D1C6F380113C
:103BF000284605F05DFC002C3CD02046013800BF73
:103C000000BF00BF00BF00BF00BF00BF00BF00BFBC
:103C100000BF00BF00BF00BF00BF00BF00BF00BFAC
:103C200000BF00BF00BF00BF00BF00BF00BF00BF9C
:103C300000BF00BF00BF00BF00BF00BF00BF00BF8C
:103C400000BF00BF00BF00BF00BF00BF00BF00BF7C
:103C500000BF00BF00BF00BF00BF00BF00BF00BF6C
:103C600000BF00BF00BF00BF00BF00BF00BF00BF5C
:103C700000BFC3D1C6F3C011284605F019FC002CC3
:103C80003CD02046013800BF00BF00BF00BF00BFCE
:103C900000BF00BF00BF00BF00BF00BF00BF00BF2C
:103CA00000BF00BF00BF00BF00BF00BF00BF00BF1C
:103CB00000BF00BF00BF00BF00BF00BF00BF00BF0C
:103CC00000BF00BF00BF00BF00BF00BF00BF00BFFC
:103CD00000BF00BF00BF00BF00BF00BF00BF00BFEC
:103CE00000BF00BF00BF00BF00BF00BF00BF00BFDC
:103CF00000BF00BF00BF00BF00BFC3D101212846E5
:103D000005F0D6FB002C3CD02046013800BF00BF98
:103D100000BF00BF00BF00BF00BF00BF00BF00BFAB
:103D200000BF00BF00BF00BF00BF00BF00BF00BF9B
:103D300000BF00BF00BF00BF00BF00BF00BF00BF8B
:103D400000BF00BF00BF00BF00BF00BF00BF00BF7B
:103D500000BF00BF00BF00BF00BF00BF00BF00BF6B
:103D600000BF00BF00BF00BF00BF00BF00BF00BF5B
:103D700000BF00BF00BF00BF00BF00BF00BF00BF4B
:103D8000C3D10020F8BD00BF04207047002802DC2A
:103D90001C20FDF759BD0B68DB0701D40D20F8E7A7
:103DA00000207047024B01221A64D3F84005704787
:103DB00000800040044B01221A64D3F840054FF400
:103DC0007A73B0FBF3F07047008000400048704702
:103DD00060D100001D20704770B5054D2B5C8B42F3
:103DE00004460E4602D005F039FB2E5570BD00BFCB
:103DF000D805002070B50024084D2646635D012BD0
:103E000008D10021204605F053FB0021204605F093
:103E100025FB665501341D2CF0D170BDD80500205E
:103E200070470F2070473B207047000070B5046852
:103E3000E20702D54568EB0704D40D20BDE87040C9
:103E4000FDF702BD64101C2C30D8194E335D012BD8
:103E500018D00121204605F001FB01231B2C33550E
:103E600010D1144BDA6E144B202AB8BF4FF0A04388
:103E700002F01F0203EB8203D3F8002742F44072E2
:103E8000C3F800270D4BD3F8082132B1D3F818211D
:103E9000002AFBD00022C3F81821A5F34A0189109B
:103EA000204605F089FA064B01221A5570BD00BF65
:103EB000D8050020CCE300000003005000C0014002
:103EC000B405002008B50846FFF7B0FF002008BD84
:103ED00013B50A4A044692E8030022686B46042A96
:103EE00083E8030019464FF0020003D101F0BAF84D
:103EF00002B010BD01F0DCF8FAE700BFD4D000003A
:103F000008B50846FFF7E4FF002008BD10B5084CCF
:103F100063792BB10021052005F0A0FA002363711D
:103F2000052005F0E1FA00280CBF0420002010BD98
:103F3000D805002010B5084CE37A2BB100210B20E6
:103F400005F08CFA0023E3720B2005F0CDFA00286F
:103F50000CBF0420002010BDD805002010B50B4A6E
:103F60000B4C0C480C490023C2F80035A2F5C832AE
:103F7000C2F810350122626042604A60C4F8003520
:103F8000C0F80035C1F8003510BD00BF00F0014099
:103F900000C0014000100240002002401C2870B503
:103FA00004460D4632D81A4E335C012B04D0012151
:103FB00005F054FA012333551C2C12D1FFF7CEFF24
:103FC000144B1A6F144B202AB8BF4FF0A04302F0D5
:103FD0001F0203EB8203D3F8002742F44072C3F8B8
:103FE00000270E4B1B5D4BB1002D40F2FF312046E8
:103FF00008BF0021BDE8704005F0DEB9291C20464D
:1040000018BF0121BDE8704005F052BA70BD00BF75
:10401000D8050020CCE3000000030050B4050020C8
:104020000368D90702D40D20FDF70EBC41680A1FB2
:10403000514251415810FFF7B1BF08B50846FFF78C
:10404000EFFF002008BD0000F8B5324CD4F848312D
:10405000ABB10023D4F84855C4F848312E4B18684A
:1040600000280CDB2D4A1178B1FA81F14909117051
:1040700005F01EFA2A4B1B882B44C4F84835254B03
:10408000D3F84C21002A37D00021264ED3F84C45D6
:10409000C3F84C113378244D33B12B68032B03D86C
:1040A000224AD05C05F004FA2B68204F01335A42B3
:1040B00002F0030203F0030358BF53422B600022B7
:1040C000042B194619D00133F81810F8010CFF28F9
:1040D00001D10122F4E702B12960012105F0E8F9DC
:1040E000012333702A68124B33F8122004F10C03B9
:1040F0001344084AC2F84C35F8BD4FF0FF3304F5BD
:104100008C44044A2B605C3400233370C2F84C4565
:10411000F2E700BF0080004018000020F6050020F4
:104120000C000020F5050020D40500201C00002014
:104130000E000020094B0A4940F2DC521A805A80D6
:104140009A80DA80074A00231370074AFF2008701C
:1041500048708870C8701360704700BF0E00002060
:104160001C000020F5050020D4050020024B4FF074
:10417000FF321A60704700BF18000020024A03484F
:104180000D2102F099B800BFDCD00000EFDA00008A
:1041900038B54FF4E131284804F02EFE274B0122B8
:1041A00000211A61C3F804150321C3F8081504217E
:1041B000C3F810151A604FF080430221C3F8181598
:1041C0009A604FF01023D3F80C32DB070FD51C4B4D
:1041D000C3F80425D3F80024002AFBD04FF01022A6
:1041E0006FF00101C2F80C120022C3F80425082068
:1041F00005F026F8134A0023FF21995401331D2BA3
:10420000FBD1114B114D01221A600020104A0423EA
:1042100001461468002CFCD02C681160013B44EA74
:104220000020F6D10B4B01221A6004F03FFFBDE8DD
:10423000384001F0EDB800BFB07C012000800040A4
:1042400000E00140D805002000D0004008D5004023
:1042500000D1004004D00040F8B506460948094F97
:104260000C4604F009FE8442A8BF04463546AB1B49
:104270009C4205DD384604F005FE05F8010BF6E723
:104280002046F8BDB07C01200146014804F0B9BDCC
:10429000B07C012010B5054C204604F0BFFD20463F
:1042A0004FF4E131BDE8104004F0A6BDB07C012020
:1042B000C3070CD4064B1B68834208D8054B1B6808
:1042C000984204D850F8043C002B18BF1846704799
:1042D00000060020FC0500200B4908B50122002340
:1042E00041F823200133642BFAD1084B1A60084BA4
:1042F000084A1846002107F09BF9074B40F8043F95
:10430000064B186008BD00BF888E01200800002001
:104310000406002070670100A09D0500F80500203C
:10432000034B044A1A60044B044A1A60FFF7D4BFD7
:104330000006002004060020FC050020746D01200A
:10434000044B1B681868C0F30F10023820EAE070B5
:10435000704700BFF805002000B59BB00246054934
:1043600001A807F0BFFC01A802F06DFA02F07CFD85
:10437000FCE700BF3BD20000C30713D4042802D8D7
:1043800012D00B487047036803F00F03042B01D1D0
:1043900004307047092B09D0064A0748032B18BF81
:1043A00010467047054870470548704705487047F4
:1043B000FACC000026D200002FD2000015D2000057
:1043C00000CD00001FD20000064B074900201A68EC
:1043D00043F8040CC2F30F12023203EB82038B4248
:1043E000F5D3704708060020746D01202F4B304A2A
:1043F0001868304B2DE9F0411C682F4D136803F00D
:104400000F01072928D81368C3F30F13023302EBF7
:104410008302AA42F2D32949002251F82200FFF771
:1044200047FF41F822000132642AF6D1244A10687D
:10443000FFF73EFF1060234A106810B1FFF738FF06
:104440001060214B214C1E680021F0274FF03C08E2
:10445000B14214DBBDE8F081C3F30F1302EB830319
:104460009A42D0D01968CE0707D4884205D28C4230
:1044700003D351F8041C01B11960043BF0E707FBBA
:1044800001F31A191B5D0BB90131E1E71269551EE1
:1044900008FB012204EB82021832002DF4DB52F8F3
:1044A000040DFFF705FF013D1060F6E70006002050
:1044B00008060020FC050020746D0120888E012074
:1044C00008000020746D0120AC050020307D012023
:1044D000C307F0B540D4214B1C68A0423CD3204B0D
:1044E0001D68A84238D850F8043CABBB03680246AC
:1044F000C3F30F13012673B9904242F8046C2BD01A
:10450000116851F8043C51F82370176041F82320DA
:10451000013B0A46EFE752F82310CF0702EB830C6A
:1045200018D48C4216D88D4214D351F8047C8FB91C
:104530000F6807F00F0EBEF1070F08D9CCF8007016
:1045400042F8043C0B680A60C3F30F13E1E741F83B
:10455000046CD0E7013BCEE7F0BD00BF00060020B1
:10456000FC0500200D4930B50D4C0B461A6853F878
:10457000045CC2F30F12901C65B18B4214BF0A4653
:10458000002243F8042C01EB800103EB8003A342DB
:10459000ECD330BD12011A60F7E700BF0806002017
:1045A000746D0120144B2DE9F041144C1E464FF060
:1045B00000083268C2F30F1712070FD07D1C9E420D
:1045C0004FEA850505D018462A46314607F017F808
:1045D00003465A1904352B44C2F80080023706EB13
:1045E0008706A642E5D3E41AA410013C044A24013C
:1045F0001C601360BDE8F08108060020746D012086
:10460000F80500202DE9F0419AB0FFF7CBFB214DD2
:104610000746002455F824000134FFF759FF642CA5
:10462000F8D11D4B1868FFF753FF1C4B186808B1F1
:10463000FFF74EFF1A4DDFF874800026D8F80030DF
:104640009E4218DBFFF78EFFFFF7D0FEFFF7AAFFB1
:10465000FFF7A8FB134B14491B681B68C3F30F1328
:10466000C21B023B01A807F03DFB01A802F0EBF8DA
:104670001AB0BDE8F0812B7813B90136F035DDE7CB
:104680002C69013C002CF8DB05EB84039869FFF7EB
:104690001FFFF6E7888E012008000020746D0120BE
:1046A000307D0120F8050020F5D10000AC05002088
:1046B0002DE9F8431B4C23681B684D1CC3F30F13F3
:1046C0009D42064688461746A1460CDBFFF79AFF37
:1046D00023681B68C3F30F139D4204DB0A20BDE867
:1046E000F843FDF7B1B808F10202D9F800009B1AAF
:1046F0001B0140F82230002340F8043C06F00F066E
:10470000034646EA0816940043F8046B0119083C76
:10471000C9F800101C44A34201D3BDE8F88343F854
:10472000047BF8E7F8050020F8B510F0010704460F
:104730000E462CD1174B1B68834228D8164B1B689A
:10474000834224D9154D28600068012200F00F0033
:10475000FFF7AEFF2C682F600546C0B1214604303C
:1047600051F8042BC2F30F12B242A8BF3246920096
:1047700006F03AFFFFF728FE44F8045CFFF736FE28
:104780002268074B44F8047C134023602C462046E3
:10479000F8BD00BF00060020FC050020746D01205C
:1047A000F0FF0F00011D0022042091FBF0F1FFF744
:1047B0007FBF38B5054608460C46FFF7F3FF50B1FA
:1047C000C21C2B46591B8C4206DC002CACBF0419C2
:1047D000041C0023237138BD13F8011B02F8011FCC
:1047E000F0E7F0B502289BB00C4604DC1C20FDF776
:1047F0002BF81BB0F0BD0868C20706D4042804D902
:10480000036803F00F03042B01D00E20EFE74B6881
:1048100013F00107F9D1042BF7D91B6803F00F033C
:10482000042BF2D18B68DB0701D40D20DFE7FFF703
:10483000A3FD06466068FFF79FFDA5681AAC014618
:1048400004F8647D6D10304603F009FE29466423A8
:10485000224603F066FE204607F08AFA014620460B
:10486000FFF7A7FFC5E7000010B50446ADF5806D62
:1048700010B9FFF797FF0BE003F017FD013806288A
:1048800027D8DFE800F008081017280423000020CC
:104890000DF5806D10BD204603F081FD011B204603
:1048A000FFF787FFF4E7204603F02DFD400040F0BE
:1048B0000100EDE769464FF48062204603F03DFDBC
:1048C000684607F055FA01466846E9E704210348BF
:1048D000E6E70020CDE70420DAE700BF9CD2000025
:1048E000022838B50C4604DC1C20BDE83840FCF733
:1048F000ABBF0868C10706D4042804D9036803F0D5
:104900000F03042B01D00E20EFE76368DA07FAD417
:10491000042BF8D91B6803F00F03042BF3D1A36811
:10492000DB0701D40D20E0E7FFF726FD05466068B0
:10493000FFF722FDA46801466410284603F08FFDAE
:10494000214603F0CBFDBDE83840FFF78DBF0128BD
:1049500038B50C4604DC1C20BDE83840FCF774BFB9
:104960000868C10706D4042804D9036803F00F03BC
:10497000042B01D00E20EFE76368DA07FAD4042B8A
:10498000F8D91B6803F00F03042BF3D1FFF7F4FCF5
:1049900005466068FFF7F0FC0146284603F05FFD1E
:1049A00003F0DBFD400040F0010038BD012870B588
:1049B00005460C4604DC1C20BDE87040FCF744BFF3
:1049C0000868C10706D4042804D9036803F00F035C
:1049D000042B01D00E20EFE76368DA07FAD4042B2A
:1049E000F8D91B6803F00F03042BF3D1FFF7C4FCC5
:1049F00006466068FFF7C0FC022D014615D0A4688A
:104A0000E30712D56410304603F029FD054603F094
:104A10004CFC012812D1002C02DD0135012C07D1FC
:104A20002846BDE87040FFF71FBF4FF0FF34EAE7AC
:104A3000284603F0C3FC013C0546EFE70228EFD10E
:104A4000002CEDDD0135012CEAD00022114628466C
:104A500003F0DEFC03F0B2FC013C0546F3E7086816
:104A600008B5C30706D4042804D9036803F00F036C
:104A7000042B04D00E20BDE80840FCF7E5BEFFF78C
:104A80007BFC0378232B08BF01301022002107F0A4
:104A900033FA00F10053B3F1804F01D31420EAE759
:104AA000400040F0010008BD10B510F0010402D034
:104AB0004410204610BD042812D9026802F00F02EB
:104AC000042A07D1FFF758FC0A222146BDE810400E
:104AD00007F012BA032A03D10A2221460430F5E76F
:104AE0000D20FCF7B1FEE4E708B50868FFF7DCFF2E
:104AF00006F0CAF904F044FE0022054B06F02EFA37
:104B000004F0B0FD06F0DAFC400040F0010008BD02
:104B100000408F4008B50868FFF7C6FF07EE900A0F
:104B2000B8EEE77ADFED0A7A67EE277A17EE900A99
:104B300006F0BCF904F0E0FD0022064B06F00EFA88
:104B400004F090FD06F0BAFC400040F0010008BD02
:104B5000D30237390000D04004282DE9F0410C463B
:104B600004DC1C20BDE8F041FCF76EBE0868FFF7CE
:104B70009BFF07466068FFF797FF0646A068FFF7B0
:104B800093FF0546E068FFF78FFF80462069FFF737
:104B90008BFFAE4201D11F20E4E7BF1BA0EB080052
:104BA0007843AD1B90FBF5F04044400040F001001D
:104BB000BDE8F081024A0348092101F07DBB00BF36
:104BC00054D200004CD20000002070471E20FCF799
:104BD0003BBE1E20FCF738BE1E20FCF735BE1E2053
:104BE000FCF732BE1E20FCF72FBE1E20FCF72CBEA9
:104BF0001E20FCF729BE1E20FCF726BE1E20FCF757
:104C000023BE1E20FCF720BE1E20FCF71DBE1E206A
:104C1000FCF71ABE1E20FCF717BE1E20FCF714BEC0
:104C20001E20FCF711BE1E20FCF70EBE1E20FCF756
:104C30000BBE1E20FCF708BE1E20FCF705BE1E2082
:104C4000FCF702BE1E20FCF7FFBD1E20FCF7FCBDDA
:104C50001E20FCF7F9BD1E20FCF7F6BD1E20FCF758
:104C6000F3BD1E20FCF7F0BD1E20FCF7EDBD1E209D
:104C7000FCF7EABD1E20FCF7E7BD0000024A03482E
:104C80001E2101F019BB00BFF4D20000E4D30000E4
:104C9000034B01221A60034B186890401043704781
:104CA0009C6D0120786D01202DE9F043EFF3108415
:104CB000012304F0010483F31088164A1649126890
:104CC0000E68013A9340154A1568154A12684FF06C
:104CD00002094FF00E0C4FF00D0E4FF00608A3B175
:104CE00018422A600AD0774639000139FDDC32606B
:104CF000474639000139FDDC5B08F0E74F463900D3
:104D00000139FDDC32606746F3E784F31088BDE8C3
:104D1000F08300BF20000020806D0120846D012001
:104D20008C6D012070B5084E084D002456F8240003
:104D30000021FFF751F855F8240000210134FFF756
:104D40004BF8052CF2D170BD74D50000C8D8000016
:104D50002DE9F041134E144D144F0024002156F854
:104D60002400FFF739F855F8248001214046FFF769
:104D700033F8B8F1220F10D857F828200C4B202A0E
:104D8000B8BF4FF0A04302F01F0203EB8203D3F839
:104D9000002742F44072C3F800270134052CDDD10E
:104DA000BDE8F08174D50000C8D80000CCE3000055
:104DB000000300502DE9F3413B4D4FF441732C6843
:104DC000ADF804300A238DF80630BCBBFFF7AAFF0C
:104DD000DFF8E480264658F8267001213846FEF7B1
:104DE000FBFF01360021384604F062FB052EF2D1AC
:104DF00000260DF1040816F8087001213846FEF768
:104E0000EBFF01360121384604F052FB032EF2D1AC
:104E100000210420FEF7E0FF00213046FEF7DCFF12
:104E200000210A20FEF7D8FF01232B60FEF7BAFF0E
:104E30001E4B1860204602B0BDE8F0811B4B1C6879
:104E4000FEF7B0FF844298BF001BB0F57A6F29DBF4
:104E5000022004F0FBF9042004F00AFA04460320BF
:104E600004F006FA07460A2004F002FA064601207A
:104E700004F0ECF9012004F0FBF9E0193044C0F52E
:104E800032600323023090FBF3F0094B0028BCBFD3
:104E900000221A60074AA8BF186000232B60136025
:104EA0000124C7E70024C5E7946D0120A06D01200F
:104EB000786D01209C6D0120C8D8000008B5054B15
:104EC00000221A60044B1B680BB103F08DF900201F
:104ED00008BD00BF986D0120147B012010B5041E91
:104EE0001CDA00241049114B114A0B600433136083
:104EF000104B53F824301F2B81BF0F4808600F4917
:104F0000116003F01F024FF0010303FA02F38CBF9C
:104F10000C310B490B4A0B60136010BDFEF75AFFB2
:104F2000A042DEDDDEE700BF846D012008050050F1
:104F3000806D0120CCE30000080800500C080050F0
:104F4000180500508C6D012008B50B68DA074CBFBE
:104F50005B104FF0FF3301280DDD4A68042A14BFAF
:104F600018222022054918460A60FEF759FFFFF76C
:104F7000B5FF002008BD1822F4E700BF2000002084
:104F8000002808B50CDD0B68042B084B14BF012268
:104F900000221A6006D0FFF7C5FE054B00221A60FA
:104FA000002008BDFFF7D4FEFAE700BF906D012096
:104FB000786D012010B510F0010402D04410204695
:104FC00010BD042812D9026802F00F02042A07D18A
:104FD000FFF7D2F90A222146BDE8104006F08CBF47
:104FE000032A03D10A2221460430F5E70D20FCF7FD
:104FF0002BFCE4E7086810F0010370B51CD0FFF744
:10500000D9FF0346203B5E2B27D8154C03EB8303C7
:105010000022012110462344052A1AD09E5C052453
:1050200010252E4218BF4018013C4FEA41014FEABB
:105030006505F6D10132EFE70428E3D9026802F0F2
:105040000F010429DED1C2F30F13002BDAD003794C
:10505000D8E7400040F0010070BD0120FCE700BF30
:1050600088D5000038B508680D46FFF7A3FF044651
:105070006868FFF79FFF621E042A014612D8431E8C
:10508000042B0FD8084803EB83031344056801225F
:1050900002FA03F32B430360044B1B6813B1204651
:1050A00003F0A3F8002038BD986D0120147B012087
:1050B00038B508680D46FFF77DFF04466868FFF7BE
:1050C00079FF621E042A014614D8431E042B11D80E
:1050D000094803EB83031344012202FA03F3026835
:1050E00022EA0302054B02601B681BB10022204626
:1050F00003F07BF8002038BD986D0120147B01205F
:105100002DE9F04F054685B008680C46FFF752FFC1
:10511000022D01903CDD6068FFF74CFF0746A06858
:10512000FFF748FF0446231DDFF8C8A00293661E60
:105130004FF00108029B9E4206F1010935D006EBB3
:105140008602531E07F1050B3D460393AB4522D063
:10515000042E19D86A1E042A16D8039B019ADAF87D
:1051600000005919224B4FF0010C18EA020E0CFAFC
:1051700001F11B6811D00143CAF8001023B1624647
:105180004946284603F031F84FEA48080135DDE783
:1051900001242746C7E74E46CCE720EA0101CAF8BA
:1051A0000010002BF0D07246EAE73D1D042D1BD8FD
:1051B000012C19D1DFF83C80DFF834900026D8F8B4
:1051C000003004FA05F223EA0203C8F80030D9F8E7
:1051D0000030013623B100223146781D03F005F876
:1051E000052E05F10505EAD1002005B0BDE8F08FD8
:1051F000147B0120986D01202DE9F843394B1B6881
:105200000C461BB94FF0FF30FFF768FE206810F026
:1052100001083AD1042838D9036803F00F03092B99
:1052200033D10746304D57F8044F304E641040F2EA
:105230005969A04552DA57F8040FFFF7BBFEC0F3D7
:105240000742C0F307235B43524393FBF9FC92FBF5
:10525000F9F32A68202AC1B208BFC0F305604FEAFB
:10526000032308BF56F8202043EA0C4301FB01F159
:1052700091FBF9F143EA010308BF42EA0323184610
:10528000FFF712FD08F10108D3E7FFF793FEC0F323
:105290000742C0F3072340F259655B43524393FB37
:1052A000F5F492FBF5F3104A1268202AC1B204BF4C
:1052B0000E4AC0F305604FEA032308BF52F82020CE
:1052C00043EA044301FB01F191FBF5F143EA0103D9
:1052D00008BF42EA03231846FFF7E6FC0020BDE8BA
:1052E000F88300BF8C6D01202000002064D70000EF
:1052F000086808B5C30703D5FFF75CFE054B1860C7
:10530000054B1B681BB1034B186802F06FFF0020B0
:1053100008BD00BF986D0120147B01202DE9F843E2
:10532000334B1C68002C59D1324E326852B9324B83
:105330001B683BB9314B1B68002B4FD0BDE8F843CD
:10534000FFF738BD2E4D2B6863B92C4B1B68002B23
:1053500040D1294A336810681146002840D10B60BB
:10536000FFF7F6FC2B68274EDFF88C90264F002BBA
:10537000CCBF03F1FF330423002156F82300FEF7CE
:105380002BFD2A68214B53F8228057F8240004EBA8
:10539000840101EB0803D9F80010194101F0010163
:1053A000013404F085F8052CEFD12B68012156F863
:1053B0002300FEF711FD2B68002156F8230004F0AE
:1053C00077F82B68013393FBF4F404EB84041C1B83
:1053D0002C6003E0FFF7EEFC0028BAD1BDE8F883AB
:1053E000002BBCD11360BDE8F843FFF79BBC00BFA6
:1053F000906D0120986D0120886D01209C6D012029
:105400007C6D012074D50000C8D8000064D800006D
:105410004FF0FF30FFF762BD024A03480A2100F057
:105420004BBF00BF78D80000DCD800004FF080539D
:1054300010B51A69094B0224C3F8044522F003028F
:10544000884203D30022C3F8042510BDD3F80044DA
:10545000002CFBD0C3F808051044F1E700E0014040
:10546000002815BF4FF4D2214FF4B4214FF4B420DB
:105470004FF49620FFF7DABF00280CBF4FF49623B5
:105480004FF4B4231868030E532B0CBF20F07F4059
:1054900000207047064B0122C3F80425D3F80024EE
:1054A000002AFBD000220160C3F80425704700BF2A
:1054B00000E00140002821F07F4141F0A6410CBFEF
:1054C0004FF496204FF4B420FFF7E4BF0A4B30B5F9
:1054D0000124C3F80445002903DC0022C3F8042595
:1054E00030BD52F8044BD3F80054002DFBD040F8E7
:1054F000044B0139EFE700BF00E0014038B54C68CC
:10550000023405460A462146FFF7E0FF05EB84001A
:1055100038BD0000124B1B68002B0BBF4FF4B422A8
:105520004FF4D2224FF496234FF4B42328B91A1D16
:10553000DB79522B08BF1046704782420DD9C378E1
:10554000522B0AD14368023300EB8300824204D914
:10555000C378522B18BF002070470020704700BF4F
:10556000A46E01202DE9F0410020B4B0FFF7D2FF76
:105570000024DFF8A4800546274626464DBB224D71
:105580002868FFF779FF3B463246CDE900401F49C6
:1055900002A806F0A7FB02A801F055F91C4B1A68F7
:1055A0002B68002B0CBF4FF496234FF4B423D21A70
:1055B0004FF4704164235343009193FBF1F302A82D
:1055C000144906F08FFB02A801F03DF934B0BDE8A4
:1055D000F08169682A6801918B1C1F44D1B2C2F323
:1055E00007239C42C2F30742009102A84146B8BF7C
:1055F0001C4606F077FB02A801F025F92846FFF7C4
:1056000089FF01360546B9E7A46E0120F6D90000EE
:10561000A86E0120A0D90000E2D9000070B50020DA
:10562000FFF72AFF05460120FFF726FF0C4B1E68F7
:10563000B6FA86F485424FEA5414B8BF05462046B0
:105640001C60FFF70DFF074A074B002E18BF1346DB
:10565000064A691C2046BDE870401360FFF72ABF68
:10566000A46E012004B0040004A00500A86E01206F
:1056700070B50020FFF700FF02460120FFF7FCFE97
:105680001F4E204C054672B968B94FF4D2214FF431
:105690009620FFF7CBFE01212846FFF70BFF1A4BA0
:1056A0003560236029E0AA4208DD00233360164BF1
:1056B00023604FF4B4212368002017E001233360F6
:1056C000124B23604FF4D221F5E7120E522A08D074
:1056D00000B123600E4801F0B6F8BDE87040FFF756
:1056E0009DBF5A68023203EB820301208B4205D230
:1056F0001A68551CE9D10028D3D170BD2160FCE7A0
:10570000A46E0120A86E012004B0040004A00500CE
:10571000BBD9000010B50020FFF7FCFE014608B918
:10572000084610BD8478FFF7F5FEDA2C08BF014665
:10573000F5E7000038B500214FF4FF621B4805F083
:1057400077FFFFF7E7FF1949002490B91848174C75
:105750000123F02101FB030212F8F05C2DB112F8D5
:10576000EF5C54F8355042F8E85C01330B2BF1D173
:1057700038BD0368C3F307420A2A0BD1C3F30722DB
:10578000FF2A04D001EBC20541F832002B71FFF76C
:10579000C1FEDAE7132AFAD1C3F30723FF2B1EBF9A
:1057A00001EBC30241F833401471F0E79086012009
:1057B000307D012000B59BB0FFF75AFFFFF7BAFF1D
:1057C00000230B491A4651F8330000B1013201336E
:1057D000FF2BF8D1074901A806F084FA01A801F0CF
:1057E00032F8054801F02FF81BB05DF804FB00BF4C
:1057F000908601202BDA00003FDA00002DE9F04FFF
:105800004FF480729FB0604C6048002105F010FF9B
:105810004FF4807200215E4805F00AFFD4F8009032
:10582000B9FA89F84FEA58184046FFF719FEA24620
:10583000584B594C0020B9F1000F08BF1C46FFF728
:1058400069FF064648BB4846FFF716FE534D411C0C
:105850004046FFF72FFECAF800802C60FFF76AFF72
:10586000FEF718FDDAF800302A68002B0CBF4FF461
:1058700096234FF4B423D21A4FF470416423534358
:10588000009193FBF1F305A8454906F02BFA05A812
:1058900000F0D9FF1FB0BDE8F08F3568C5F30743AE
:1058A000A3F10A02092AC5F3072546D8374B595DEB
:1058B00091BB10223B48DFF8ECB005F0B9FE37464B
:1058C0003A68C2F307218D4209D1C2F307410B297F
:1058D00026D013292BD00A2901D1CBF800703846E5
:1058E000FFF718FE07460028EAD12E4F396881B12C
:1058F0002046FFF703FE0123044657F8231029B181
:1059000020460393FFF7FAFD039B04460133042B63
:10591000F3D11E4A012353553046FFF7FBFD90E7B4
:10592000D2B2022ADBDC0BEB82025760D7E71022EF
:105930000021584605F07CFED1E7A3F11502082AA4
:10594000EAD8134A525D002AE6D1152B0CBF314626
:10595000002130460368C3F30742152A0ED01D2AE2
:1059600008BF0021FFF7D6FD0028F3D119B120466A
:10597000FFF7C4FD04460123054ACCE7C3F3072320
:105980009D4208BF0146EDE7A46E0120A46D0120F1
:10599000AC6E012004A0050004B00400A86E012034
:1059A00085D9000018900120FFF728BF2DE9F84F96
:1059B000DFF8A8B0274F03339246042293FBF2F698
:1059C000DBF80030B41C002B3B684FEA84040CBFAA
:1059D0004FF4B4224FF4D22223449A4281460D461A
:1059E000B84614D2FFF70AFFDBF80030002B3B6803
:1059F0000CBF4FF4B4224FF4D22223449A4206D271
:105A0000154800F020FF00273846BDE8F88F2D022A
:105A10005FFA8AF141F0A441ADB2D8F800700D43AD
:105A20004FEA094101F47F0129433846FFF732FD6F
:105A300007F108053146381DC8F80050FFF72AFD68
:105A40001EB10A9A2846FFF741FD083C2544C8F8D4
:105A50000050D9E7A86E01205FD90000A46E012094
:105A6000704770470A4B0022C3F8002101225A6098
:105A7000D3F80021002AFBD00022C3F80C21012218
:105A80009A60044B0222C3F880211A60704700BF5D
:105A90000010004000E100E0074B0222C3F8802024
:105AA000064B0022C3F8102101221A61D3F81021FD
:105AB000002AFBD0704700BF00E100E0001000406A
:105AC00008B504490A780AB1FFF7E6FF002008701C
:105AD00008BD00BFAD6F0120024B1868400040F0C8
:105AE0000100704730700120024B1868400040F000
:105AF00001007047240000201FB5064B06491A68B4
:105B000001A806F0EFF8082101A8FEF752FE05B043
:105B10005DF804FB34700120D0DA00001FB54FF0AF
:105B2000805306491A6E01A806F0DCF8082101A886
:105B3000FEF73FFE05B05DF804FB00BFD0DA0000C1
:105B400010B5054C204606F013F901462046BDE885
:105B50001040FEF72EBE00BF39700120104B1B68AD
:105B60005A1C10B514D0CBB1012B13D0022B13D07B
:105B7000042B13D00B4C0C4A052B08BF14462046AF
:105B800006F0F6F801462046BDE81040FEF711BECB
:105B9000064CF4E7044CF2E7054CF0E7054CEEE761
:105BA00028000020DADA0000E0DA0000D5DA000090
:105BB000BBD00000B4D0000070B504460D461646B8
:105BC000FEF7F8F84FF0805301221B6E6270E2700E
:105BD000020AA271020CE2711A0A0021607163725A
:105BE000000EA2721A0C1B0E2670A1702571207275
:105BF000E272237370BD000010B521480278002ABC
:105C00003DD14FF08043C3F8002101221A60D3F840
:105C10000021002AFBD01B4B1B4C00220721C3F89C
:105C20000C25C3F808151949C3F81025C3F81C152D
:105C3000C3F824250121C3F82C250822C3F8301508
:105C4000C3F81425C3F818450224C3F834454FF6A9
:105C5000FF74C3F83C450E4CC3F838451824C3F80C
:105C60005445C3F80423D3F8002242F01002C3F8CD
:105C70000022084AC3F80425FFF7F4FE017010BDA6
:105C8000AD6F0120001000402000040274696275AD
:105C900021100100AE6F012013B50A4A0A4B0728F4
:105CA0000446CDE900230BD8084B1B780BB9FFF74E
:105CB000A3FF02AB1C44064B14F9082CC3F80C25B7
:105CC00002B010BDE2ECF0F4F8FC0004AD6F01206E
:105CD00000100040F8B5104B1B7804460BB9FFF7D5
:105CE0008BFF0E4E3378ABB10D4A1278D21A02F008
:105CF00003010C4A02EB411202F1200710685168BF
:105D0000254603C50832BA422C46F7D1013B337011
:105D10000120F8BD1846FCE7AD6F01203870012066
:105D2000AC6F0120AE6F012030B5002889B02ADDAC
:105D30000D6815F0010426D1042D26D92B6803F037
:105D40000F03092B21D16B683F2B1EDD6846FFF73F
:105D5000C1FFB0B19DF800200435A242A8BF1DF8D4
:105D6000043004F10104A6BF5B0043F001030123EA
:105D7000202C45F8043FF0D1054BDDF809201A60CE
:105D8000042009B030BD0020FBE72046F9E700BF42
:105D90003470012030B5384B1B788BB00BB9FFF74E
:105DA0002BFF02A8FFF796FF10B900200BB030BD03
:105DB0009DF808300B2BF8D99DF80930012BF4D150
:105DC0009DF80B30012BF0D12C4D2D4C2D4ADDF8D8
:105DD000111000232B6023709DF80C3013602A4AA9
:105DE000116023B9DDF815302B6000230FE0012B83
:105DF00011D1DDF815309DF819202B600DF11A0135
:105E00000E239342A8BF134600229A4230D10022AB
:105E1000E2540420CAE7022B05D19DF81520122375
:105E20000DF11601EDE7042B0DD10AAA6B4652F8CD
:105E3000130D516803C3DDE9000103F085FB05F094
:105E40003DFB2860D1E7052BCFD10AAA6B4652F85B
:105E5000130D516803C3DDE9000103F075FB05F084
:105E60002DFB9DF81D2028600A230DF11E01C8E7B7
:105E7000885CA0540132C8E7AD6F0120307001206A
:105E800039700120280000203470012010B5154B16
:105E90001B7804460BB9FFF7AFFEFFF7FDFD124B71
:105EA0000022C3F80445C3F8002101221A60D3F888
:105EB0000021002AFBD00022C3F80C2101229A60A5
:105EC000094AD2F80C31002BFBD0084B1978084B4B
:105ED00003EB4113C2F80435FFF7DEFDBDE81040C7
:105EE000FFF7C0BDAD6F012000100040AC6F012076
:105EF000AE6F012000B5002889B01DDD0B6813F0DE
:105F0000010219D1042B17D9196801F00F010929D1
:105F100012D159683F290FDD043353F8040F10F0F4
:105F2000010118BFC0F347010DF802100132202A09
:105F3000F3D16846FFF7AAFF002009B05DF804FB23
:105F4000002810B511DD0C68E3070ED56410532C42
:105F50000BD8074B1B780BB9FFF74EFEFFF79CFDE4
:105F6000044BC3F80845FFF77DFD002010BD00BFBE
:105F7000AD6F012000100040002810B50DDD0C6849
:105F8000E3070AD56410FF2C07D8054B1B780BB923
:105F9000FFF732FE034BC3F82445002010BD00BFBD
:105FA000AD6F012000100040002808B505DD08682D
:105FB000C30702D54010FFF76FFE002008BD70B583
:105FC000002888B020DD086810F001041CD10428E6
:105FD0001AD9036803F00F03042B15D1FEF7CCF98F
:105FE000064605F0C5FE122828BF1220054600F11E
:105FF0000D0202216846FFF7DFFD8DF80D50A54226
:1060000005DC6846FFF742FF002008B070BD0DEBCD
:106010000403325D9A730134F1E72DE9F041012860
:1060200088B00D4630DD086810F001042CD104283A
:106030002AD9036803F00F03042B25D14B68DB0733
:1060400022D5FEF799F9804605F092FE6D680E287C
:1060500028BF0E206E10074600F11102012168468C
:10606000FFF7AAFD6B128DF80D606D14360E8DF8DA
:106070000E308DF80F508DF810608DF81170A7421A
:1060800006DC6846FFF702FF002008B0BDE8F0819B
:106090000DEB040318F804209A740134EFE730B5CF
:1060A000002889B016DD0C68E30713D56510684633
:1060B00010220021FFF780FD63128DF80D5064144B
:1060C0002D0E68468DF80E308DF80F408DF810506B
:1060D000FFF7DCFE002009B030BD0000174BD3F8FD
:1060E000002122B10022C3F8002101229A60D3F8D6
:1060F0000C2102B30021C3F80C11D3F80024012AAB
:106100000F4A19D1D3F848355B4213600D4A137812
:10611000032B9CBF013313700B4A1378013303F038
:1061200003031370094A02EB4313044AC2F804350F
:10613000024B01229A6070471160F9E7001000409D
:106140002400002038700120AC6F0120AE6F0120C8
:1061500008B50A4B1B787BB1FFF79EFC0849072363
:10616000C1F80835FFF77EFC0023C1F8243506206E
:10617000BDE80840FFF790BD08BD00BFAD6F01202E
:1061800000100040024A0348102100F095B800BFFB
:1061900050DA000047DA0000044A05491368C85481
:1061A0000133C3F309031360704700BF6C7401200F
:1061B0006C70012070B51249124A0B68834202DCF0
:1061C00000230B6018E0845CA4F1FA06012E00F1B4
:1061D000010506D8AB4210DDAC5C14B1283C9F2C05
:1061E00001D82846EAE70446151A165D2E550134F3
:1061F000A342FADC181A086070BD1470FAE700BFF9
:10620000787801207874012008B5FDF7CBFD074BA5
:106210001A68824284BF00221A601B68C01A44F6C2
:106220002063984294BF0020012008BD64700120C3
:1062300010B5FFF76FFA044608B9204610BD837801
:106240001D2B08BF0446FFF765F9F5E7F8B50C4CC0
:106250000C4E0D4F002523683268934203D0F85C42
:10626000FEF712F828B91DB1FDF7A4FD074B186021
:10627000F8BD23680133C3F3090323600125EAE76E
:10628000707401206C7401206C7001206870012012
:1062900070B5074E074D044633682A689B1ADB43E6
:1062A000C3F30903A34200DB70BDFFF7CFFFF3E7A1
:1062B0006C74012070740120F0B5074D2B680B2B16
:1062C00008DC064F0C245C433E19C6E90112013379
:1062D00038512B60F0BD00BF74740120289001205C
:1062E0002DE9F04FB3B0044605F042FD012803D874
:1062F000002033B0BDE8F08F23785B2BF8D1013854
:106300002518235C5D2BF3D101343A21204605F09A
:1063100018FD06460028EBD0071B002FE8DD2146BC
:106320003A46684605F03EFD32AB711C00241F441E
:106330006D1AA54207F8C84CDADD2A4619A805F0FF
:1063400031FD32AB1D44134B134ED3F8009005F8CA
:10635000644C4FF00C0AA145CADD0AFB04F3694600
:10636000985903EB060805F0F9FC054618B9D8E979
:106370000187454501DB0134EDE719A957F83500E0
:1063800007EBC50B05F0EAFC10B9DBF80400B0E739
:106390000135EEE7747401202890012008B5FBF761
:1063A0008DF8FFF739F8FBF7AFF8FDF7E7FEFEF7DA
:1063B00001FCFEF763FCFFF7E5FE01F091F901F047
:1063C000E9FE01F015FFBDE8084002F04BB90000FE
:1063D00008B54FF416620021034805F029F9034B74
:1063E00000221A6008BD00BF307D0120AC050020EE
:1063F000174B53F83000836803F07F031C2B70B5F4
:106400000D46144601D0002070BDC36803F07F0222
:10641000042AF8D1026902F07F02192AF3D11B0A7B
:1064200000EB83001030FDF7A7FF0378064633B179
:1064300005F09EFCA042E6D10023A34201DB01202F
:10644000E2E7F15CEA5C9142DDD10133F5E700BFA0
:106450009086012008B5FDF7ADFC074B1A68824213
:1064600084BF00221A601B68C01AB0F5FA6F2CBFF7
:106470000020012008BD00BF68700120064B074ABC
:106480001B6812689B1ADB43C3F309038342D4BF22
:1064900000200120704700BF6C740120707401203F
:1064A000F8B507460E4614461D4673B90320FFF79C
:1064B000E5FF10B3FA20FFF76FFEF8B2FFF76CFEAE
:1064C000F0B2BDE8F840FFF767BE501DFFF7D6FFFA
:1064D00098B1FB20FFF760FEF8B2FFF75DFEF0B267
:1064E000FFF75AFEE0B2FFF757FEC4F30720FFF7AD
:1064F00053FE2E46731B9C4200DCF8BD16F8010BC0
:10650000FFF74AFEF6E70000F8B50C4E0C4D0024EC
:10651000F0273368A34203DCBDE8F840FFF758BF1B
:1065200007FB04F359195B5D2BB100231A46497828
:106530001120FFF7B5FF0134EBE700BFAC050020E9
:10654000307D0120F8B50E4C0E4E07460025BC42AA
:1065500005F1010511D0237853B100231A46617863
:106560001120FFF79DFFF0220021204605F060F882
:106570000A2D04F1F004EAD1F8BD3560F8E700BF58
:10658000307D0120AC0500202DE9F04F12F001060E
:10659000ADF54F7D82468B4617D001238DF8143020
:1065A00042FA03F354128DF8153052141B0E8DF875
:1065B00017208DF818308DF8164005AB0522FFF72F
:1065C0006FFF0DF54F7DBDE8F08F042A2CD91168BF
:1065D00001F00F03042B38D105AD022310462B70B8
:1065E000FDF7CAFE044605F0C3FBB0F5487F03463D
:1065F00004F1FF31A8BF4FF448739E4206F1010237
:106600000DD1B0F5487F06D96D4B19889B78ADF850
:1066100032138DF834332B4659465046CFE7164691
:1066200011F8012FAA55E8E740F0C680A2F1040C4A
:10663000DCF100024FF0030342EB0C028DF8143042
:106640008DF8152005AB0222E6E7092B40F091807A
:10665000154604238DF8143055F8043F4FEA6308BB
:10666000B8F1200F8DF815804FEA6323A8BF4FF0D3
:1066700020088DF816308DF8178006AC032205210E
:10668000B04502DC05ABE21AC6E755F8040F10F07E
:10669000010706D1042847D9036803F00F03022B32
:1066A0000DD14FF0010323704310637047121B0E8E
:1066B0004014A770E070237105340136E0E7042B25
:1066C00030D123464FF0020C03F802CBCDE9012173
:1066D00000930393FDF750FE814605F049FB0C281B
:1066E000DDE901210AD8009B6070874201D1DC19E5
:1066F000E3E719F80740DC550137F6E723460C209D
:1067000003F8010F09F1FF3009F1080910F8017FC2
:1067100003F8017F4845F9D12E23E3722373637395
:106720000E34CAE7012B08D12346071F03F8022BBA
:106730007842784160701C46BFE7092B09D10423D9
:1067400023704368581060705B12A370E7700434C4
:10675000B3E7032B0AD121700368C3F30F10C3F30F
:106760004173C3EB800363701B12EEE727700134A3
:10677000A3E7032B7FF425AF05238DF81430C1F375
:106780000F13C1F34171C1EB830164294FEA212347
:106790008DF81510A8BF64218DF816308DF81710EC
:1067A00003328E4205AB01DB0A1D35E7334412F894
:1067B000010F18710136F4E7002A7FF402AF35E7C4
:1067C0000ACD00000F4970B5F022002402FB04132B
:1067D0005D78854203D001340A2CF7D170BDF022D8
:1067E0001846002104F024FF074A1368013BA34226
:1067F00000D11460002329461A461120BDE87040DC
:10680000FFF74EBE307D0120AC05002030B5B3B09F
:1068100032AC0223054604F8C83D05F0A9FAC728A2
:1068200028BFC720691E0023984207DC421C23466C
:10683000FE211420FFF734FE33B030BD013311F8D0
:10684000012FE254F0E770B5B2B00446FFF702FE44
:10685000C0B132AD0223204605F8C83D05F088FAE4
:10686000C72828BFC7200646013C0023B3420BDBE4
:1068700006F13200FFF70CFD2B46721CFF2114209D
:10688000FFF70EFE32B070BD013314F8012FEA5449
:10689000ECE700002DE9F04F0128B9B081468846A9
:1068A00003DC1B20FAF7D0FF57E00868C20729D4A1
:1068B000042827D9036803F00F03042B22D1FDF726
:1068C0005BFD0546D8F80400C3071DD404281BD976
:1068D000036803F00F03042B16D1FDF74DFD0646A8
:1068E000204B1B6803930027039BBB420EDC0096E2
:1068F0002B461D4AC82106A805F0C0F906A8FFF7D7
:10690000A2FFCEE7194DDDE7184EE9E70C237B43E4
:10691000174A2946985803EB020B05F01FFA044664
:1069200018B9DBE9013A9C4201DB0137DCE70AEBED
:10693000C40231465AF834000593049205F00EFA69
:10694000DDE90423834658B9536808F10801A9F129
:1069500002009847074BC3F800B039B0BDE8F08F8C
:106960000134E0E774740120B1DB00004BD2000079
:1069700028900120746D01202DE9F0411F4F204A1D
:10698000D7F8008005460023F02098450EDC00244F
:10699000F02000FB04F15318565C8EB101340A2C30
:1069A000F7D11848BDE8F041FFF74DBF00FB03F1F8
:1069B00054186478AC4201D1515CE9B90133E4E781
:1069C000F0223146184604F033FE0F49457051F865
:1069D000351085700222A0450270C0E90212C0E99C
:1069E000046601DC01343C60002329461A4610206D
:1069F000BDE8F041FFF754BDBDE8F081AC050020D3
:106A0000307D0120F9DF00009086012070B5FFF78E
:106A10007BFD094EFF246FF0070505FB046393F827
:106A2000FC37043B012B03D8E043C0B2FFF7A4FFBF
:106A3000013CF2D170BD00BF908601202DE9F041EC
:106A400006460F46FDF7B5FE0D4BDFF8388018609F
:106A5000002408EBC4031B79062B01D0032B09D1BA
:106A6000E5B23A4631462846FFF7C2FC10B1284647
:106A7000FFF782FF0134FF2CEBD1BDE8F08100BFAE
:106A80000800002090860120F8B5094F0546FF2434
:106A90006FF0070606FB047393F8FC37AB4203D193
:106AA000E043C0B2FFF768FF013CF3D1F8BD00BF7F
:106AB000908601202DE9F84FFDF774F9584B1A68BC
:106AC000824284BF00221A601A6842F20F71821A51
:106AD0008A420BD95349186000235A181279073A91
:106AE000022A0FD90833B3F5FF6FF6D1BDE8F88F4E
:106AF0000720FFF7C9FF8AF800802EE00820FFF783
:106B0000C3FF3FE0FDF756F9002814BF04460124F7
:106B10000020FDF7FBF981460020FDF70BFA424DFE
:106B2000424E0746B9F1000F17D02B68002B70D1E9
:106B300033682C60002B6FD0DFF8F8B0DFF8F0A0DE
:106B40009BF800304FF00108002BD1D10920FFF74E
:106B50009BFF8AF800808BF80080AFB133689BB947
:106B60002B6834601BB3DFF8C8B0DFF8C8A09BF80F
:106B700000304FF00108002BC0D10920FFF784FF3F
:106B80008BF800808AF800802B6883B1284A11783E
:106B9000904661B99C4238BF2C602B68E31A312BB8
:106BA00005D90720FFF770FF012388F8003032680D
:106BB00082B1204B1978984661B9A24288BF3460EF
:106BC0003368E41A312C05D90820FFF75DFF012353
:106BD00088F800302B685BB1B9F1000F08D1144C74
:106BE000227812B90720FFF74FFF00232B60237094
:106BF0003368002B3FF47AAF002F7FF477AF0D4C52
:106C0000227812B90820FFF73FFF0023336023707A
:106C10006CE7002FA2D1B9E7002FA1D1B4E700BFE4
:106C20006070012090860120507001205870012072
:106C3000547001205C70012013B50446FFF764FC1A
:106C4000FEF70FFF00230093134B1B6813B9684630
:106C5000FDF73EF902A9042341F8043D0120FEF7A7
:106C60008FF900210846FEF729F9FEF757FBFFF7D9
:106C70006FFAFDF773F9FDF75DFAFDF777FAFEF7A6
:106C8000C7FBFDF7B7F824B1FDF726FB0348FFF774
:106C9000DAFD02B010BD00BF147B0120EADF000066
:106CA000002301461A461120FFF7FABB07B513125D
:106CB0008DF801208DF802301314120E8DF800109B
:106CC0008DF803308DF8042001466B460522132011
:106CD000FFF7E6FB03B05DF804FB0A46014612200D
:106CE000FFF752BC70B505460C46FFF7B3FB58B131
:106CF00004F13200FFF7CCFA2B46224600211B207C
:106D0000BDE87040FFF7CCBB70BD10B4144603461D
:106D10000A46142021465DF8044BFFF7C1BB000072
:106D200030B5084C01444FF0FF33884201D3D843BB
:106D300030BD10F8015BDAB26A4054F8222082EAD2
:106D40001323F2E7CCDB0000FE2837B5044614D845
:106D50000B4B53F8300080B1416808308900FFF7D1
:106D6000DFFF02AD45F8040D0920FFF791FA2B462D
:106D7000042221461720FFF793FB03B030BD00BF6C
:106D800090860120254AF8B500231846174652F888
:106D9000331001B101300133FF2BF8D100EB800437
:106DA0000A20FFF775FAFB20FFF7F6F92720FFF717
:106DB000F3F90020FFF7F0F9E0B2FFF7EDF9C4F3C3
:106DC0000720FFF7E9F9164B00241E68FA2396FB0B
:106DD000F3F657F83400E0B1416808308900FFF756
:106DE0009FFF05460520FFF753FAE0B2FFF7D4F9FD
:106DF000E8B2FFF7D1F9C5F30720FFF7CDF9C5F3E6
:106E00000740FFF7C9F9280EFFF7C6F9304602F030
:106E10006BF90134FF2CDCD1F8BD00BF9086012056
:106E200004000020F8B50746FFF702FA4FF0FF35DF
:106E300004460CB92846F8BD2668C6F30743152B4F
:106E40000CD104F10801384604F088FF08B9C6F3F4
:106E500007252046FEF75EFB0446EAE71D2B08BF28
:106E60004FF0FF35F5E700002DE9F04FAE4CDFF8AD
:106E7000D8829DB0FFF7EAF92068C0F580614044F0
:106E8000FDF7EAF9236818442060464688B1FCF70C
:106E900089FFA64B186098F80030FA2B40F0568115
:106EA0002368022B08DCFFF7AFF910B10120FFF7D0
:106EB00081F91DB0BDE8F08F98F8010098F8024004
:106EC000831E242B00F22681DFE813F02500390011
:106ED0003D00410044004D00240157008C00960005
:106EE0009D00B300F4000B012401240124012401BE
:106EF0002401240124012401240124011F0124016F
:106F00002401240124012401240124012401240159
:106F1000240124019A00FF2C0FD02046FFF752FCD9
:106F2000834A002342F8343002EBC4022146137135
:106F3000132000931A46FEF739FD0320B7E72046D9
:106F4000FFF71AFDF9E72046FFF73CFCF5E7FFF7EE
:106F50005DFDF2E7FFF7D8FA0020FFF76DFE7548F8
:106F6000FFF771FCE9E7632CE7D8734B214653F830
:106F700024201520FFF708FBDFE7FFF759F96FF032
:106F800007080446002CD8D02768C7F30743152B01
:106F900004D02046FEF7BEFA0446F3E704F10806E3
:106FA000304604F0E5FE05460530FFF771F9FB2099
:106FB000FFF7F2F81D20FFF7EFF8C7F30720FFF700
:106FC000EBF8E8B2FFF7E8F8C5F30720FFF7E4F8BD
:106FD000A8EB0407F3199D42DBDD16F8010BFFF760
:106FE000DBF8F7E7002300931A4619461D20FEF749
:106FF000DDFCFDF771F9A0E72046FFF7A5FE9CE751
:10700000FFF7C0FE99E7FCF7E1FE4C4A00906421CF
:107010004B4B03A804F032FE022303A88DF80C307A
:1070200004F0A6FE03AB024600211620FFF738FA53
:1070300083E7444BDFF8F8801F680025FA2397FBAD
:10704000F3F758F8354008EBC50354B3D4F804906F
:1070500093F804B04FEA8906B01DFFF719F9FB2039
:10706000FFF79AF8012006F1010AFFF795F8E8B258
:10707000FFF792F85FFA8AF0FFF78EF8CAF307205D
:10708000FFF78AF85846FFF787F808342644A642E7
:107090000BD8FFF7DBF809FB07F002F025F8FFF744
:1070A000D5F80135FF2DCCD147E714F8010BFFF7D8
:1070B00073F8ECE70024FFF727FA2346224621461F
:1070C0000094DA20FEF772FC21464FF4FF62184864
:1070D00004F0AEFAFDF700F921462046FDF7EEFE7A
:1070E0002BE7012C02D1FEF73DFA26E7022C02D154
:1070F000FEF75AFC21E7032C03D100210846FDF7D7
:10710000DDFE0120FFF798FD17E700231A46214610
:107110001A208BE7A0F1C803052B3FF60EAF002223
:107120001146FAF7FBF908E778780120647001202E
:1071300090860120CCDF0000888E0120E3DF000074
:10714000DEDF00000400002078740120FB2B7FF4B8
:10715000ADAE2268042A7FF7A6AEB8F8037040F2FD
:10716000F6339F423FF7A2AE3B1D9A427FF79BAE9C
:1071700018F80330FE2B7FF499AE98F8010098F8C8
:1071800002401B2807F1FF356BD01CD807284FD0D1
:10719000082826D001281BD1FF2C12D02046FFF74B
:1071A00011FB98F80550534B00932146BB1E2A460D
:1071B0000A20FEF7FBFB504B43F8340003EBC404FA
:1071C0002571781D73E61D285FD050D31E2874D01A
:1071D000A0F1C803052BF4D8484A2946FAF79EF9CE
:1071E000EFE7632CEDD898F80530022B0CD0032B79
:1071F00014D0012BE5D1D8F80630414A5B0043F0AA
:10720000010342F82430DCE7002DDADDB91E3948ED
:10721000FDF7CFFA3A4B43F82400D2E798F806304E
:10722000002B374B0CBF0022042243F82420C8E770
:10723000632DC6DC2A46314903A804F0D5F91CABFE
:107240001D4403A8002305F8643CFFF7EBFD00286C
:10725000B7DB2B4B214653F820201520FFF794F97C
:10726000AFE7294608F10500FFF7E8FBA9E7FF2C87
:10727000A7D098F80520022AA3D81E4B00932146D8
:10728000BB1E0B20FEF792FB9BE7632DA8BF632577
:10729000002303A99D420BDC1CAA25EAE5731344D5
:1072A000002203F8642C152000916B1C2146E9E7AD
:1072B000F2185279CA540133ECE7022C13D0032C94
:1072C00014D0012C7FF47DAF002D7FF77AAF98F8B2
:1072D00005301BB1322BA8BF32231C4664235C430C
:1072E000084B1C606DE7FEF7BBFB6AE7FEF7B9FBD6
:1072F00067E700BF7E740120908601207D74012025
:10730000888E012004000020084B01221A60084AE0
:107310001368002BFCD0074B1868042390FBF3F094
:107320000638400040F00100704700BF00C0004038
:1073300000C1004008C500400120704710B5064C50
:10734000204601F0A5FA0549204601F007FB044B51
:1073500001221A6010BD00BF387B0120801A060090
:107360007C78012010B5064C204601F091FA0549C1
:10737000204601F0F3FA044B01221A6010BD00BF51
:10738000F47B0120801A0600807801201FB50021BF
:107390000E20FCF721FD01210D20FCF71DFD012130
:1073A0000F20FCF719FD1D4801F0CAF91C4B1D49BF
:1073B0001B681D4A8B4212780FD84FF0007301935F
:1073C000002303938DF8082004AB13E90E00134843
:1073D00005B05DF804EB01F0C9B914498B4202D83D
:1073E0004FF08063EBE712498B4202D84FF0006305
:1073F000E5E710498B4202D84FF08053DFE70E4992
:107400008B4202D84FF00053D9E70C498B4294BF0E
:107410004FF080434FF00043D1E700BF187B0120BD
:107420003000002048E801002C00002090D003002C
:1074300020A1070040420F0080841E0000093D008B
:10744000002814DD0B68DA0711D50D4A5B100128FE
:1074500013600C4A09D04B68D90706D55B10022B84
:1074600009D0032B09D0012B03D002231360002085
:1074700070470023FAE70323F8E70123F6E700BF8C
:10748000300000202C000020002810B50EDD0C6814
:10749000E3070BD56410012C08DD054B1B680BB905
:1074A000FFF74CFF2146034801F058FA002010BDB9
:1074B0007C780120387B012008682DE9F843C30758
:1074C00004D40D20BDE8F843FAF7BEB94010FCF72C
:1074D000A7FC051E12DBFCF77DFCA8420EDB022197
:1074E0002846FCF779FC4FF4FA620121284601F0A6
:1074F00033FE28B901462846FCF76EFC002036E032
:10750000DFF8748000244FF00109002707264FF4AC
:107510007A720121284601F01FFE0028EED02828AB
:10752000C4BF09FA06F31F4316F1FF36EFD204F881
:1075300008700134052CE8D100212846FCF74CFCEA
:10754000012206210920FDF7B3F80028D6D0034612
:107550000B2243F8042F074900F1180411F8012FFA
:10756000520042F0010243F8042FA342F6D1BDE8D5
:10757000F88300BF83780120847801200028F8B5C3
:1075800021DD0C6814F001061DD1042C1BD92368E1
:1075900003F00F02032A16D1C3F30F15C3F341738F
:1075A000C3EB8505FFF7F2FE084F0334B54207DD54
:1075B00014F8011F384601F0E6F801362070F5E7AF
:1075C000024801F0DFF80020F8BD00BF187B012061
:1075D00010B50468E30704D40D20BDE81040FAF7A5
:1075E00033B96410FF2C01D91720F6E7FFF7CEFE60
:1075F000E1B2044801F0C7F8024801F0C3F80020E6
:1076000010BD00BF187B012038B5074DFFF7BEFE47
:107610000021284601F0B7F80446284601F0B2F8E8
:10762000600040F0010038BD187B0120274A82B07D
:1076300001210023ADF80630C2F8F015C2F800159C
:1076400019461A0102F1804202F5E0420133082B8B
:10765000C2F81415C2F81015F3D11C4B4FF4E062B8
:10766000C3F818250422C3F81425C3F810250DF11A
:107670000602C3F82C260122C3F830261A60D3F87C
:107680000021002AFBD00022C3F8002101225A6009
:107690000E4B1A46D3F804110029FBD00021C3F881
:1076A000041101219960D2F81431002BFBD0002085
:1076B000C2F81401C2F80005BDF806301BB28342BF
:1076C000C8BFA3F50B70400002B0704700700040C7
:1076D00008B5FFF7ABFF400040F0010008BD000017
:1076E000024A03480F21FEF7E7BD00BF10E000008B
:1076F00088E000000C4B1B6870B506460D4614462A
:107700000BB9FFF71BFEF1B2084801F0A5F9E9B289
:10771000064801F085F8E1B2044801F081F8034819
:10772000BDE8704001F003BA7C780120387B01206D
:1077300008B50368D90705D54168CA0702D582682C
:10774000D00704D40D20BDE80840FAF77DB85810E2
:10775000802801D91520F6E74910FF2901D9162004
:10776000F1E75210FF2A01D91720ECE7FFF7C2FF1B
:10777000002008BD0C4B1B6870B506460D4614462C
:107780000BB9FFF7EFFDF1B2084801F065F9E9B276
:10779000064801F045F8E1B2044801F041F8034819
:1077A000BDE8704001F0C3B980780120F47B01206E
:1077B00001282DE9F04173DD0D68EA0770D5394BDA
:1077C0004C681B686D100BB9FFF7B8FDE9B236487D
:1077D00001F042F914F0010613D06410FF2C02D915
:1077E0001720FAF731F8E1B22F4801F019F82E48C6
:1077F00001F09DF918B12320FAF726F80020BDE822
:10780000F081042CF3D9236803F00F02092A1AD15E
:1078100054F8047FDFF890807F10B742E7DD54F81A
:10782000045FEB070BD56D10FF2D02D91720FAF777
:107830000BF8E9B2404600F0F3FF0136EDE7172000
:10784000FAF702F8F9E7032A15D1261DC4F1FF243F
:10785000C3F30F1504F57F04C3F34173124FC3EB59
:107860008505FC3433199D42C1DD16F8011B3846ED
:1078700000F0D6FFF6E7042AB9D12046FCF77CFDDC
:107880000546204604F074FA074E07462C46631B53
:107890009F42ACDD14F8011B304600F0C1FFF6E753
:1078A0000120ACE77C780120387B012038B5134BF0
:1078B0001B6804460D460BB9FFF740FDE4B22146B4
:1078C0000F4801F0C9F8E9B20D4800F0A9FF002106
:1078D0000B4801F0CBF808B1404238BD01222146E7
:1078E000074801F0B6F8064800F091FF0028F4D0F0
:1078F0000348BDE8384000F08DBF00BF7C78012010
:10790000387B012008B50368D90702D54168CA074A
:1079100004D40D20BDE80840F9F796BF5810802820
:1079200001D91520F6E74910FF2901D91620F1E702
:10793000FFF7BCFF400040F0010008BD38B5124B16
:107940001B6804460D460BB9FFF70CFDE4B2214657
:107950000E4801F081F8E9B20C4800F061FF0B48D5
:1079600001F0E5F808B1404238BD01222146074840
:1079700001F06FF8054800F04AFF0028F4D00348F2
:10798000BDE8384000F046BF80780120F47B01203C
:1079900038B50D211D20FFF7D1FF5A28174C0CD107
:1079A000012222702A211D20FFF7E4FE022001F0AF
:1079B0009BFB134B01221A6038BD0F211920FFF7E2
:1079C000BDFF332805D1022323708F2220211920E7
:1079D000EAE70D211E20FFF7B1FFC7280AD10325D2
:1079E00000222A211E202570FFF7C4FE2A462A21E4
:1079F0001E20D9E700232370D8E700BF3400002001
:107A00008C780120002838B504DC1C20BDE8384003
:107A1000F9F71ABF0B6813F0010401D10D20F5E747
:107A20005B10012B2ADD022B03D0052BB4BF0224EF
:107A30000324194B1B680BB9FFF7AAFF174B93F9E7
:107A40000050022D1CD0032D1ED0012D11D1032C6E
:107A500008BF022400222A211D20FFF78BFE2246A8
:107A60000E211D20FFF786FE2A462A211D20FFF742
:107A700081FE022001F038FB002038BD0024D8E749
:107A8000220123211920F2E7032C14BF22460222EF
:107A90000E211E20EBE700BF8C780120340000206F
:107AA000204B1B6810B504460BB9FFF771FF1E4B46
:107AB00093F90030022B0AD0032B25D0012B26D1BD
:107AC00021461D20FFF73AFF4FF0FF3405E0012C5F
:107AD00013D129211920FFF731FF7F28C8BFA0F556
:107AE00080706FF07E039842B8BF1846C823584391
:107AF0007F2390FBF3F0604310BD032C0BD12B21AF
:107B00001920DFE72D21FBE721461E20DAE74FF0A1
:107B1000FF340020EAE7052CF4D04FF0FF340020BA
:107B2000DFE700BF8C7801203400002008B5012079
:107B3000FFF7B6FF400040F0010008BD08B5032084
:107B4000FFF7AEFF400040F0010008BD08B505207A
:107B5000FFF7A6FF400040F0010008BD38B5134B09
:107B60001B6813B90120FFF79BFF114B93F90030FD
:107B7000013301D1FFF70CFF0120FFF791FF04460D
:107B80000320FFF78DFF05460520FFF789FF6D43B2
:107B900004FB045400FB004003F076F901F0F0FD13
:107BA00003F08CFC400040F0010038BD8C780120CF
:107BB00034000020234B1B6870B506460BB9FFF755
:107BC000D1FB214C94F9001000291BDA0F21192058
:107BD000FFF7B4FE332811D11C4B68221A701C4BDE
:107BE0001E2500221A7060210C2228462570FFF7FE
:107BF000C1FD022261212846FFF7BCFD94F9001067
:107C000000291EDBC9B21348124D00F025FF0F4BAF
:107C10001048197800F004FE0E4800F088FF217823
:107C20000C48062200F015FF741E0536284600F0A9
:107C3000EEFD30B1284600F0EDFD04F8010FB4422E
:107C4000F4D170BD8078012035000020370000207D
:107C500036000020F47B012073B5002368460093B2
:107C6000ADF80430FFF7A6FFFFF7FEF81C4B9DF8B8
:107C7000015093F900609DF802009DF800309DF8D6
:107C800003409DF804209DF8051006B345EA032340
:107C900044EA00201BB200B241EA0222114991F9E4
:107CA0000010102912B202BFDB105210C010002BBE
:107CB000B8BF5B420028B8BF4042002A1844B8BF92
:107CC00052421044400040F0010002B070BD43EA4F
:107CD000052340EA04201BB200B242EA0122DDE79C
:107CE00036000020350000200128F8B535DD0F688A
:107CF000FB0732D54D6815F001062ED1042D2CD985
:107D00002B6803F00F03092B27D16C68144B641008
:107D10001B68202CA8BF20240BB9FFF70FFBC7F36B
:107D2000470122460F480F4F00F093FE0435A6424C
:107D300011DA0C4800F06BFD18B9700040F001003A
:107D4000F8BD384600F066FD400040F0010045F8FF
:107D5000040F0136EBE76000F0E70120F0E700BF19
:107D60007C780120387B01200A4B0B4A30B5D3F8D0
:107D700034450A4BA34208BF1346013B0246FF2489
:107D8000151AA94205DD13F8015F02F8015B1C70AA
:107D9000F6E730BD008002409478012094790120FC
:107DA000064B01225A60DA60D3F85821002AFBD032
:107DB0000022C3F80025024B1A6070470080024081
:107DC0009078012038B52C4B1B680D4623B925202F
:107DD000BDE83840F9F738BD012801DC1C20F7E781
:107DE0000C68E10709D4042C09D9236803F00F03B8
:107DF000DA1E012A05D92420EAE70223F8E7012345
:107E0000F6E76A68D20701D41120E1E7042B0CD110
:107E10002046FCF7B1FA03F0ABFF6A685210013A52
:107E200001D4824209DB1220D2E72068C0F30F128E
:107E3000C0F34170C0EB8200EFE71049D1F8203168
:107E4000C3B1801A80280E4AA8BF802004340023C2
:107E5000834204DA14F8015B9D540133F8E70023F0
:107E6000C1F84805C1F8203101238B60400040F083
:107E7000010038BD1846F9E79078012000800240E3
:107E8000947A012070B5174D174CD5F83435174E3C
:107E90009C4214BF234633464FF480721846FF219C
:107EA00003F0C6FB4FF48073C5F83405C5F83835C8
:107EB0000023C5F8083101232B60D5F8340584422E
:107EC00008BF344604F1FF00A21E0178FF2900F12B
:107ED000FF3301D19A4202D1001B013070BD184618
:107EE000F3E700BF008002409479012094780120DC
:107EF000002838B504DC1C20BDE83840F9F7A4BCE4
:107F00000D68EB0706D4042D04D92B6803F00F038A
:107F1000032B01D02420EFE7124B1B680BB925205F
:107F2000EAE7114BD3F808310BB9012038BDFFF750
:107F3000A9FF041EF9D001DA1B20DDE7284650F81E
:107F4000043BC3F30F12C3F34173C3EB82039C42A0
:107F500028BF1C462146FFF707FF600040F00100E4
:107F6000E4E700BF90780120008002400028F8B5C7
:107F700004DC1C20BDE8F840F9F766BC0968CB07B3
:107F800001D40D20F6E71E4D1E4C2B68491023B17D
:107F9000D4F800350BB1FFF703FF1B4B1A68C4F888
:107FA00014255B68C4F80C354FF486734B43C4F852
:107FB0002435164B4FF48072FF21184603F038FB2E
:107FC0004FF48073C4F83405C4F83835104BC4F846
:107FD00044358023C4F848352023C4F800320026F5
:107FE00001270823C4F800350520C4F8086127607C
:107FF000C4F84865A76001F077F82F603046F8BDF7
:108000009078012000800240CCE3000094780120A9
:10801000947A012070B5124E04460D46002D14DDF1
:10802000D6F8203193B1802D10DC0E4B621914F874
:10803000011B03F8011FA242F9D1094B0022C3F82A
:108040004855C3F8202101229A6070BDFDF766F9FA
:10805000FEF730FDFEF708FF012001F045F8DDE7EF
:1080600000800240937A012006490A6808B52AB1C7
:10807000054BD3F800350BB1FFF792FE00200860E6
:1080800008BD00BF907801200080024038B51C4B2D
:108090001B6823B92520BDE83840F9F7D5BB194B3B
:1080A000D3F8083113B9184D284638BDFFF7EAFE5A
:1080B000041EF8D001DA1B20EDE7E11C0022891034
:1080C0000320FCF7F5FA054608B90A20E3E7214644
:1080D0000430FFF749FEEB07E6D4042DE4D92A6803
:1080E00002F00F03032BDFD104F00303C3F10403F9
:1080F0005B0703F0C04322F0C04213432B60D3E779
:10810000907801200080024038000020002837B518
:1081100004DC1C20F9F798FB03B030BD1C4B1B6836
:108120000BB92520F6E7086810F001040CD04310C5
:10813000FF2B01D92820EDE702A8012100F8013D1D
:10814000FFF768FF0020E7E7042813D9036803F06E
:108150000F02042A10D1FCF70FF9054603F008FEC0
:108160008028014603D92620F9F76EFBEAE7284666
:10817000FFF750FF2046CFE7032AFBD1C3F30F11CF
:10818000C3F34173C3EB81018029ECDC0430EFE7DA
:1081900090780120024A03480621FEF78DB800BFFF
:1081A00034E1000064E100000020704701207047C6
:1081B0000020704700207047012070470020704762
:1081C0000020704700207047002070470020704753
:1081D0000020704700207047002070470020704743
:1081E00000207047002070477047704770470000BC
:1081F000024A03481021FEF75FB800BF84E1000087
:1082000004E200000246104601320378013B1F2BB6
:10821000F9D9704708B5FFF7F5FF0378002B39D07F
:10822000222B00F1010011D1037823B1222B00F1A0
:10823000010204D11046BDE80840FFF7E3BF5C2B04
:1082400002D1437803B1821C1046EDE73A2BF2D0FD
:108250002C2BF0D07B2B0BD1FFF7D4FF0378002B16
:10826000E9D07D2B01D10130E5E7FFF7D3FFF5E73A
:108270005B2B10D00246104612F8013B002BDAD0DF
:10828000202BD8DD2C2B05D003F0DF015D2901D098
:10829000222BF0D108BDFFF7B5FF0378002BCAD021
:1082A0005D2BE0D0FFF7B6FFF7E708B5F0B1FFF7B9
:1082B000A9FF0378222B1AD07B2B1AD05B2B1AD064
:1082C000A3F13002092A05D92D2B05D14278303A85
:1082D000092A07D8032009E0742B0ED0662B0ED094
:1082E0006E2B0ED0181C18BF0120404208BD042080
:1082F000FCE70220FAE70120F8E70520F6E7062070
:10830000F4E70720F2E738B5FFF77CFF03782D2B61
:1083100011D101304FF0FF34431E00210A2501E046
:1083200005FB012113F8012F303AD0B20928F7D903
:1083300004FB01F038BD0124EEE710B51446FFF749
:1083400061FF0378222B02D000230B7010BD621E48
:1083500001300378222BF7D0002BF5D05C2B07D00F
:10836000441C002AF0DD01F8013B013A2046F0E709
:108370004378622B00F1020409D0662B09D06E2BE2
:1083800009D0722B09D0742B08BF0923E9E7082311
:10839000E7E70C23E5E70A23E3E70D23E1E710B560
:1083A0000446FFF737FF0346A342184605D9027873
:1083B000013A1F2A03F1FF33F6D910BD08B590B179
:1083C000037883B1FFF71EFF037803F0DF035D2B13
:1083D00009D0FFF71FFF03782C2B08BF0130BDE841
:1083E0000840FFF70FBF002008BD38B50D1E0DDD9A
:1083F00003785B2B0AD10130FFF704FF0124A5426B
:1084000005D0FFF7DBFF10B10134F8E7002038BDDD
:1084100038B5154609B100230B70F8B10378E3B104
:10842000FFF7F0FE03782C2B044603D10130FFF751
:10843000E9FE044623787D2B0FD019B12A46204649
:10844000FFF77BFF2046FFF7E5FE03783A2B05D1C7
:108450000130BDE83840FFF7D5BE002038BD2DE91A
:10846000F0410D469AB004462F789FB32E2128463E
:1084700003F067FC804690B1461B303F092F13D8AC
:108480002846FFF740FF01462046FFF7AEFF0446AF
:1084900004B3B8F1000F1DD001363544E4E7284697
:1084A00003F066FC0646E8E723787B2B11D1601CBD
:1084B000642201A9FFF7ACFF044658B132462946B1
:1084C00001A803F05DFC0028E2D02046FFF7A2FEE1
:1084D000EEE7002420461AB0BDE8F08138B50D1E45
:1084E00004461CDDFFF7E1FE012807D1601C012DC9
:1084F00000D138BDFFF762FF013DF8E702280ED139
:1085000000221146601CFFF783FF012DF1D0FFF719
:1085100055FF00221146FFF77BFF013DF5E70020E4
:10852000E7E7F8B50C1E074615461E4613DDFFF7B4
:10853000BCFE02280FD132462946781CFFF768FF9F
:10854000012C00D1F8BDFFF739FF32462946FFF76D
:108550005FFF013CF4E70020F4E710B50446C8B122
:10856000FFF750FE03787B2B0AD101300024002254
:108570001146FFF74DFF68B1FFF74CFE0134F6E7F7
:108580005B2B06D101300024FFF718FF10B1013436
:10859000FAE70024204610BD002870B514DD0D68F0
:1085A000EB0711D56D10013DFDF7B4F800264FF033
:1085B000FF3460B916B3304603F0DAFB01463046AB
:1085C000BDE87040FCF7F5B84FF0FF35ECE7036805
:1085D000C3F30742152A0BD1C3F307239C42B8BF4C
:1085E0001C469D4201D100F10806FCF793FFE0E72D
:1085F0001D2A04BF00264FF0FF34F6E7601C400040
:1086000040F0010070BD000010B508680C46FBF793
:10861000B3FEFEF707FC0028A2BF034B626843F8D5
:108620002020002010BD00BF888E012008B50868FA
:10863000FBF7A2FEFEF7F6FB0028AABF024B0120C3
:1086400053F8200008BD00BF888E012008B50868D7
:10865000FBF792FEFEF7E6FB0028ACBF04200020EB
:1086600008BD0000024A03480421FDF725BE00BFF3
:10867000A8E20000A3E2000008B5FBF789FDFBF7C4
:108680004FFEFDF78BFE0448FEF7DDF8FDF792F88C
:10869000BDE80840FEF7BAB9F7E20000FAF7B8BE45
:1086A00038B50025057329B90B4B0C4A0C48252118
:1086B00002F02CFF01600B4951F82220027151F8A1
:1086C000233083719DF8103051F823304371022319
:1086D000C371856038BD00BF0FE300006EE300008A
:1086E0001DE30000CCE30000037B23B943738373D5
:1086F000036101230373704784B00DF1100C0CE982
:108700000E009DF80810026800230129C2F8003508
:10871000039B12D00BD303290CD0C2F85435019B14
:10872000C2F824350123C2F8003504B0704743F085
:108730000203F2E743F00403EFE743F00603ECE73C
:1087400010B5FFF7D1FF03688279C3F80825427995
:10875000C3F80C250279C3F81025034BBDE810407F
:108760000ECBFFF7C9BF00BF2C7B012010B485B032
:1087700001AC84E80E0094E80E0005B05DF8044BEF
:10878000FFF7BABF70470368C3F81C15D3F8082178
:10879000002AFBD0D3F818050022C3F80821C0B284
:1087A0007047000007B5094B09490A484FF080425D
:1087B0001A6000229A6002221A710F2300930E227F
:1087C0000D23FFF76DFF03B05DF804FB2C7B012048
:1087D00000300240187B01202DE9F84380460D4609
:1087E000174601EB02090C464C45A4EB05060BD0DD
:1087F000D8F8003014F8011B1B6840469847002841
:10880000F2D13046BDE8F8833E46FAE770472030A3
:1088100000F03CBA203000F02BBA203000F03CBA17
:1088200038B5437F0D460BB9002038BD00F1680410
:10883000204600F039FA0028F6D12046294600F0FB
:1088400008FA0120F1E700002DE9F0411E4600255D
:108850004FF47A73C0E901530C4B044640F8203BB7
:108860008846174600F0ECF904F1680000F0E8F9DA
:108870009DF8183063769DF81C302676C4E904878D
:10888000A37665772046BDE8F08100BFB4E3000021
:10889000F0B5837E2E4C2F4D0121C17654F8232054
:1088A000437E54F8233012F0200F14BF2F464FF0B0
:1088B000A04702F01F0213F0200F03F01F0308BFB0
:1088C0004FF0A04502F5E07203F5E07340F20C664C
:1088D00047F8226045F8236003694FF0CC72C3F873
:1088E000242503690622C3F80025827E036954F813
:1088F0002220C3F80825427E036954F82220C3F8D9
:108900000C2590F91830144A5C0903F01F039940B4
:1089100004F1600342F8231090F91830002BBDBF1A
:1089200003F00F0302F6FC32D2189B18B5BF4023A8
:108930004022137683F8002390F918300122590958
:1089400003F01F0302FA03F3034A42F82130F0BD9B
:10895000CCE300000003005000E100E0C37EA3B1BF
:1089600003690022C3F800250A4B99420ED90A4B2D
:10897000994294BF4FF080614FF0C8610369C3F81A
:10898000241503690622C3F8002570474FF0CC7107
:10899000F4E700BFA086010090D003002DE9F0416C
:1089A000044688461F461546002A50D000F120068E
:1089B000304600F059F92369C3F8888523690122FC
:1089C0001A622369C3F834652369C3F838552369EB
:1089D0001A602269D2F84C311BB9D2F82431002B2D
:1089E000F8D00023C2F84C312269D2F85C311BB9AF
:1089F000D2F82431002BF8D00023C2F85C31226970
:108A00006FB9D2F8243153B90123D3612369D3F864
:108A10004821002AFBD00022C3F8482109E00123A5
:108A200053612369D3F80421002AFBD00022C3F844
:108A300004212369D3F8242112B10022C3F8242190
:108A40002369D3F83C052066C0B2BDE8F08110462A
:108A5000FBE70123FFF7A2BF10B5044680F8B01072
:108A6000683000F001F90123637710BDF8B50023E9
:108A70004377036990F8B020C3F88825036901267D
:108A80001E62036900F168050446C3F84455284690
:108A90000F4600F0FBF82369C3F8480523699E6080
:108AA0002369D3F850211AB9D3F82421002AF8D029
:108AB0000022C3F85021284600F0E8F8236930B1BD
:108AC000D3F860211AB9D3F82421002AF8D0002263
:108AD000C3F8602123696FB9D3F8242152B9012268
:108AE000DA612369D3F84821002AFBD00022C3F8B9
:108AF000482109E001225A612369D3F80421002AA0
:108B0000FBD00022C3F804212369D3F8240168B103
:108B10000022C3F824212369D3F8C404C3F8C40491
:108B2000022803D004280CBF03200420F8BD012133
:108B3000FFF79CBF70B54369D3F86421044692B136
:108B40000022012500F12006C3F864210577304694
:108B500000F08AF86369C3F8346563694022C3F89A
:108B6000382563691D636369D3F86821DAB100258C
:108B7000C3F8685104F1680601236377257730460E
:108B800000F072F8D4F8B43003B1984763696577A0
:108B90003046C3F8446500F079F86369C3F84805C6
:108BA000636901225A636369D3F8042162B1002228
:108BB000C3F80421237F3BB16369D3F83C05D4F8A3
:108BC000B830206603B198476369D3F8242152B1C5
:108BD0000022C3F824216369D3F8D024C3F8D02439
:108BE000636901225A6170BD0148FFF7A3BF00BF4E
:108BF000387B01200148FFF79DBF00BFF47B0120B7
:108C000007B514231322CDE900324FF0402211465C
:108C100004230848FFF718FE074A08481E231F21AF
:108C2000CDE9003103231146FFF70EFE03B05DF8D6
:108C300004FB00BF387B012000300040F47B0120A2
:108C400008B54022002102F0F3FC0022C0E9102206
:108C500008BD026C10B5531C446C03F03F039C42EA
:108C60001CBF8154036410BD0023C0E9103370475A
:108C7000D0E9102393421FBFC25C013303F03F03CE
:108C8000436414BF10464FF0FF307047D0E91030F6
:108C9000181A48BF40307047D0E91023934214BFE0
:108CA000C05C4FF0FF307047036C406C013303F041
:108CB0003F031B1A58425841704700000649074AB3
:108CC000074B9B1A03DD043BC858D050FBDC00F077
:108CD00013F8F7F7B5FA000070E800000000002074
:108CE00044020020FEE7FEE7FEE7FEE7FEE7FEE7C0
:108CF000FEE7FEE7FEE7FEE7394B1A680D2A08D1CA
:108D00004FF080420021C2F80C11C2F81011C2F8D5
:108D100038151B680D2B46D14FF08052314BD2F8DD
:108D20000414C3F82015D2F80814C3F82415D2F897
:108D30000C14C3F82815D2F81014C3F82C15D2F867
:108D40001414C3F83015D2F81814C3F83415D2F837
:108D50001C14C3F84015D2F82014C3F84415D2F8F7
:108D60002414C3F84815D2F82814C3F84C15D2F8C7
:108D70002C14C3F85015D2F83014C3F85415D2F897
:108D80003414C3F86015D2F83814C3F86415D2F857
:108D90003C14C3F86815D2F84014C3F86C15D2F827
:108DA0004424C3F870250E4B1B680D2B09D14FF0DE
:108DB0008043D3F80024D20744BF6FF00102C3F808
:108DC0000024094AD2F8883043F47003C2F888308E
:108DD000BFF34F8FBFF36F8F044B054A1A60704784
:108DE0003001001000C0004000ED00E03C00002019
:108DF0000090D0030120704703681322DB691847F5
:108E000070470369C3F81C150369D3F81C21002AB5
:108E1000FBD00022C3F81C210120704710B490F948
:108E20005C30144C59090122203103F01F0302FA6F
:108E300003F344F8213003695DF8044B0421C3F8BF
:108E4000081303695A600369DA6003690022C3F8F2
:108E5000002502694FF0FF33C2F80C350269C2F8F1
:108E600014350269C2F8083502691430C2F81035A9
:108E7000FFF7FABE00E100E01430FFF707BF14303F
:108E8000FFF70ABF1430FFF7F3BE0000036990F844
:108E90005E2010B5C3F80C25036990F85D20C3F877
:108EA000142590F861200369012A01BF90F85F4002
:108EB000C3F81045036990F8604006BFC3F8084541
:108EC00003690022B1F5966FC3F86C2569D9B1F535
:108ED000166F69D9B1F5965F69D9B1F5165F68D992
:108EE000B1F5615F67D9B1F5964F66D9B1F5E14F3C
:108EF00065D9B1F5164F64D9B1F5614F64D9B1F5B3
:108F0000963F64D9B1F5E13F63D9B1F5613F63D9CB
:108F1000364B994263D9B1F5E12F63D9B1F5612F91
:108F200094BF4FF070634FF080530269C2F824354C
:108F300003690422C3F8002501690023C1F8083140
:108F40000169C1F81C31016901230B6001698B6063
:108F50000169C1F8042390F95C20510902F01F0255
:108F600093406031224A42F8213090F95C30002B66
:108F7000BDBF03F00F0302F6FC32D2189B18B5BF39
:108F800060236022137683F8002390F95C3001227D
:108F9000590903F01F0302FA03F3154A42F821307E
:108FA00010BD4FF49E23C0E74FF41D23BDE7114BC6
:108FB000BBE7114BB9E7114BB7E7114BB5E7114BC5
:108FC000B3E74FF41D03B0E74FF46B03ADE70E4B6F
:108FD000ABE74FF0EB73A8E74FF06C73A5E74FF0EA
:108FE0008063A2E74FF0E8639FE700BF90D00300E3
:108FF00000E100E000B013000050270000F03A004C
:1090000000A04E0000C0750000903A012DE9F0412B
:109010001E4600254FF47A73C0E901530D4B0446F8
:1090200040F8143B17468846FFF70AFE0A4AC4F880
:10903000108084F85C7052F8263084F85D309DF81A
:10904000183052F8233084F85E3084F8615020469E
:10905000BDE8F08160E40000CCE3000010B50369D6
:10906000D3F8082104464AB1D3F818151430C9B210
:10907000FFF7EFFD23690022C3F8082110BD0000AF
:109080000148FFF7EBBF00BFB07C012007B52223EA
:1090900000930222212303490348FFF7B7FF03B0DF
:1090A0005DF804FB00200040B07C012008B102F014
:1090B0008DBD70470A4B19680A4B30B5D3F80405CB
:1090C0000C060D0A44EA00024FF47A712B46A2FB0B
:1090D000014501FB0355E00B40EA454030BD00BFB0
:1090E000147D01200010014038B5044648B1FFF757
:1090F000E1FF054600F01AF8FFF7DCFF401BA04235
:10910000F8D338BD074B0022C3F8042182B0D3F84E
:109110000431054A0193019B13680133DBB21360EC
:1091200002B0704700100140147D01207047704765
:1091300008B500F067F8FFF7FAFF0120FFF7D4FF4A
:10914000FFF79AFA034CFFF7A9FA002CFBD0AFF314
:109150000080F8E70000000038B5174B174D53F8B2
:109160002030174813F0200F4FF0010403F01F03C5
:1091700004FA03F408BF4FF0A04000292B681149FE
:10918000B3FBF1F300F5A26002FB03F321464FF0BD
:109190000A02B3FBF2F314BF2246002200F014F8D7
:1091A00042F2107358434FF47A722B68B3FBF2F318
:1091B000B0FBF3F038BD00BFCCE300003C00002062
:1091C0000003005040420F0030B504680C40944248
:1091D00006D1013B002BF8D112E0013B002B0FD050
:1091E00004680C409442F8D1002405680D40954273
:1091F00004D101349C42F8D1002002E0201C00E0A0
:10920000181C30BD0D4BE02283F811234FF40032BF
:10921000C3F880211A604FF080430122C3F818255B
:109220009A6003F588330021C3F808150221C3F8BA
:109230000413C3F844131A60704700BF00E100E054
:10924000014B1860704700BF580000200228064AF2
:10925000064B1BBF002111600121012212BF1A60C1
:1092600011601860704700BF207D0120540000206D
:10927000222837B50CD84B4B53F82030052B00F083
:10928000828007D8032B12D07BD8022B00F081807C
:10929000002074E01D2B78D003D81C2BF8D10522B8
:1092A00006E01E2B73D01F2BF2D1082200E0022211
:1092B0003D4B196808296EDD0A296FDD0D29B5BF00
:1092C0000C240E24022303233848C0F8F035012370
:1092D000C0F8003500200546030103F1804303F583
:1092E000E04301300828C3F81455C3F81055F3D1F2
:1092F0002F4B18682F4B1B6800021B0303F480538D
:1093000000F4E0601843294BC3F81805C3F814258E
:10931000C3F810250DF10602C3F82C260122C3F86C
:1093200030261A60D3F80021002AFBD00022C3F8AF
:10933000002101225A601D4B1A46D3F8040100286F
:10934000FBD00020C3F8040101209860D2F814314A
:10935000002BFBD00023C2F81431BDF906209A423D
:10936000124AB8BFADF80630A142C2F80035BDF9C7
:10937000060004D035BF611A091BC840884003B0FD
:1093800030BD032294E7042292E7062290E70722E9
:109390008EE701228CE70824002395E70A240123A5
:1093A00092E700BFCCE300005000002000700040B6
:1093B00054000020207D0120222830B53CD8224BCB
:1093C00053F82000214B00221D4653F82240B4F1EF
:1093D000FF3F32D11E4C45F822006FEA41411D4D3E
:1093E0001D4B246853F822306FEA514125F81210C2
:1093F000012101FA04F4C3F86005013CC3F86405D7
:1094000005EB4202C3F86805C3F86C050020C3F8F9
:109410000015C3F80C05C3F80405C3F80845C3F8E4
:109420001405C3F81005C3F82025C3F82415C3F8A4
:109430002815C3F82C05996030BD8442CAD001328A
:10944000042AC2D1F8E700BFCCE3000040000020AE
:1094500058000020187D012088E40000222815D83B
:10946000114B124A53F8203013F0200F08BF4FF071
:10947000A04203F01F03032908D8DFE801F002101F
:10948000080C03F5E073002142F82310704703F540
:10949000E0730C21F8E703F5E0730421F4E703F52A
:1094A000E0730321F0E700BFCCE3000000030050AD
:1094B000222813D80A4B53F820000A4B10F0200F33
:1094C0004FF0010200F01F0008BF4FF0A0438240A0
:1094D00011B9C3F80C257047C3F80825704700BFC1
:1094E000CCE3000000030050222810D8094B0A4AA0
:1094F00053F8203013F0200F08BF4FF0A04203F0C4
:109500001F03D2F81005D84000F00100704700207A
:10951000704700BFCCE30000000300502DE9F0418C
:1095200006460D4601EB02080C464445A4EB050730
:1095300007D0336814F8011B1B6830469847002891
:10954000F3D13846BDE8F0812DE9F041C1F30A5767
:10955000A7F2FF35132D82B002460B460C464FEAA8
:10956000D178064633DC002D4EDB3C49294103EA25
:109570000100104326D049080B4052EA03060CD0E4
:109580004FF48023132D24EA010143FA05F444EA41
:1095900001040CBF4FF000460026314901EBC8081A
:1095A0002346D8E9004532462046294601F020FBF3
:1095B000CDE9000122462B46DDE9000101F016FB52
:1095C00002460B461046194602B0BDE8F081332D25
:1095D00007DDB5F5806FF5D101F00AFB02460B46B9
:1095E000F0E7A7F213474FF0FF31F9400842E9D006
:1095F00049080842D1D04FF0804320EA010143FAE4
:1096000007F741EA0706C8E721F000410143D9D036
:10961000C3F3130101434E420E43114D5C0C360B54
:10962000640406F4002305EBC80243EA0401D2E90E
:1096300000450B4602462946204601F0D9FACDE9FD
:10964000000122462B46DDE9000101F0CFFA21F0AE
:109650000041024641EAC873B4E700BFFFFF0F00B4
:1096600098E40000F8B5C1F30A57A7F2FF35132DAF
:1096700002460B460C4610DC002D29DB8C461D49AA
:1096800029410B422AD04FF400242C41644424EA9F
:109690000104002621463046F8BD332D05DDB5F521
:1096A000806F1ED010461946F8BDA7F213474FF041
:1096B000FF3121FA07F73842F4D00123C5F1330511
:1096C00003FA05F5461928BFE41826EA0706E1E77C
:1096D000013501F0004407D00026DBE70028D2D195
:1096E000E0E701F085FAF8BD44F07F5444F44014FB
:1096F0000026CFE7FFFF0F0030B51F4A21F00043DF
:10970000934287B01CDD1D4A934205DD02460B469D
:1097100001F06CFA07B030BD02AA00F091F800F039
:1097200003000128DDE9042312D002281CD0A0B1D7
:10973000DDE9020100F068FB01F1004107B030BD36
:10974000002300930022002301F086F807B030BD0B
:10975000DDE9020100F058FBDCE70124DDE902014C
:10976000009401F079F8D5E70124DDE902010094C5
:1097700001F072F8E0E700BFFB21E93FFFFFEF7F58
:109780002DE9F04F8BB004460D4600F07BFA294BD3
:1097900093F900A0BAF1FF3F06460F4612D02246C9
:1097A0002B462046294601F073FE834650B94FF000
:1097B00000084FF000092046294642464B4601F07A
:1097C0003FFE20B9304639460BB0BDE8F08F01228C
:1097D000194BCDF820B00092CDE90445CDE9024502
:1097E0000193BAF1000F17D042464B464046494616
:1097F00001F0DEFCBAF1020FCDE906010ED101F055
:10980000A3FE21230360089B73B9DDE90667304698
:1098100039460BB0BDE8F08FCDE90689684601F006
:1098200057F90028EFD1EAE701F08EFE089B0360AC
:10983000EBE700BF5C000020A8E40000000000008F
:109840002DE9F047CA4B21F000479F4290B0804677
:10985000894640F38F80C74B9F420C46924626DCD8
:109860000029B9A3D3E9002340F38F8001F0BEF9AA
:10987000C14B9F4204460D4600F04781B4A3D3E993
:10988000002301F0B3F902460B46CAE90023204643
:10989000294601F0ABF9AEA3D3E9002301F0A6F904
:1098A0000125CAE90201284610B0BDE8F087B34B94
:1098B0009F4240F38980B24B9F4200F31C813D15CB
:1098C000A5F21645A7EB055319461F46064601F0BB
:1098D000F5FD01F0D9FA8046894642464B463046AE
:1098E0003946CDE90A8901F081F90022A54B01F042
:1098F00035FB8946804601F0E1FD01F0C5FA0646D8
:109900000F4632463B4640464946CDE90C6701F0DA
:109910006DF900229B4B01F021FB00220023CDE9D1
:109920000E0101F083FD002800F060810023304625
:109930003946002201F07AFD002814BF01230223DA
:10994000914A019202212A4600910AA8514600F04C
:1099500083FB002C054614DADAF80420DAF80C3020
:1099600002F1004203F100434542CAF80420CAF85C
:109970000C3006E000200021C2E90089C2E90201A2
:109980000025284610B0BDE8F08701F031F97A4B88
:109990009F4204460D4600F00B816DA3D3E90023DE
:1099A00001F026F902460B46CAE900232946204663
:1099B00001F01CF966A3D3E9002301F019F94FF077
:1099C000FF35CAE90201DCE700F0FCFF62A3D3E93E
:1099D00000238046894601F0C1FA00226B4B01F05A
:1099E00007F901F06BFD054601F04EFA56A3D3E9E5
:1099F0000023CDE9060101F0B1FA02460B464046CC
:109A0000494601F0F3F852A3D3E900238046894682
:109A1000DDE90601CDE9028901F0A0FA1F2D024619
:109A20000B46CDE9042340F3B380DDE90423DDE9EF
:109A3000020101F0DBF8804689463F15C9F30A535D
:109A4000FB1A102B40F3B18045A3D3E90023DDE9D5
:109A5000060101F083FA8046894602460B46DDE99D
:109A6000020101F0C3F802460B46DDE90201CDE92F
:109A7000082301F0BBF842464B4601F0B7F83AA381
:109A8000D3E9002380468946DDE9060101F066FA44
:109A900042464B4601F0AAF80B46CDE904010246C6
:109AA000DDE9080101F0A2F8C1F30A53FF1A312FD2
:109AB0008046894600F39C809DED087BCAE90089B9
:109AC0008DED027B42464B46DDE9020101F08EF846
:109AD000DDE9042301F08AF8002CCAE90201BFF68F
:109AE00050AF09F1004401F100436D42CAE900841E
:109AF000CAE9020345E702460B4601F077F8002564
:109B0000CAE90201CAE900013BE715A3D3E9002332
:109B100001F06CF814A3D3E900230D46044601F0CC
:109B200065F802460B46CAE900232946204601F0A3
:109B30005DF80DA3D3E9002301F058F80125CAE927
:109B400002011EE7AFF3008000004054FB21F93F03
:109B50003163621A61B4D03D83C8C96D305FE43FA0
:109B60000000601A61B4D03D7370032E8A19A33BC4
:109B7000FB21E93F7BD90240FB21F93FFB21394121
:109B8000FFFFEF7F0000704130E500000000E03F84
:109B90004046494601F02AF8394B6A1E804653F880
:109BA0002230BB4289463FF448AFCAE9008989E7C1
:109BB0002BA3D3E9002301F01BF82BA3D3E9002347
:109BC0000D46044601F014F802460B46CAE900238C
:109BD0002946204601F00AF823A3D3E9002301F027
:109BE00007F84FF0FF35CAE90201CAE60323A7E6EA
:109BF0001FA3D3E90023DDE9060101F0AFF9064612
:109C00000F4602460B46DDE9080100F0EFFF8046F3
:109C1000894602460B46DDE90801CDE9028900F0DC
:109C2000E5FF32463B4600F0E1FF13A3D3E90023F2
:109C300006460F46DDE9060101F090F932463B4643
:109C400000F0D4FF02460B4640464946CDE90423C6
:109C500000F0CCFF80468946A7E700BFAFF3008045
:109C60000000601A61B4D03D7370032E8A19A33BC3
:109C70000000002E8A19A33BC14920259A837B3915
:109C8000B0E400005E4A8A432DE9F04104460D46E7
:109C900000F0958000290B460646844656DD0F15D8
:109CA00000F0A580C3F31303A7F2FF3743F480133A
:109CB0004FEADC72F80702EB43034FEA4C0504D588
:109CC000ED0F05EB43034FEA8C0500267F10B446E9
:109CD00016224FF400110CEB010098424FEAD574A4
:109CE0004FEA450503DC1B1A00EB010C0E44013A58
:109CF00004EB43034FEA5101EDD110469646202470
:109D00004FF0004209E051D05B00013C03EBD573FA
:109D10004FEA52024FEA450537D0634502EB0E0188
:109D2000F1DD002901EB020E0ADBE046A3EB0C0398
:109D3000A94288BF03F1FF336D1A1044C446E3E71C
:109D4000BEF1000FF1DB0CF10108EFE721F000425A
:109D5000024329D0002942D10146CA0A153B4905D0
:109D6000002AFAD012F4801001D044E0604652007C
:109D7000D40200F1010CF9D5CCF1200401FA0CFC5D
:109D8000E1401F1A41EA02038CE72B4321D144082A
:109D9000731003F17F53F20703F5001348BF44F03B
:109DA000004403EB07512046BDE8F081A942ABD83F
:109DB000002901EB020EC3DB98460023BCE70246F4
:109DC0000B4601F0CBF822462B4600F011FFBDE810
:109DD000F081411C16BF421C01365408D8E70246E8
:109DE00000F004FF02460B4601F0E2F9DCE71A46F8
:109DF00031463B46B6E78C4620244FF0FF30BFE7A4
:109E00000000F07F000000002DE9F04F21F0004835
:109E1000B8F1795F85B006460F4692469B466BDAED
:109E200001F04CFB002800F0E18032463B46304612
:109E3000394601F093F874A3D3E9002304460D4694
:109E400001F08CF872A3D3E9002300F0D1FE224682
:109E50002B4601F083F870A3D3E9002300F0C6FE7F
:109E600022462B4601F07AF86DA3D3E9002300F0D7
:109E7000BFFE22462B4601F071F86BA3D3E9002305
:109E800000F0B4FE22462B4601F068F868A3D3E93F
:109E9000002300F0ADFE22462B4601F05FF8CDE92D
:109EA00000010022664B2046294601F057F8DDE903
:109EB0000023804689462046294601F04FF8524645
:109EC00004460D465B463046394601F047F80246E7
:109ED0000B462046294600F089FE02460B464046C6
:109EE000494600F083FE02460B460020554900F02B
:109EF0007DFE05B0BDE8F08F02460B4601F02EF85E
:109F000041A3D3E9002304460D4601F027F840A3FE
:109F1000D3E9002300F06CFE22462B4601F01EF828
:109F20003DA3D3E9002300F061FE22462B4601F059
:109F300015F83BA3D3E9002300F05AFE22462B4636
:109F400001F00CF838A3D3E9002300F04FFE2246BD
:109F50002B4601F003F836A3D3E9002300F048FEB6
:109F60002B46224600F0FAFF374B9845CDE9000119
:109F700097DD364B98453EDCA8F500130022002003
:109F800030499046994600F031FECDE902010022A9
:109F90002B4B2046294600F0E1FF42464B4600F09D
:109FA00025FEDDE90023804689462046294600F04B
:109FB000D5FF524604460D465B463046394600F012
:109FC000CDFF02460B462046294600F00FFE024612
:109FD0000B464046494600F009FE02460B46DDE9C5
:109FE000020100F003FE05B0BDE8F08F1549002026
:109FF00005B0BDE8F08F9FED107B4FF000088DEDB0
:10A00000027BDFF84C90C2E7D43888BEE9FAA8BDDD
:10A01000C4B1B4BD9EEE213EAD529C804F7E923EB7
:10A020009015CB19A001FA3E7751C1166CC1563F6D
:10A030004C5555555555A53F000000000000E73F21
:10A040000000E03F0000F03F3233D33F0000E93F23
:10A050000000D23F000000002DE9F04FADF5197D62
:10A06000BE4CA29EBE4D54F826600793D41E85FBBD
:10A070000475E417C4EBA50424EAE4741D46631CCC
:10A08000A3EB8303013D02EBC3030593731904960D
:10A090000994019503900B91A4EB05071AD43B4456
:10A0A000002400255E1C0DF18008DDF88C9208E08C
:10A0B00059F8270000F0E8FE0137B742E8E802014E
:10A0C00008D0002FF4DA013720462946B742E8E8E5
:10A0D0000201F6D1049B002B079B4FEAC3030293B6
:10A0E0002ADB039A20A902EB030801EB0309049B76
:10A0F00072AA02EBC30B0DF5E07A019B002B4FF027
:10A1000000064FF0000711DB039C4D4675E9022362
:10A11000F4E8020100F022FF02460B4630463946C1
:10A1200000F066FD444506460F46EFD1EAE80267B7
:10A13000DA4509F10809E0D1DDE902040499204477
:10A140008B0082460BA8A3F10802C31808930CAB3E
:10A1500013440A938B4698AB03EBCB03BBF1000F80
:10A1600053E9284529DD70AB03EBCB080DF130092D
:10A1700000227C4B2046294600F0F0FE01F09EF9BB
:10A1800000F082FE0022784B06460F4600F0E6FE05
:10A1900002460B462046294600F028FD01F08EF9C4
:10A1A00078E9022349F8040B3946304600F020FDD7
:10A1B00070AB984504460D46DAD1DDF81490204680
:10A1C00029464A4600F088FC00224FF07F5304469F
:10A1D0000D4600F0C3FE00F0FBFB0022634B00F0D5
:10A1E000BDFE02460B462046294600F0FFFC0D4608
:10A1F000044601F063F9804600F046FE0B46024635
:10A200002946204600F0F2FC4B46002B06460F463E
:10A2100040F3E1800BF1FF320CA9C9F1180351F8AA
:10A22000225045FA03F101FA03F30CA8EB1A40F8A7
:10A230002230C9F11705884443FA05F5002D2CDDBD
:10A24000BBF1000F08F1010840F381820C9C002C47
:10A2500040F0A780BBF1010F0AD00CA9012251F8F0
:10A26000044F531C002C40F09E809B451A46F6D1AB
:10A27000059B002B0EDD012B00F0D980022B09D1AC
:10A280000BF1FF320CAB0CA953F82230C3F31503CA
:10A2900041F82230022D00F0AF800022002330462A
:10A2A000394601F0C3F8002800F05382049B0BF1FB
:10A2B000FF394B4510DC0BF180430CAA013B089899
:10A2C00002EB8303002253F80419834242EA01029D
:10A2D000F9D1002A40F0B680049B0CAA013B52F849
:10A2E0002330002B40F0A1800A9A012352F8041970
:10A2F00001330029FAD05B440BF10109994506931B
:10A300004CDC099A079909EB020801EB0B0508F1EF
:10A31000804802EB030BA39B08F1FF3803EB88088E
:10A3200070AB03EBC909A39B20A903EB8B0301EBE3
:10A33000C505029358F8040F00F0A6FD0B460199DD
:10A340000246002905F1080BC5E900234FF000067D
:10A350004FF000071CDB039C0CE000BF78E6000018
:10A36000ABAAAA2A0000703E000070410000204005
:10A3700075E90223F4E8020100F0F0FD02460B4605
:10A380003046394600F034FC544506460F46EFD1BE
:10A39000029B9845E9E802675D46CBD1DDF818B02D
:10A3A000D9E6012300220CA9C4F180749B4541F831
:10A3B00022400EDD51F8232001EB8B0001EB8303DB
:10A3C0006FF07F4100E01A688A1A43F8042B834239
:10A3D000F9D101244CE706D10BF1FF330CAA52F856
:10A3E0002350ED152AE700227B4B01F03DF80028B1
:10A3F00040F0A381054650E732463B4600207749AE
:10A4000000F0F4FB06460F46002C3FF446AF059AD9
:10A410007249002000F060FB02460B463046394688
:10A4200000F0E4FB06460F4637E7012363E70BF134
:10A43000FF320CAB0CA953F82230C3F3160341F8DA
:10A44000223027E70CAB059A53F82930183ACDE9AA
:10A45000068505926BB909F18043013B0CA901EB1C
:10A46000830353F8041909F1FF39183A0029F8D089
:10A470000592059A5949002000F02EFBB9F1000F12
:10A4800004460D46C0F2C0814FEAC90370AA02EB30
:10A49000030808930CAB03EB8906DFF844B14FF0D7
:10A4A000000A08F10807043656F8040D00F0ECFC29
:10A4B00022462B4600F052FD5B4667E902015246F8
:10A4C0002046294600F04AFD0CAB9E4204460D464C
:10A4D000EAD148AB03930193CDF8149009F101033D
:10A4E000DDF810900293C3464FF0000AB9F1000F57
:10A4F000C0F22A81DFF8EC805D4635A3D3E9002362
:10A5000000260027002403E0544510DCF8E802236D
:10A51000F5E8020100F022FD02460B4630463946BE
:10A5200000F066FB0134A14506460F46ECDA019BBC
:10A53000E3E802670193029B0AF1010A9A45ABF135
:10A54000080BD3D1A29BDDF81490032B39D8DFE898
:10A5500013F0D900060006004D0048AB0393B9F193
:10A56000000F4FF000004FF0000109DB039D05EBE9
:10A57000C904083474E9022300F03AFBA542F9D17A
:10A58000079B002B40F01E810B9BC3E900010B468B
:10A5900003990246D1E9000100F028FBB9F1000F50
:10A5A0000CDD4AAD01240134F5E8022300F020FB64
:10A5B000A145F8DA079B002B40F014810B9BC3E9FF
:10A5C0000201069B03F007000DF5197DBDE8F08F31
:10A5D00000000040FB21F93F0000E03F0000F03F99
:10A5E0000000703E40E6000048AB0393B9F1000F55
:10A5F00040F32781039ACDF810904FEAC9030193E5
:10A60000D318D3E900AB09F10053013B02EBC908B1
:10A610000293914678E9026752465B4630463946D6
:10A6200000F0E6FA04460D4602460B46304639462F
:10A6300000F0DCFA52465B4600F0DAFAC145A24669
:10A64000AB46C8E90201C8E90045E3D1DDF8109046
:10A65000B9F1010F40F3F580019B039A029913446D
:10A66000C900D3E9006701F1080A019192440DF590
:10A67000947B7AE9028932463B464046494600F0DF
:10A68000B7FA04460D4602460B464046494600F0DE
:10A69000ADFA32463B4600F0ABFAD34526462F468C
:10A6A000CAE90201CAE90045E3D1019C039B1034C9
:10A6B000002000211C4403F1100574E9022300F07E
:10A6C00097FAA542F9D1039C079ED4E90023D4E967
:10A6D0000245002E00F08A8003F1004701F100439B
:10A6E0000B99C1E90403069B2646944605F10044F4
:10A6F00003F00700C1E900C7C1E902640DF5197D47
:10A70000BDE8F08F089C039D0834002000212C44F4
:10A7100074E9022300F06CFAA542F9D1079B13B14A
:10A7200001F1004319460B9BC3E90001069B03F0AE
:10A7300007000DF5197DBDE8F08FBBF1000F08F1A2
:10A74000010874DD022581E500260027EFE60024DC
:10A750008EE5CDE90685059D304639466A4200F012
:10A76000BBF90022384B06460F4600F07DFE00B3D1
:10A770000022364B3046394600F0F0FB00F09EFEDA
:10A78000044600F081FB00222F4B00F0E7FB0B4654
:10A7900002463946304600F029FA00F08FFE0BF1F0
:10A7A00001090CAB183543F82B00059543F82940F7
:10A7B0005FE63046394600F081FE0CABD94643F8DF
:10A7C0002B0056E60B9C01F10043C4E900030B4645
:10A7D00003990246D1E9000100F008FAB9F1000F2F
:10A7E0003FF7DFAE01F100431946E7E60B9EC6E9ED
:10A7F0000023069BC6E9040103F00700C6E90245F1
:10A800000DF5197DBDE8F08FA29B032B3FF6D9AE65
:10A8100001A252F823F000BF29A800005BA50000A8
:10A820005BA50000E9A500000020002176E7324684
:10A830003B460020064900F0D9F9022506460F469E
:10A840002BE5002000213EE7000070410000703E33
:10A850000000F03F000000002DE9F04F21F000461D
:10A86000B6F1795F85B004460D469046994604DA04
:10A8700000F024FE002800F0858022462B4620466A
:10A88000294600F06BFB06460F4602460B46204663
:10A89000294600F063FB41A3D3E9002382468B469F
:10A8A0003046394600F05AFB3EA3D3E9002300F0BE
:10A8B0009DF932463B4600F051FB3CA3D3E900230F
:10A8C00000F096F932463B4600F048FB39A3D3E945
:10A8D000002300F08BF932463B4600F03FFB37A3E4
:10A8E000D3E9002300F084F90E9BCDE900019BB36E
:10A8F0000022294B4046494600F030FBDDE90023A9
:10A90000CDE902015046594600F028FB02460B46AD
:10A91000DDE9020100F06AF932463B4600F01EFB19
:10A9200042464B4600F062F919A3D3E900230646DC
:10A930000F465046594600F011FB02460B46304682
:10A94000394600F055F902460B462046294600F0EC
:10A950004DF905B0BDE8F08F02460B46304639464A
:10A9600000F0FCFA0AA3D3E9002300F03FF95246B5
:10A970005B4600F0F3FA22462B4600F039F905B0A9
:10A98000BDE8F08F2046294605B0BDE8F08F00BF36
:10A99000495555555555C53F0000E03F7CD5CF5A28
:10A9A0003AD9E53DEB9C2B8AE6E55A3E7DFEB15750
:10A9B000E31DC73ED561C119A0012A3FA6F81011B9
:10A9C0001111813F21F0004319467047000000003B
:10A9D0002DE9F041C1F30A57A7F2FF35132D0246C6
:10A9E0000B460C46884606461DDC002D3CDB364FE8
:10A9F0002F4101EA070C5CEA000C19D030A3D3E91F
:10AA0000002300F0F5F80022002300F037FDC8B362
:10AA1000002C04DA4FF4801343FA05F5A84428EA21
:10AA2000070400262EE0332D06DDB5F5806F2DD00E
:10AA300010461946BDE8F081A7F213474FF0FF3CDE
:10AA40002CFA07F70742F3D01DA3D3E9002300F047
:10AA5000CFF80022002300F011FD98B1002C21DB7B
:10AA600026EA070644460DE015A3D3E9002300F0CB
:10AA7000BFF80022002300F001FD18B1002C08DB14
:10AA80000026344621463046BDE8F08100F0B0F89B
:10AA9000D0E724F000430D4A1E43002E18BF144691
:10AAA0000026EFE7142D08D00123C5F1340503FA81
:10AAB00005F5AE1928BF9844D2E704F10108CFE7A5
:10AAC0009C7500883CE4377EFFFF0F000000F0BF5C
:10AAD0000020704700000000F8B5C1F30A53044697
:10AAE0000D460E4617460BBB21F000460346334386
:10AAF0001BD0354B002200F031FA344B9F42044604
:10AB00000D4635DBC1F30A530E46363B3B4440F25B
:10AB1000FE72934232DC002B11DD26F0FF4626F454
:10AB2000E00646EA035520462946F8BD40F2FF728A
:10AB30009342EBD102460B4600F05AF8F8BD13F1F0
:10AB4000350F28DA4CF250339F4222462B460ADD5D
:10AB500019A1D1E9000100F03DF817A3D3E90023C2
:10AB600000F0FCF9F8BD16A1D1E9000100F032F8BF
:10AB700013A3D3E9002300F0F1F9F8BD22462B46D8
:10AB80000DA1D1E9000100F025F80BA3D3E90023C2
:10AB900000F0E4F9F8BD26F0FF4626F4E00636336F
:10ABA00046EA0355204629460022094B00F0D6F913
:10ABB000F8BD00BFAFF300809C7500883CE4377E91
:10ABC00059F3F8C21F6EA50100005043B03CFFFFCF
:10ABD0000000903C03F0004321F0004242EA0301F0
:10ABE000704700BF81F0004102E000BF83F00043E6
:10ABF00030B54FEA41044FEA430594EA050F08BF18
:10AC000090EA020F1FBF54EA000C55EA020C7FEADB
:10AC1000645C7FEA655C00F0E2804FEA5454D4EB58
:10AC20005555B8BF6D420CDD2C4480EA020281EA22
:10AC3000030382EA000083EA010180EA020281EA5A
:10AC40000303362D88BF30BD11F0004F4FEA0131AC
:10AC50004FF4801C4CEA113102D0404261EB4101BB
:10AC600013F0004F4FEA03334CEA133302D0524241
:10AC700063EB430394EA050F00F0A780A4F10104FD
:10AC8000D5F1200E0DDB02FA0EFC22FA05F2801837
:10AC900041F1000103FA0EF2801843FA05F359411D
:10ACA0000EE0A5F120050EF1200E012A03FA0EFC9C
:10ACB00028BF4CF0020C43FA05F3C01851EBE371C6
:10ACC00001F0004507D54FF0000EDCF1000C7EEBE3
:10ACD00000006EEB0101B1F5801F1BD3B1F5001F21
:10ACE0000CD349085FEA30004FEA3C0C04F1010440
:10ACF0004FEA445212F5800F80F09A80BCF1004F69
:10AD000008BF5FEA500C50F1000041EB045141EAEA
:10AD1000050130BD5FEA4C0C404141EB010111F4EB
:10AD2000801FA4F10104E9D191F0000F04BF014696
:10AD30000020B1FA81F308BF2033A3F10B03B3F174
:10AD400020020CDA0C3208DD02F1140CC2F10C0204
:10AD500001FA0CF021FA02F10CE002F11402D8BF62
:10AD6000C2F1200C01FA02F120FA0CFCDCBF41EA2E
:10AD70000C019040E41AA2BF01EB0451294330BDFD
:10AD80006FEA04041F3C1CDA0C340EDC04F11404DA
:10AD9000C4F1200220FA04F001FA02F340EA0300B1
:10ADA00021FA04F345EA030130BDC4F10C04C4F1F7
:10ADB000200220FA02F001FA04F340EA03002946D7
:10ADC00030BD21FA04F0294630BD94F0000F83F421
:10ADD000801306BF81F480110134013D4EE77FEA04
:10ADE000645C18BF7FEA655C29D094EA050F08BF50
:10ADF00090EA020F05D054EA000C04BF1946104631
:10AE000030BD91EA030F1EBF0021002030BD5FEA74
:10AE1000545C05D14000494128BF41F0004130BD9C
:10AE200014F580043CBF01F5801130BD01F00045F0
:10AE300045F0FE4141F470014FF0000030BD7FEA63
:10AE4000645C1ABF194610467FEA655C1CBF0B465E
:10AE5000024650EA013406BF52EA033591EA030F75
:10AE600041F4002130BD00BF90F0000F04BF00216D
:10AE7000704730B54FF4806404F132044FF00005A0
:10AE80004FF0000150E700BF90F0000F04BF002119
:10AE9000704730B54FF4806404F1320410F000457F
:10AEA00048BF40424FF000013EE700BF42004FEA7A
:10AEB000E2014FEA31014FEA02701FBF12F07F43F7
:10AEC00093F07F4F81F06051704732F07F4208BFAE
:10AED000704793F07F4F04BF41F40021704730B5B5
:10AEE0004FF4607401F0004521F000411CE700BF01
:10AEF00050EA010208BF704730B54FF000050AE084
:10AF000050EA010208BF704730B511F0004502D584
:10AF1000404261EB41014FF4806404F132045FEA86
:10AF2000915C3FF4D8AE4FF003025FEADC0C18BF2F
:10AF300003325FEADC0C18BF033202EBDC02C2F121
:10AF4000200300FA03FC20FA02F001FA03FE40EAB3
:10AF50000E0021FA02F11444BDE600BF70B54FF0B7
:10AF6000FF0C4CF4E06C1CEA11541DBF1CEA135595
:10AF700094EA0C0F95EA0C0F00F0DEF82C4481EAFD
:10AF8000030621EA4C5123EA4C5350EA013518BF1D
:10AF900052EA033541F4801143F4801338D0A0FB0A
:10AFA00002CE4FF00005E1FB02E506F00042E0FBB7
:10AFB00003E54FF00006E1FB03569CF0000F18BFBD
:10AFC0004EF0010EA4F1FF04B6F5007F64F5407465
:10AFD00004D25FEA4E0E6D4146EB060642EAC621F8
:10AFE00041EA55514FEAC52040EA5E504FEACE2E65
:10AFF000B4F1FD0C88BFBCF5E06F1ED8BEF1004F68
:10B0000008BF5FEA500E50F1000041EB045170BDE3
:10B0100006F0004646EA010140EA020081EA030127
:10B02000B4EB5C04C2BFD4EB0C0541EA045170BD23
:10B0300041F480114FF0000E013C00F3AB8014F19D
:10B04000360FDEBF002001F0004170BDC4F10004E6
:10B05000203C35DA0C341BDC04F11404C4F1200567
:10B0600000FA05F320FA04F001FA05F240EA0200C2
:10B0700001F0004221F0004110EBD37021FA04F6F8
:10B0800042EB06015EEA430E08BF20EAD37070BDB2
:10B09000C4F10C04C4F1200500FA04F320FA05F011
:10B0A00001FA04F240EA020001F0004110EBD37013
:10B0B00041F100015EEA430E08BF20EAD37070BD83
:10B0C000C4F1200500FA05F24EEA020E20FA04F35C
:10B0D00001FA05F243EA020321FA04F001F000410B
:10B0E00021FA04F220EA020000EBD3705EEA430E7C
:10B0F00008BF20EAD37070BD94F0000F0FD101F0AB
:10B100000046400041EB010111F4801F08BF013CE3
:10B11000F7D041EA060195F0000F18BF704703F021
:10B120000046520043EB030313F4801F08BF013DA8
:10B13000F7D043EA0603704794EA0C0F0CEA135564
:10B1400018BF95EA0C0F0CD050EA410618BF52EA1E
:10B150004306D1D181EA030101F000414FF0000024
:10B1600070BD50EA410606BF1046194652EA430632
:10B1700019D094EA0C0F02D150EA013613D195EAA6
:10B180000C0F05D152EA03361CBF104619460AD1EE
:10B1900081EA030101F0004141F0FE4141F47001F8
:10B1A0004FF0000070BD41F0FE4141F4780170BDE8
:10B1B00070B54FF0FF0C4CF4E06C1CEA11541DBF4D
:10B1C0001CEA135594EA0C0F95EA0C0F00F0A7F84F
:10B1D000A4EB050481EA030E52EA03354FEA01317C
:10B1E00000F088804FEA03334FF0805545EA13138F
:10B1F00043EA12634FEA022245EA111545EA106557
:10B200004FEA00260EF000419D4208BF964244F1ED
:10B21000FD0404F5407402D25B084FEA3202B61A0C
:10B2200065EB03055B084FEA32024FF480104FF4E0
:10B23000002CB6EB020E75EB030E22BFB61A754654
:10B2400040EA0C005B084FEA3202B6EB020E75EBE7
:10B25000030E22BFB61A754640EA5C005B084FEA4F
:10B260003202B6EB020E75EB030E22BFB61A75461C
:10B2700040EA9C005B084FEA3202B6EB020E75EB27
:10B28000030E22BFB61A754640EADC0055EA060EE8
:10B2900018D04FEA051545EA16754FEA06164FEA2B
:10B2A000C30343EA52734FEAC2025FEA1C1CC0D1D7
:10B2B00011F4801F0BD141EA00014FF000004FF064
:10B2C000004CB6E711F4801F04BF01430020B4F125
:10B2D000FD0C88BFBCF5E06F3FF6AFAEB5EB030CDD
:10B2E00004BFB6EB020C5FEA500C50F1000041EBDA
:10B2F000045170BD0EF0004E4EEA113114EB5C04A7
:10B30000C2BFD4EB0C0541EA045170BD41F4801179
:10B310004FF0000E013C90E645EA060E8DE60CEA81
:10B32000135594EA0C0F08BF95EA0C0F3FF43BAF9E
:10B3300094EA0C0F0AD150EA01347FF434AF95EA55
:10B340000C0F7FF425AF104619462CE795EA0C0F39
:10B3500006D152EA03353FF4FDAE1046194622E706
:10B3600050EA410618BF52EA43067FF4C5AE50EAE0
:10B3700041047FF40DAF52EA43057FF4EBAE12E7D0
:10B380004FF0FF3C06E000BF4FF0010C02E000BFB1
:10B390004FF0010C4DF804CD4FEA410C7FEA6C5C94
:10B3A0004FEA430C18BF7FEA6C5C1BD001B050EA37
:10B3B000410C0CBF52EA430C91EA030F02BF90EA22
:10B3C000020F0020704710F1000F91EA030F58BFE1
:10B3D000994208BF90422CBFD8176FEAE37040F043
:10B3E000010070474FEA410C7FEA6C5C02D150EAE1
:10B3F000013C07D14FEA430C7FEA6C5CD6D152EA9C
:10B40000033CD3D05DF8040B704700BF8446104660
:10B4100062468C461946634600E000BF01B5FFF75F
:10B42000B7FF002848BF10F1000F01BD4DF808ED2F
:10B43000FFF7F4FF0CBF012000205DF808FB00BF00
:10B440004DF808EDFFF7EAFF34BF012000205DF85A
:10B4500008FB00BF4DF808EDFFF7E0FF94BF0120A7
:10B4600000205DF808FB00BF4DF808EDFFF7CEFFA8
:10B4700094BF012000205DF808FB00BF4DF808EDE7
:10B48000FFF7C4FF34BF012000205DF808FB00BFB8
:10B490004FEA410C7FEA6C5C02D150EA013C0AD1D0
:10B4A0004FEA430C7FEA6C5C02D152EA033C02D1C2
:10B4B0004FF0000070474FF0010070474FEA410223
:10B4C00012F5001215D211D56FF47873B3EB6252F6
:10B4D00012D94FEAC12343F0004343EA505311F01D
:10B4E000004F23FA02F018BF404270474FF00000AF
:10B4F000704750EA013005D111F0004008BF6FF0ED
:10B50000004070474FF00000704700BF1FB51C4659
:10B51000094B1B680546D86852B1084B0091CDE92C
:10B52000013207492B46224600F028F800F0BAFD08
:10B53000044B1A46F2E700BF6000002088E60000D6
:10B5400095E600004BD20000014B1868704700BF21
:10B550006000002008B5074B044613B10021AFF38B
:10B560000080054B1868836A03B19847204601F0B4
:10B5700071FB00BF00000000C4E600000EB403B57C
:10B58000014603AB054853F8042B0068019300F013
:10B5900081F802B05DF804EB03B070476000002052
:10B5A00070B50D4E0D4CA41BA4100025A54209D169
:10B5B0000B4E0C4C01F050FBA41BA4100025A5421F
:10B5C00005D170BD56F8253098470135EEE756F89D
:10B5D000253098470135F2E7300200203002002084
:10B5E000300200204002002010B5431E0A44914260
:10B5F00000D110BD11F8014B03F8014FF7E7884265
:10B6000010B501EB020307D8421E99420AD011F887
:10B61000014B02F8014FF8E78342F5D98118D21A9D
:10B62000D34200D110BD13F8014D01F8014DF7E7E9
:10B6300002440346934200D1704703F8011BF9E727
:10B640009368013B002B10B4936008DA9469A3421D
:10B6500001DB0A2903D15DF8044B00F063BC1368D9
:10B66000581C1060197008465DF8044B7047F8B517
:10B6700006460F461446D518AC4201D1002007E01B
:10B680003A4614F8011B3046FFF7DAFF431CF3D1AA
:10B69000F8BD00002DE9F04F9DB00C46174603930E
:10B6A000064618B183690BB900F0F4FD7B4B9C4250
:10B6B00057D17468A38918075DD52369002B5AD028
:10B6C0000023099320238DF8293030238DF82A3068
:10B6D0004FF0010BB846454615F8013B0BB1252B41
:10B6E00054D1B8EB070A0BD053463A4621463046B0
:10B6F000FFF7BDFF013000F0C280099B534409935E
:10B7000098F80030002B00F0BA8000234FF0FF3291
:10B71000CDE90523049307938DF853301A93A84677
:10B72000052218F8011B5E4800F0C2FE049B78BB9E
:10B73000D90644BF20228DF853201A0744BF2B227C
:10B740008DF853202A782A2A2AD0079AA846002062
:10B750000A25414611F8013B303B092B69D960B3FA
:10B7600024E0504B9C4201D1B468A3E74E4B9C426D
:10B7700008BFF4689EE72146304600F025FC00280B
:10B780009ED04FF0FF301DB0BDE8F08FA846A2E775
:10B79000434A801A0BFA00F0184304904546BEE76E
:10B7A000039A111D12680391002A01DB079204E03D
:10B7B000524243F002030792049398F800302E2B74
:10B7C0000ED198F801302A2B38D1039B1A1D1B6823
:10B7D0000392002BB8BF4FF0FF3308F10208059326
:10B7E000324D98F800100322284600F061FE40B167
:10B7F0004023401B03FA00F0049B034308F10108B7
:10B80000049398F800102A488DF82810062208F1B1
:10B81000010700F04DFE002837D0264B1BBB039BD1
:10B82000073323F0070308330393099B4B44099321
:10B8300050E705FB0232012088468AE7002308F121
:10B840000108059319460A25404610F8012B303AA5
:10B85000092A03D9002BC3D00591C1E705FB0121BB
:10B8600001238046F0E703AB00932246124B04A964
:10B870003046AFF30080B0F1FF3F8146D5D1A389B8
:10B880005B063FF57EAF09987DE703AB0093224648
:10B89000094B04A9304600F087F8ECE71CE70000EC
:10B8A000C8E600003CE70000FCE60000CEE6000031
:10B8B000D2E60000000000006FB600002DE9F0475E
:10B8C00091461F468A680B69DDF820809342B8BF15
:10B8D0001346C9F8003091F8432006460C4612B1D1
:10B8E0000133C9F800302368990642BFD9F8003007
:10B8F0000233C9F80030256815F0060507D104F1B8
:10B90000190AE368D9F800209B1AAB4228DC94F8A6
:10B9100043302268003318BF012392062DD404F16E
:10B92000430239463046C047013020D02368E568DD
:10B93000D9F8002003F00603042B08BFAD1AA36852
:10B9400022690CBF25EAE57500259342C4BF9B1A06
:10B95000ED184FF000091A344D451AD1002008E0C7
:10B960000123524639463046C047013003D14FF0DB
:10B97000FF30BDE8F0870135C3E7E1185A1C3020DD
:10B9800081F84300224494F8451082F843100233B2
:10B99000C5E70123224639463046C0470130E6D08C
:10B9A00009F10109D8E700002DE9F04301F1430C4A
:10B9B0000C46097E85B06E291746064698460C9AB5
:10B9C00000F0B38022D8632936D00AD8002900F0CD
:10B9D000B980582900F0838004F1420584F84210B0
:10B9E00032E0642901D06929F6D120681368050680
:10B9F00003F104012AD51B681160002B03DA2D2204
:10BA00005B4284F843206F480A2239E0732900F032
:10BA10009D8008D86F2920D07029DDD1236843F09C
:10BA20002003236003E0752917D07829D4D1782327
:10BA300084F84530644855E01368191D1B6811608F
:10BA400004F1420584F8423001238CE01B68116048
:10BA500010F0400F18BF1BB2CFE713682568181D00
:10BA60001060280601D51B6802E06806FBD51B881C
:10BA700054486F2914BF0A220822002184F8431079
:10BA80006568A560002DC0F29580216821F0040151
:10BA90002160002B3DD1002D40F08E806546082AA4
:10BAA0000BD12368DB0708D5236962689A42DEBFA1
:10BAB000302305F8013C05F1FF35ACEB05032361AC
:10BAC000CDF800803B4603AA21463046FFF7F6FE3C
:10BAD00001304DD14FF0FF3005B0BDE8F08339485B
:10BAE00084F84510136821681D1D1B6815600A063F
:10BAF0000BD5CA0744BF41F0200121601BB9226861
:10BB000022F0200222601022B7E74D0648BF9BB208
:10BB1000EFE76546B3FBF2F102FB1133C35C05F8B6
:10BB2000013D0B460029F5D1B9E713682568616925
:10BB3000181D106028061B6801D5196002E06A060E
:10BB4000FBD51980002323616546B9E71368191DE9
:10BB500011601D6862680021284600F0A9FC08B148
:10BB6000401B606063682361002384F84330A7E7CB
:10BB700023692A4639463046C0470130AAD0236897
:10BB80009B0713D4E068039B9842B8BF1846A3E70D
:10BB900001234A4639463046C04701309AD0013524
:10BBA000E368039A9B1AAB42F2DCEBE7002504F151
:10BBB0001909F5E7002BACD1037884F8423004F181
:10BBC00042056CE7D9E60000EAE6000038B50D4B07
:10BBD0001C68A36B05467BB9182000F04DFC0A4A8F
:10BBE0000A4BA063C0E90023094B83600B238381C8
:10BBF00001220023C0E90423A36B00221D615A61C6
:10BC000038BD00BF600000200E33CDAB34126DE6AE
:10BC1000ECDE050038B5134B1C68A36B7BB918200C
:10BC200000F02AFC104A114BA063C0E90023104B1E
:10BC300083600B23838101220023C0E90423A16BCD
:10BC40000C480A694B690C4C504304FB0300A2FBEF
:10BC500004230344541C43F10005C1E9044525F0C5
:10BC6000004038BD600000200E33CDAB34126DE6CD
:10BC7000ECDE05002DF451582D7F954C0CB430B5F9
:10BC8000174B0C1E9DB01D6808DA8B232B604FF0FC
:10BC9000FF301DB0BDE8304002B070474FF4027372
:10BCA000ADF8143014BF04F1FF3323460493079317
:10BCB0004FF6FF7302900690ADF81630209A21AB34
:10BCC00002A92846019300F06BFD431CBCBF8B23E7
:10BCD0002B60002CDDD0029B00221A70D9E700BF38
:10BCE000600000200EB400B59CB01DAB0290069021
:10BCF0006FF00041094807910491094953F8042B5A
:10BD000005910068019302A900F04AFD029B002200
:10BD10001A701CB05DF804EB03B07047600000209F
:10BD20000802FFFF10B503461A785C1C3AB9013BC4
:10BD300011F8012B03F8012F002AF9D110BD234679
:10BD4000F2E7C9B2034610F8012B1AB18A42F9D1C1
:10BD500018467047002918BF0023F9E710F8012B97
:10BD600011F8013B012A28BF9A42F7D0D01A704738
:10BD7000034613F8012B002AFBD1181A013870472B
:10BD800010B56AB10139841810F8013B11F8012F80
:10BD9000934203D1A04201D0002BF5D1981A10BDD7
:10BDA0001046FCE770B50139044602B970BD234660
:10BDB00011F8015F03F8015B561E2DB91444A3422C
:10BDC000F4D003F8015BFAE71C463246EDE7F0B524
:10BDD00003787BB1044623782046661C7BB14A1E5B
:10BDE000631E12F8015F4DB113F8017FAF42344674
:10BDF000F7D0F0E70B78002B18BF0020F0BD1846F5
:10BE0000FCE72DE9F0478046894692461E460F46DC
:10BE10003D46089815F8014B00F0C6FA20444378D7
:10BE200013F0080332D12D2C32D17C78BD1C0122B5
:10BE3000002E5DD0102E09D1302C07D12B7803F0C5
:10BE4000DF03582B4FD16C7810260235002A14BF1F
:10BE50004FF000416FF000410027B1FBF6FC38467F
:10BE600006FB1C1EA4F13003092B17D81C46A64262
:10BE700023DD7B1C07D084451CD301D1A64519DBEB
:10BE800000FB0640012715F8014BEBE72F46BFE703
:10BE90002B2C04BFBD1C7C781A46C9E7A4F14103D2
:10BEA000192B01D8373CE2E7A4F16103192B04D820
:10BEB000573CDCE74FF0FF37E5E77B1C08D1222336
:10BEC000C8F800300846BAF1000F07D1BDE8F08786
:10BED00002B14042BAF1000FF8D00FB105F1FF39BD
:10BEE000CAF80090F2E73024002EAFD10826ADE763
:10BEF000302CA3D00A26A9E7084B37B51C68084D9B
:10BF0000236A002B08BF2B46009313460A460146BE
:10BF10002046FFF776FF03B030BD00BF6000002071
:10BF2000C4000020F8B50E461446054618B18369D2
:10BF30000BB900F0AFF9214B9C422AD16C68A36980
:10BF4000A360A3891A072ED5236963B323692068E8
:10BF5000C01A6369F6B28342374604DC214628469C
:10BF600000F02EF928BBA368013BA36023685A1C8C
:10BF700022601E7063690130834204D0A389DB070D
:10BF800019D50A2E17D12146284600F019F990B18B
:10BF90000FE00B4B9C4201D1AC68D0E7094B9C42AF
:10BFA00008BFEC68CBE72146284600F00DF80028D2
:10BFB000CCD04FF0FF373846F8BD00BF1CE700007B
:10BFC0003CE70000FCE60000324B70B51D680646F9
:10BFD0000C4625B1AB6913B9284600F05BF92E4B2E
:10BFE0009C420FD16C68B4F90C309AB215072CD46E
:10BFF000D00611D40922326043F04003A3814FF0F0
:10C00000FF303EE0254B9C4201D1AC68EBE7244B6E
:10C010009C4208BFEC68E6E7510712D5616B41B15D
:10C0200004F14403994202D0304600F091FA002313
:10C030006363A38923F02403A3810023636023693E
:10C040002360A38943F00803A38123694BB9A38923
:10C0500003F42073B3F5007F03D02146304600F08F
:10C06000CBF9A28912F001030CD00023A36063690D
:10C070005B42A361236953B9B4F90C3013F080001B
:10C08000BAD170BD920758BF6369A360F2E7002080
:10C09000F7E700BF600000201CE700003CE700005D
:10C0A000FCE6000008B5062000F0A8FC012000F026
:10C0B000D1FD00008A892DE9F041054610070C46A4
:10C0C00058D44B68002B05DC0B6C002B02DC0020E5
:10C0D000BDE8F081E66A002EF9D0002312F4805208
:10C0E0002F68216A2B6032D0606DA3895A0705D56D
:10C0F0006368C01A636B0BB1236CC01A002302463D
:10C10000E66A216A2846B047431CA38906D12968FC
:10C110001D2948D8294ACA40D60744D50022626062
:10C12000D9042269226004D5421C01D12B6803B9CD
:10C130006065616B2F600029C9D004F14403994206
:10C1400002D0284600F004FA00206063C0E7012313
:10C150002846B047411CC8D12B68002BC5D01D2BE9
:10C1600001D0162B01D12F60B1E7A38943F0400322
:10C17000A381ADE70F69002FA9D093070E6808BF10
:10C180004B690F6018BF0023A6EB07088B60B8F15E
:10C19000000F9CDD43463A46216AA66A2846B0470E
:10C1A000002806DCA38943F04003A3814FF0FF3051
:10C1B0008EE70744A8EB0008E9E700BF0100402034
:10C1C00038B50B6905460C46DBB118B183690BB96C
:10C1D00000F060F80C4B9C4209D16C68B4F90C304B
:10C1E0007BB121462846BDE83840FFF763BF074BC7
:10C1F0009C4201D1AC68F1E7054B9C4208BFEC685A
:10C20000ECE7002038BD00BF1CE700003CE7000061
:10C21000FCE60000002310B50446C0E9003383604B
:10C2200081814366C281C0E90433836119460822D3
:10C230005C30FFF7FDF9054B6362054BA362054BCC
:10C24000E362054B2462236310BD00BF35CA0000C2
:10C2500057CA00008FCA0000B3CA0000014900F0AD
:10C2600085B800BFC1C1000070B54A1E682555439E
:10C270000E4605F1740100F0B9F9044640B1002101
:10C28000C0E900160C30A06005F16802FFF7D0F994
:10C29000204670BD836910B5044633BBC0E9123334
:10C2A0000365124B124A1B688262984204BF012345
:10C2B000836100F01FF86060204600F01BF8A0606A
:10C2C000204600F017F80022E06004216068FFF7C4
:10C2D000A1FF01220921A068FFF79CFF0222122181
:10C2E000E068FFF797FF0123A36110BDC4E60000DB
:10C2F0005DC20000F8B51B4B1E68B369074613B951
:10C300003046FFF7C7FF4836D6E90134013B03D575
:10C31000336833B13668F7E7B4F90C506DB168345F
:10C32000F4E704213846FFF79FFF30600028F1D181
:10C330000C233B6004462046F8BD0B4B6566C4E900
:10C340000055A560C4E90335C4E90555082229460E
:10C3500004F15C00FFF76CF9C4E90D55C4E912550E
:10C36000E9E700BFC4E600000100FFFF2DE9F84344
:10C370008046894600F14804002614B93046BDE8DD
:10C38000F883D4E90175013F01D52468F5E7AB894D
:10C39000012B07D9B5F90E30013303D029464046A9
:10C3A000C84706436835EEE7D0F8EC00704770B533
:10C3B0000E46B1F90E10002996B014461D4607DA54
:10C3C00000232B60B3891A0610D44FF480630EE06B
:10C3D0006A4600F0A1FB0028F2DB019A02F47042E9
:10C3E000A2F500535A425A412A60EEE7402300204A
:10C3F000236016B070BD00008B8973B59D0706469B
:10C400000C4607D504F147032360236101236361D0
:10C4100002B070BD01AB6A46FFF7C9FF009905463F
:10C42000304600F0E3F848B9B4F90C309A05EFD47F
:10C4300023F0030343F00203A381E3E70D4BB36250
:10C44000A389206043F08003A381009B6361019B6B
:10C4500020615BB1B4F90E10304600F06FFB28B1DB
:10C46000A38923F0030343F00103A381A3891D43A0
:10C47000A581CDE75DC20000024B0146186800F0BF
:10C48000B5B800BF6000002082B001B901A942B177
:10C490004BB113780B601278101C18BF012002B04A
:10C4A00070471046FBE76FF00100F8E7000000005E
:10C4B00001F0FF01102A2BDB10F0070F08D010F855
:10C4C000013B013A8B422DD010F0070F42B3F6D159
:10C4D000F0B441EA012141EA014122F007047FF072
:10C4E00000070023F0E80256083C85EA010586EAC9
:10C4F000010685FA47F5A3FA87F586FA47F6A5FA05
:10C5000087F68EB9EED1F0BC01F0FF0102F0070210
:10C5100032B110F8013B013A83EA010313B1F8D1BB
:10C520000020704701387047002D06BF354603389C
:10C53000073815F0010F07D1013015F4807F02BFD5
:10C54000013015F4C03F0130F0BC0138704700BF26
:10C5500038B50546002945D051F8043C0C1F002B86
:10C56000B8BFE41800F00CFB1F4A1368104633B93B
:10C57000636014602846BDE8384000F002BBA34267
:10C580000CD921686218934204BF1A685B68636023
:10C5900004BF521822600460ECE713465A680AB1DF
:10C5A000A242FAD919685818A0420BD12068014458
:10C5B000581882421960DDD1106852685A600144EF
:10C5C0001960D7E702D90C232B60D3E72068211824
:10C5D0008A4204BF11685268626004BF0918216072
:10C5E0005C60C7E738BD00BF247D012070B5CD1C5D
:10C5F00025F0030508350C2D38BF0C25002D064607
:10C6000001DBA94203D90C233360002070BD00F088
:10C61000B7FA214A1468214691B9204C23681BB906
:10C62000304600F0B3F920602946304600F0AEF9FC
:10C63000431C24D10C233360304600F0A2FAE4E717
:10C640000B685B1B18D40B2B0FD90B60CD50CC188B
:10C65000304600F096FA04F10B00231D20F007008D
:10C66000C31AD3D05A42E250D0E78C424B6816BF6F
:10C67000636013600C46EBE70C464968CCE7C41CCA
:10C6800024F00304A04205D0211A304600F07EF9C0
:10C690000130CFD02560DBE7247D0120287D0120FB
:10C6A000F8B5074614460E4621B91146BDE8F840D4
:10C6B000FFF79CBF22B9FFF74BFF25462846F8BD80
:10C6C00000F060FAA0420FD221463846FFF78EFFF5
:10C6D00005460028F2D031462246FEF785FF314656
:10C6E0003846FFF735FFE9E73546E7E72DE9F0473C
:10C6F0008E689E4282460C469046994637D88A8973
:10C7000012F4906F31D0256809696F1A65690223A8
:10C7100005EB450595FBF3F509F101033B449D420B
:10C7200038BF1D46530530D52946FFF75FFF064643
:10C7300050B90C23CAF80030A38943F04003A38109
:10C740004FF0FF30BDE8F0873A462169FEF74CFF15
:10C75000A38923F4906343F08003A381266165617C
:10C760003E44ED1B2660A5604E464E4500D94E4620
:10C77000324641462068FEF742FFA3689B1BA36038
:10C7800023681E4426600020DCE72A46FFF788FF66
:10C7900006460028E2D121695046FFF7D9FEC8E7D6
:10C7A0002DE9F04F9DB0804603938B891D060C4602
:10C7B00016460FD50B696BB94021FFF717FF2060B4
:10C7C000206128B90C23C8F800304FF0FF30C7E0D3
:10C7D000402363610023099320238DF829303023FF
:10C7E0008DF82A304FF0010B37463D4615F8013BD6
:10C7F0000BB1252B3ED1B7EB060A0BD05346324680
:10C8000021464046FFF772FF013000F0A480099BEB
:10C81000534409933B78002B00F09D8000234FF098
:10C82000FF32CDE90523049307938DF853301A9313
:10C830002F46052217F8011B4F48FFF739FE049BCE
:10C84000D0B9D90644BF20228DF853201A0744BF1F
:10C850002B228DF853202A782A2A15D0079A2F46A2
:10C8600000200A25394611F8013B303B092B4DD9F0
:10C87000B8B10FE02F46B8E73F4A801A0BFA00F034
:10C88000184304903D46D3E7039A111D12680391A3
:10C89000002A01DB079204E0524243F002030792B0
:10C8A00004933B782E2B0CD17B782A2B33D1039B1E
:10C8B0001A1D1B680392002BB8BF4FF0FF330237DD
:10C8C00005932E4D397803222846FFF7F1FD38B144
:10C8D0004023401B03FA00F0049B034301370493F9
:10C8E000397827488DF8281006227E1CFFF7E0FDD6
:10C8F000002838D0234B13BB039B073323F00703D7
:10C9000008330393099B4B4409936DE705FB0232FF
:10C9100001200F46A6E700230137059319460A2593
:10C92000384610F8012B303A092A03D9002BC8D019
:10C930000591C6E705FB012101230746F0E703AB9C
:10C9400000932246104B04A94046AFF30080B0F19B
:10C95000FF3F8146D6D1A3895B063FF536AF0998E4
:10C960001DB0BDE8F08F03AB00932246064B04A92F
:10C970004046FFF719F8EAE7C8E60000CEE60000F7
:10C98000D2E6000000000000EDC6000038B5064CFD
:10C99000002305460846236000F046F9431C02D1F7
:10C9A000236803B12B6038BDB89001201F2938B52A
:10C9B00004460D4604D9162303604FF0FF3038BDFE
:10C9C000426C12B152F821304BB9204600F030F8D9
:10C9D0002A4601462046BDE8384000F017B8012B32
:10C9E0000AD0591C03D1162303600120E7E7002475
:10C9F00042F82540284698470020E0E7024B0146D0
:10CA00001868FFF7D3BF00BF6000002038B5074C9F
:10CA10000023054608461146236000F0EDF8431C4C
:10CA200002D1236803B12B6038BD00BFB89001204C
:10CA300000F0D2B810B50C46B1F90E1000F0AAF80B
:10CA40000028ABBF636DA3891B1823F48053ACBFD0
:10CA50006365A38110BD2DE9F0411F468B89DB057D
:10CA600005460C46164605D502230022B1F90E10E4
:10CA700000F074F8A389B4F90E1023F48053A38155
:10CA800032463B462846BDE8F04100F023B810B5D9
:10CA90000C46B1F90E1000F061F8431CA38915BFD4
:10CAA000606523F4805343F48053A38118BFA381AE
:10CAB00010BDB1F90E1000F01FB849B1FF2A85BFB3
:10CAC0008A2303600A704FF0FF3098BF012070473F
:10CAD0000846704738B5074C0546084611460022FF
:10CAE00022601A4600F0AEF8431C02D1236803B15D
:10CAF0002B6038BDB890012038B5064C00230546A0
:10CB00000846236000F058F8431C02D1236803B1A3
:10CB10002B6038BDB890012038B5074C002305467E
:10CB200008461146236000F04FF8431C02D12368E9
:10CB300003B12B6038BD00BFB890012038B5064C5A
:10CB4000002305460846236000F04EF8431C02D13E
:10CB5000236803B12B6038BDB890012038B5074C6D
:10CB6000054608461146002222601A4600F04CF89D
:10CB7000431C02D1236803B12B6038BDB89001205B
:10CB80007047704751F8043C181F002BBCBF0B586E
:10CB9000C018704738B5074C0546084611460022B4
:10CBA00022601A4600F038F8431C02D1236803B112
:10CBB0002B6038BDB8900120024B58221A604FF00C
:10CBC000FF307047B8900120024B58221A604FF096
:10CBD000FF307047B8900120024B58221A604FF086
:10CBE000FF307047B8900120024B58221A60002095
:10CBF000704700BFB8900120024B58221A604FF0D6
:10CC0000FF307047B8900120024B58221A604FF055
:10CC1000FF307047B8900120024B58221A604FF045
:10CC2000FF307047B8900120044A05491368002B73
:10CC300008BF0B4618441060184670472C7D012031
:10CC4000C0900120024B58221A604FF0FF3070470D
:10CC5000B8900120FEE700BFF8B500BFF8BC08BCE3
:10CC60009E467047F8B500BFF8BC08BC9E467047AA
:10CC700064617461000000000ECD00001D0300001F
:10CC800017CD0000CD0B00001DCD00000D040000ED
:10CC900025CD0000890C00002CCD0000B50D000052
:10CCA00031CD00001906000037CD0000F10700006B
:10CCB00042CD00007704000047CD0000F10F0000D6
:10CCC00053CD00004F0300005DCD0000F90A0000C5
:10CCD0006BCD00009507000078CD00007D090000B5
:10CCE00084CD00005D07000072616E646F6D0061AD
:10CCF0006C6C006C61737400300066616C7365006D
:10CD00007472756500252E3135732E2E2E006D61DF
:10CD10006B654C6973740072616E67650061646471
:10CD20004C6173740064656C657465006A6F696E4C
:10CD30000073706C697400636F707946726F6D5424
:10CD40006F0066696E64006A6F696E537472696E13
:10CD5000677300756E69636F6465417400756E6911
:10CD6000636F6465537472696E67006E65774279AC
:10CD700074654172726179006173427974654172C0
:10CD800072617900667265654D656D6F727900003C
:10CD9000FDCD0000D114000002CE0000EB14000015
:10CDA00025CD0000EF14000008CE0000D5140000CF
:10CDB00012CE0000F31400001BCE0000F714000098
:10CDC00025CE0000FB1400002ECE0000FF14000052
:10CDD00039CE00000315000045CE0000D914000034
:10CDE0004ECE0000E314000058CE0000DD14000019
:10CDF00063CE0000E714000066696C65006F706523
:10CE00006E00636C6F736500656E644F6646696C97
:10CE10006500726561644C696E65007265616442AB
:10CE2000797465730072656164496E746F00617036
:10CE300070656E644C696E6500617070656E644209
:10CE4000797465730066696C6553697A65007374FB
:10CE50006172744C697374006E657874496E4C69C4
:10CE600073740073797374656D496E666F000000AA
:10CE7000F418000004190000181900008C190000B3
:10CE8000BE190000EE190000201A0000421A00002E
:10CE9000821A0000BC1A00000C1B00004A1B000094
:10CEA000AA1B0000EA1B00000A1C00003E1C000038
:10CEB0007E1C0000A01C0000CA1C0000F41C000026
:10CEC000E0320000B81D0000801E0000F21E0000CD
:10CED0003C1F0000A01F0000BC1F0000DA1F000064
:10CEE0001821000058210000CA210000F82100008C
:10CEF0002822000056220000BA2200001E23000053
:10CF000080230000E223000056240000D02400000B
:10CF10003025000090250000C62500000A260000EC
:10CF20005026000096260000E82600003E2700005C
:10CF30007C2700000C280000402800008628000004
:10CF4000CC280000122900004C2900009229000082
:10CF5000D8290000342B0000CA1C00003E1C000031
:10CF60004C2A0000F4180000802A0000A62A0000C5
:10CF7000DA2A0000002B0000F4180000F41800006A
:10CF8000F4180000F4180000AA2B0000E62B0000A3
:10CF9000262C0000762C00009C2C00000A2D00009E
:10CFA000542D0000842D0000F4180000F418000037
:10CFB000A22D0000D42D0000062E00003A2E000005
:10CFC0005E2E0000BC2E0000E02E0000022F0000AC
:10CFD000242F0000562F0000882F0000AC2F0000E7
:10CFE000D02F00000230000026300000F4180000AE
:10CFF000F4180000F4180000F4180000F418000001
:10D00000583000007E300000A4300000CA3000001C
:10D01000F030000024310000583100008C31000055
:10D02000C0310000E63100000C3200004032000048
:10D03000F4180000F4180000F4180000F4180000C0
:10D04000F4180000F4180000F4180000F4180000B0
:10D05000F4180000F4180000F4180000F4180000A0
:10D0600066320000663200009A330000CA330000C6
:10D070005B2564206974656D206C6973745D00289C
:10D0800025642062797465732900286F626A65637C
:10D090007420747970653A202564290053746163A3
:10D0A0006B20756E646572666C6F7700626F6F6C73
:10D0B00065616E006E756D62657200737472696E83
:10D0C00067006C69737400627974652061727261C3
:10D0D0007900000007000000030000006DD100008F
:10D0E000E934000075D10000953500007ED10000C4
:10D0F000893D000087D10000ED34000090D1000090
:10D100008D3D000098D1000029370000A1D100001A
:10D11000E5370000AFD1000075360000BAD100003D
:10D12000013F0000C5D1000039370000D0D1000018
:10D13000C53E0000DCD1000021360000E8D100002F
:10D140003B40000000000000010000000200000061
:10D1500003000000040000000A0000001D000000A1
:10D160006D6963726F3A6269742076320068617328
:10D17000546F6E6500706C6179546F6E6500686104
:10D1800073536572766F00736574536572766F00C2
:10D19000646163496E6974006461635772697465A0
:10D1A00000736F66745772697465427974650073B1
:10D1B0007175617265576176650073657455736545
:10D1C000724C454400616E616C6F6752656164002A
:10D1D000616E616C6F675772697465006469676935
:10D1E00074616C52656164006469676974616C574D
:10D1F0007269746500474320746F6F6B202564204B
:10D2000075736563733B20667265652025642077BE
:10D210006F726473003C496E74656765723E003CD2
:10D220004C6973743E003C4F626A6563743E003C17
:10D230004279746541727261793E000D0A564D2043
:10D2400050616E69633A2025730D0A006D6973633E
:10D2500000000000A1D200005F4A0000AAD2000036
:10D26000594B0000B2D20000154B0000B6D20000AE
:10D27000E94A0000BBD2000065180000CAD20000D5
:10D28000AD490000D2D200004F490000DCD20000BE
:10D29000E1480000E8D20000E34700006E756C6CC6
:10D2A00000686578546F496E740072657363616CD1
:10D2B000650073696E00737172740062726F6164ED
:10D2C00063617374546F494445006A736F6E4765B8
:10D2D00074006A736F6E436F756E74006A736F6E5D
:10D2E00056616C75654174006A736F6E4B65794168
:10D2F00074000000E8D30000C94B0000F0D3000028
:10D30000CD4B0000FAD30000DF4B000003D4000037
:10D31000E54B00000ED40000EB4B00001AD40000D7
:10D32000F14B000028D40000F74B000030D400007F
:10D33000FD4B000036D40000034C00004BD400002D
:10D34000094C000060D400000F4C00006CD40000B9
:10D35000154C00007CD400001B4C000088D4000059
:10D36000214C000095D40000274C00009ED4000002
:10D370002D4C0000A6D40000334C0000B4D40000B3
:10D38000394C0000C5D400003F4C0000D8D4000048
:10D39000454C0000E6D400004B4C0000F5D40000E2
:10D3A000514C000008D50000574C00001ED500006D
:10D3B0005D4C00002AD50000634C00003AD5000007
:10D3C000694C000049D500006F4C000057D50000A3
:10D3D000754C00005FD50000D34B000067D50000FE
:10D3E000D94B00006E657400686173576946690027
:10D3F0007374617274576946690073746F7057690A
:10D4000046690077696669537461747573006D7954
:10D41000495041646472657373007374617274532C
:10D420005349447363616E00676574535349440004
:10D430006D794D41430068747470536572766572FE
:10D440004765745265717565737400726573706FAA
:10D450006E64546F487474705265717565737400AE
:10D4600068747470436F6E6E656374006874747072
:10D470004973436F6E6E656374656400687474709D
:10D480005265717565737400687474705265737059
:10D490006F6E7365007564705374617274007564A7
:10D4A0007053746F700075647053656E645061637F
:10D4B0006B6574007564705265636569766550616B
:10D4C000636B65740075647052656D6F7465495067
:10D4D000416464726573730075647052656D6F7436
:10D4E00065506F727400776562536F636B65745338
:10D4F0007461727400776562536F636B65744C611D
:10D5000073744576656E7400776562536F636B65FF
:10D510007453656E64546F436C69656E74004D514D
:10D520005454436F6E6E656374004D515454497387
:10D53000436F6E6E6563746564004D515454446965
:10D5400073636F6E6E656374004D5154544C617318
:10D55000744576656E74004D515454507562004D9B
:10D56000515454537562004D515454556E73756245
:10D570000000000004000000030000000A0000009A
:10D580000700000006000000000000000008080876
:10D5900000080A4A4000000A5FEA5FEA0ED92ED36B
:10D5A0006E19324489330C924C924D0808000000E9
:10D5B00004880808040804848488000A448A400017
:10D5C000048EC480000000048800000EC00000002B
:10D5D00000080001224488100C9252524C048C84A2
:10D5E000848E1C824C901E1EC244924C06CA525F0E
:10D5F000E21FF01EC13E02448ED12E1FE24488106D
:10D600000ED12ED12E0ED12EC488000800080000A5
:10D61000048004880244880482000EC00EC00804FE
:10D620008244880ED126C0040ED135B36C0C925EB4
:10D63000D2521C925C925C0ED010100E1C92525270
:10D640005C1ED01C901E1ED01C90100ED013712E8C
:10D6500012525ED2521C8808081C1FE242524C1221
:10D6600054981492101010101E113B75B1311139DD
:10D6700035B3710C9252524C1C925C90100C925229
:10D680004C861C925C92510ED00C825C1FE4848408
:10D6900084125252524C1131312A44113135BB712E
:10D6A00012524C9252112A4484841EC488101E0EB9
:10D6B000C808080E10080482410EC242424E048A75
:10D6C000400000000000001F0804800000000ED28F
:10D6D000524F10101C925C000ED0100E02424ED21F
:10D6E0004E0C925C900E06C81C88080ED24EC24C9E
:10D6F00010101C92520800080808024002424C1008
:10D70000149814920808080806001B75B131001C13
:10D71000925252000C92524C001C925C90000ED21D
:10D720004EC2000ED010100006C8049808080EC89B
:10D7300007001252524F0011312A4400113135BBFB
:10D7400000124C8C9200112A4498001EC4881E06B8
:10D75000C48C8486080808080818080C881800007B
:10D760000C836000000000000100000002000000C7
:10D770000300000004000000050000000600000097
:10D780000700000008000000090000000A00000077
:10D790000B0000000C0000000D0000000E00000057
:10D7A0000F00000010000000120000001400000034
:10D7B00016000000180000001A0000001C00000005
:10D7C0001E000000200000002300000026000000D2
:10D7D000290000002C0000002F0000003200000093
:10D7E000360000003A0000003E0000004200000049
:10D7F000460000004B0000005000000055000000F3
:10D800005A00000061000000680000006F00000086
:10D81000760000007D000000840000008B00000006
:10D820009200000099000000A0000000A700000086
:10D83000AE000000B5000000BC000000C300000006
:10D84000CA000000D1000000D8000000DF00000086
:10D85000E6000000ED000000F4000000FB00000006
:10D86000FF000000000000000200000004000000B3
:10D870000100000003000000E4D80000914C00000B
:10D88000EFD80000F1520000F9D80000BD4E0000B2
:10D8900006D90000655000000DD90000B15000000D
:10D8A00016D900000151000022D90000F54F0000F8
:10D8B00033D90000814F000043D90000F951000026
:10D8C00050D90000494F000015000000160000006C
:10D8D0001700000018000000190000006469737050
:10D8E0006C6179006C696768744C6576656C006D75
:10D8F00062446973706C6179006D62446973706C25
:10D9000061794F6666006D62506C6F74006D625590
:10D910006E706C6F74006D624472617753686170F1
:10D9200065006D625368617065466F724C65747412
:10D930006572006D62456E61626C65446973706CFE
:10D940006179006E656F506978656C53656E64002F
:10D950006E656F506978656C53657450696E004EE2
:10D960006F7420656E6F75676820726F6F6D2065CC
:10D9700076656E20616674657220636F6D70616399
:10D9800074696F6E00436F6D7061637465642046E7
:10D990006C61736820636F64652073746F72650ACD
:10D9A0002564206279746573207573656420282569
:10D9B00064252529206F6620256400426164207259
:10D9C00065636F726420666F756E6420647572693A
:10D9D0006E6720696E697469616C697A6174696FD8
:10D9E0006E00256420256420256420282564207786
:10D9F0006F72647329002564207265636F726473AB
:10DA00002C20256420776F7264732C206D61784917
:10DA1000442025642C20636F6D70616374696F6EA0
:10DA2000206379636C657320256400526573746F9D
:10DA30007265642025642073637269707473005387
:10DA400074617274656400726164696F0000000043
:10DA5000E5DA0000C15A0000F2DA0000955D00002E
:10DA600002DB0000295D000010DB0000F55E000015
:10DA70001BDB0000D95A00002BDB00005D5B0000BF
:10DA80003FDB0000415B00004EDB00009F600000B8
:10DA90005ADB00001B60000063DB0000BF5F00007A
:10DAA0006EDB0000415F000079DB0000795F000061
:10DAB00082DB0000A95F00008BDB0000E95A000058
:10DAC0009ADB00001D5B0000A3DB0000F95A000098
:10DAD00025303878006E6F6E65006F74686572006F
:10DAE000706169720064697361626C655261646936
:10DAF0006F006D657373616765526563656976650F
:10DB000064007061636B6574526563656976650076
:10DB10007061636B657453656E64007265636569FB
:10DB2000766564496E7465676572007265636569E0
:10DB30007665644D657373616765547970650072CD
:10DB400065636569766564537472696E67007365B1
:10DB50006E64496E74656765720073656E645061CA
:10DB600069720073656E64537472696E67007365E1
:10DB7000744368616E6E656C0073657447726F758F
:10DB80007000736574506F776572007369676E61BA
:10DB90006C537472656E677468006465766963655A
:10DBA0004944006C6173744D6573736167654944E2
:10DBB00000556E6B6E6F776E207072696D69746957
:10DBC0007665205B25733A25735D00000000000038
:10DBD000963007772C610EEEBA51099919C46D077A
:10DBE0008FF46A7035A563E9A395649E3288DB0ED5
:10DBF000A4B8DC791EE9D5E088D9D2972B4CB609B8
:10DC0000BD7CB17E072DB8E7911DBF906410B71D94
:10DC1000F220B06A4871B9F3DE41BE847DD4DA1ACD
:10DC2000EBE4DD6D51B5D4F4C785D38356986C13FE
:10DC3000C0A86B647AF962FDECC9658A4F5C011477
:10DC4000D96C0663633D0FFAF50D088DC8206E3B55
:10DC50005E10694CE44160D5727167A2D1E4033C67
:10DC600047D4044BFD850DD26BB50AA5FAA8B5358E
:10DC70006C98B242D6C9BBDB40F9BCACE36CD8327D
:10DC8000755CDF45CF0DD6DC593DD1ABAC30D92624
:10DC90003A00DE518051D7C81661D0BFB5F4B42127
:10DCA00023C4B3569995BACF0FA5BDB89EB8022824
:10DCB0000888055FB2D90CC624E90BB1877C6F2FA9
:10DCC000114C6858AB1D61C13D2D66B69041DC76A4
:10DCD0000671DB01BC20D2982A10D5EF8985B1717D
:10DCE0001FB5B606A5E4BF9F33D4B8E8A2C907782C
:10DCF00034F9000F8EA8099618980EE1BB0D6A7FC3
:10DD00002D3D6D08976C6491015C63E6F4516B6B7B
:10DD100062616C1CD83065854E0062F2ED95066C30
:10DD20007BA5011BC1F4088257C40FF5C6D9B065A5
:10DD300050E9B712EAB8BE8B7C88B9FCDF1DDD6202
:10DD4000492DDA15F37CD38C654CD4FB5861B24D68
:10DD5000CE51B53A7400BCA3E230BBD441A5DF4A32
:10DD6000D795D83D6DC4D1A4FBF4D6D36AE96943F5
:10DD7000FCD96E34468867ADD0B860DA732D0444A0
:10DD8000E51D03335F4C0AAAC97C0DDD3C710550CB
:10DD9000AA41022710100BBE86200CC925B5685772
:10DDA000B3856F2009D466B99FE461CE0EF9DE5EBB
:10DDB00098C9D9292298D0B0B4A8D7C7173DB3596C
:10DDC000810DB42E3B5CBDB7AD6CBAC02083B8EDFD
:10DDD000B6B3BF9A0CE2B6039AD2B1743947D5EA0A
:10DDE000AF77D29D1526DB048316DC73120B63E339
:10DDF000843B64943E6A6D0DA85A6A7A0BCF0EE498
:10DE00009DFF099327AE000AB19E077D44930FF052
:10DE1000D2A3088768F2011EFEC206695D5762F749
:10DE2000CB67658071366C19E7066B6E761BD4FE86
:10DE3000E02BD3895A7ADA10CC4ADD676FDFB9F963
:10DE4000F9EFBE8E43BEB717D58EB060E8A3D6D625
:10DE50007E93D1A1C4C2D83852F2DF4FF167BBD153
:10DE60006757BCA6DD06B53F4B36B248DA2B0DD856
:10DE70004C1B0AAFF64A0336607A0441C3EF60DFF9
:10DE800055DF67A8EF8E6E3179BE69468CB361CBE2
:10DE90001A8366BCA0D26F2536E2685295770CCC07
:10DEA00003470BBBB91602222F260555BE3BBAC548
:10DEB000280BBDB2925AB42B046AB35CA7FFD7C239
:10DEC00031CFD0B58B9ED92C1DAEDE5BB0C2649B2A
:10DED00026F263EC9CA36A750A936D02A906099C5D
:10DEE0003F360EEB8567077213570005824ABF95D0
:10DEF000147AB8E2AE2BB17B381BB60C9B8ED29253
:10DF00000DBED5E5B7EFDC7C21DFDB0BD4D2D386A9
:10DF100042E2D4F1F8B3DD686E83DA1FCD16BE811C
:10DF20005B26B9F6E177B06F7747B718E65A0888ED
:10DF3000706A0FFFCA3B06665C0B0111FF9E658F7E
:10DF400069AE62F8D3FF6B6145CF6C1678E20AA028
:10DF5000EED20DD75483044EC2B30339612667A7AE
:10DF6000F71660D04D476949DB776E3E4A6AD1AEFD
:10DF7000DC5AD6D9660BDF40F03BD83753AEBCA98C
:10DF8000C59EBBDE7FCFB247E9FFB5301CF2BDBDF9
:10DF90008AC2BACA3093B353A6A3B4240536D0BA02
:10DFA0009306D7CD2957DE54BF67D9232E7A66B39F
:10DFB000B84A61C4021B685D942B6F2A37BE0BB44C
:10DFC000A18E0CC31BDF055A8DEF022D416C6C2016
:10DFD0007461736B732073746F7070656400763155
:10DFE000373500202573202573004D656D6F7279DC
:10DFF00020636C6561726564004E6F2066726565B2
:10E00000207461736B20656E747269657300000023
:10E0100090E000005D7B00009DE0000009730000BF
:10E02000A9E000002D7B0000AFE000003D7B000078
:10E03000B5E000004D7B0000BBE00000057A000069
:10E04000D1E00000597C0000DFE0000039730000DF
:10E05000E9E00000E97C0000F1E00000B177000099
:10E06000FAE00000897400000BE100007D750000FB
:10E0700017E100004174000020E10000B9740000C5
:10E0800028E10000D176000073656E736F72730033
:10E09000616363656C65726174696F6E0074656D50
:10E0A00070657261747572650074696C745800747F
:10E0B000696C74590074696C745A007365744163B7
:10E0C00063656C65726F6D6574657252616E6765CC
:10E0D000006D61676E657469634669656C640074A0
:10E0E0006F7563685265616400693263526561648B
:10E0F00000693263577269746500693263536574ED
:10E10000436C6F636B537065656400737069457829
:10E110006368616E6765007370695365747570003C
:10E1200072656164444854006D6963726F70686F12
:10E130006E650000FDCD00006D7F000002CE000086
:10E14000698000006BE100008D80000025CE00009A
:10E15000F17E000070E100000D81000076E100001A
:10E16000C57D000073657269616C00726561640051
:10E170007772697465007772697465427974657342
:10E180000000000008E20000A981000015E2000084
:10E19000AD8100001EE20000B981000028E200000D
:10E1A000BD81000031E20000C181000036E20000C4
:10E1B000C58100003BE20000C981000047E2000089
:10E1C000CD8100004EE20000D181000057E2000046
:10E1D000D58100005CE20000D981000068E2000007
:10E1E000DD81000073E20000E18100007EE20000BA
:10E1F000E581000088E20000B181000092E20000A9
:10E20000B5810000746674007365744261636B6C61
:10E210006967687400676574576964746800676546
:10E220007448656967687400736574506978656CD3
:10E23000006C696E65007265637400726F756E6460
:10E2400065645265637400636972636C650074721F
:10E2500069616E676C650074657874006D657267DE
:10E26000654269746D6170006472617742756666BB
:10E27000657200746674546F7563686564007466D3
:10E2800074546F7563685800746674546F7563686E
:10E290005900746674546F75636850726573737552
:10E2A0007265007661727300C8E200004D8600005E
:10E2B000D2E200002D860000DBE2000009860000AB
:10E2C000E7E2000099850000766172457869737411
:10E2D00073007661724E616D65640073657456619A
:10E2E000724E616D6564007661724E616D65466F58
:10E2F00072496E6465780057656C636F6D65207454
:10E300006F204D6963726F426C6F636B7321007095
:10E310005F73706920213D204E554C4C002F686F73
:10E320006D652F6769742F2E706C6174666F726DE6
:10E33000696F2F7061636B616765732F6672616DC2
:10E3400065776F726B2D61726475696E6F6E6F7237
:10E350006469636E7266352F6C6962726172696599
:10E36000732F5350492F5350492E637070005350F0
:10E3700049436C6173733A3A535049436C61737308
:10E38000284E52465F5350495F547970652A2C20BD
:10E3900075696E74385F742C2075696E74385F749B
:10E3A0002C2075696E74385F74290000000000002D
:10E3B0000000000021880000D98700000F880000BD
:10E3C000158800001B8800000D8800000200000076
:10E3D00003000000040000001F0000001C000000FB
:10E3E0000E000000250000000B0000000A000000E5
:10E3F000090000001E000000170000000C000000D3
:10E4000011000000010000000D00000022000000CB
:10E41000FFFFFFFFFFFFFFFF1A00000020000000CA
:10E4200015000000160000000F000000180000009A
:10E430001300000024000000000000001400000091
:10E440000500000010000000080000001900000096
:10E45000280000000600000000000000000000008E
:10E46000038E00001D950000798E0000858E00004F
:10E470007F8E0000018E0000F98D00008D8E00005F
:10E480001D8E0000F58D000000C00140001002400C
:10E490000020024000D00240000000000000304395
:10E4A00000000000000030C37371727400000000AF
:10E4B000FB21F93FFB2109407CD91240FB21194087
:10E4C0007A6A1F407CD92240BBFD2540FB212940B0
:10E4D0003A462C407A6A2F405C4731407CD9324022
:10E4E0009C6B3440BBFD3540DB8F3740FB2139400E
:10E4F0001BB43A403A463C405AD83D407A6A3F40C5
:10E500004C7E40405C4741406C1042407CD94240C8
:10E510008CA243409C6B4440AC344540BBFD45401D
:10E52000CBC64640DB8F4740EB584840FB21494073
:10E5300083F9A200444E6E00FC291500D157270034
:10E54000DD34F50062DBC0003C999500419043004A
:10E550006351FE00BBDEAB00B761C5003A6E24001C
:10E56000D24D42004906E00009EA2E001C92D1007B
:10E57000EB1DFE0029B11C00E83EA700F535820026
:10E5800044BB2E009CE98400B4267000417E5F00ED
:10E59000D6913900538339009CF439008B5F840095
:10E5A00028F9BD00F81F3B00DEFF97000F9805001B
:10E5B000112FEF000A5A8B006D1F6D00CF7E3600C1
:10E5C00009CB2700464FB7009E663F002DEA5F004B
:10E5D000BA277500E5EBC7003D7BF100F73907006E
:10E5E00092528A00FB6BEA001FB15F00085D8D004C
:10E5F000300356007BFC4600F0AB6B0020BCCF0024
:10E6000036F49A00E3A91D005E619100081BE60044
:10E6100085996500A0145F008D40680080D8FF00D8
:10E6200027734D0006063100CA561500C9A87300AD
:10E630007BE260006B8CC00000000040FB21F93FD2
:10E64000000000002D44743E000000809846F83C15
:10E650000000006051CC783B00000080831BF03943
:10E660000000004020257A38000000802282E33636
:10E67000000000001DF369350200000003000000E7
:10E6800004000000060000002C2066756E637469AB
:10E690006F6E3A2000617373657274696F6E202229
:10E6A000257322206661696C65643A2066696C6531
:10E6B00020222573222C206C696E65202564257329
:10E6C00025730A0064000020232D302B2000686C85
:10E6D0004C00656667454647003031323334353685
:10E6E00037383941424344454600303132333435BE
:10E6F00036373839616263646566000000000000E7
:10E700000000000000000000000000000000000009
:10E7100000000000000000000000000000000000F9
:10E7200000000000000000000000000000000000E9
:10E7300000000000000000000000000000000000D9
:10E7400000000000000000000000000000000000C9
:10E75000000000000000000000000000504F53497E
:10E760005800002020202020202020202828282891
:10E770002820202020202020202020202020202091
:10E7800020202088101010101010101010101010E1
:10E7900010101004040404040404040404101010F1
:10E7A000101010104141414141410101010101019D
:10E7B000010101010101010101010101010110102B
:10E7C0001010101042424242424202020202020271
:10E7D00002020202020202020202020202021010FD
:10E7E00010102000000000000000000000000000E9
:10E7F0000000000000000000000000000000000019
:10E800000000000000000000000000000000000008
:10E8100000000000000000000000000000000000F8
:10E8200000000000000000000000000000000000E8
:10E8300000000000000000000000000000000000D8
:10E8400000000000000000000000000000000000C8
:10E8500000000000000000000000000000000000B8
:08E860000000000000000000B0
:08E86800D819FF7F0100000038
:10E87000FFFFFFFFE803000001000000E803DC05E4
:10E88000DC05DC05DC050000FFFFFFFFFFFFFFFFED
:10E890001800000019FCFFFFFFFFFFFF020000004F
:10E8A00040420F00FFFF01FF030000000090D00373
:10E8B000FFFFFFFFFFFFFFFFFFFFFFFFFFFFFFFF68
:10E8C0000A00000001000000080000000100000034
:10E8D00064000020000000001CE700003CE700008E
:10E8E000FCE6000000000000000000000000000046
:10E8F0000000000000000000000000000000000018
:10E900000000000000000000000000000000000007
:10E9100000000000000000000000000000000000F7
:10E9200000000000000000000000000000000000E7
:10E930000000000043000000000000000000000094
:10E9400000000000000000000000000000000000C7
:10E950000000000043000000000000000000000074
:10E9600000000000000000000000000000000000A7
:10E970000000000043000000000000000000000054
:10E980000000000000000000000000000000000087
:10E990000000000043000000000000000000000034
:10E9A0000000000000000000000000000000000067
:10E9B0000000000043000000000000000000000014
:10E9C0000000000000000000000000000000000047
:10E9D00000000000430000000000000000000000F4
:10E9E0000000000000000000000000000000000027
:10E9F00000000000430000000000000000000000D4
:10EA00000000000000000000000000000000000006
:10EA100000000000BBCA000089C400000000000024
:10EA200062E700000CCD00004BD200004BD200008A
:10EA30004BD200004BD200004BD200004BD2000062
:10EA40004BD200004BD200004BD20000FFFFFFFF73
:10EA5000FFFFFFFFFFFFFFFFFFFF0000010041532B
:10EA600043494900000000000000000000000000D1
:10EA70000000000000000000000000000000415302
:10EA800043494900000000000000000000000000B1
:10EA90000000000000000000000000000000000076
:10EAA00025020000A5870000018C00008D90000069
:04EAB000010200005F
:0400000300008CBDB0
:00000001FF
